Component: ARM Compiler 5.06 update 7 (build 960) Tool: armlink [4d3601]

==============================================================================

Section Cross References

    startup_stm32f103xb.o(RESET) refers to startup_stm32f103xb.o(STACK) for __initial_sp
    startup_stm32f103xb.o(RESET) refers to startup_stm32f103xb.o(.text) for Reset_Handler
    startup_stm32f103xb.o(RESET) refers to stm32f1xx_it.o(i.NMI_Handler) for NMI_Handler
    startup_stm32f103xb.o(RESET) refers to stm32f1xx_it.o(i.HardFault_Handler) for HardFault_Handler
    startup_stm32f103xb.o(RESET) refers to stm32f1xx_it.o(i.MemManage_Handler) for MemManage_Handler
    startup_stm32f103xb.o(RESET) refers to stm32f1xx_it.o(i.BusFault_Handler) for BusFault_Handler
    startup_stm32f103xb.o(RESET) refers to stm32f1xx_it.o(i.UsageFault_Handler) for UsageFault_Handler
    startup_stm32f103xb.o(RESET) refers to stm32f1xx_it.o(i.SVC_Handler) for SVC_Handler
    startup_stm32f103xb.o(RESET) refers to stm32f1xx_it.o(i.DebugMon_Handler) for DebugMon_Handler
    startup_stm32f103xb.o(RESET) refers to stm32f1xx_it.o(i.PendSV_Handler) for PendSV_Handler
    startup_stm32f103xb.o(RESET) refers to stm32f1xx_it.o(i.SysTick_Handler) for SysTick_Handler
    startup_stm32f103xb.o(RESET) refers to stm32f1xx_it.o(i.DMA1_Channel2_IRQHandler) for DMA1_Channel2_IRQHandler
    startup_stm32f103xb.o(RESET) refers to stm32f1xx_it.o(i.DMA1_Channel3_IRQHandler) for DMA1_Channel3_IRQHandler
    startup_stm32f103xb.o(RESET) refers to stm32f1xx_it.o(i.DMA1_Channel5_IRQHandler) for DMA1_Channel5_IRQHandler
    startup_stm32f103xb.o(RESET) refers to stm32f1xx_it.o(i.DMA1_Channel6_IRQHandler) for DMA1_Channel6_IRQHandler
    startup_stm32f103xb.o(RESET) refers to stm32f1xx_it.o(i.DMA1_Channel7_IRQHandler) for DMA1_Channel7_IRQHandler
    startup_stm32f103xb.o(RESET) refers to stm32f1xx_it.o(i.EXTI9_5_IRQHandler) for EXTI9_5_IRQHandler
    startup_stm32f103xb.o(RESET) refers to stm32f1xx_it.o(i.USART2_IRQHandler) for USART2_IRQHandler
    startup_stm32f103xb.o(RESET) refers to stm32f1xx_it.o(i.EXTI15_10_IRQHandler) for EXTI15_10_IRQHandler
    startup_stm32f103xb.o(.text) refers to system_stm32f1xx.o(i.SystemInit) for SystemInit
    startup_stm32f103xb.o(.text) refers to entry.o(.ARM.Collect$$$$00000000) for __main
    main.o(i.SystemClock_Config) refers to memseta.o(.text) for __aeabi_memclr4
    main.o(i.SystemClock_Config) refers to stm32f1xx_hal_rcc.o(i.HAL_RCC_OscConfig) for HAL_RCC_OscConfig
    main.o(i.SystemClock_Config) refers to stm32f1xx_hal_rcc.o(i.HAL_RCC_ClockConfig) for HAL_RCC_ClockConfig
    main.o(i.main) refers to stm32f1xx_hal.o(i.HAL_Init) for HAL_Init
    main.o(i.main) refers to main.o(i.SystemClock_Config) for SystemClock_Config
    main.o(i.main) refers to gpio.o(i.MX_GPIO_Init) for MX_GPIO_Init
    main.o(i.main) refers to dma.o(i.MX_DMA_Init) for MX_DMA_Init
    main.o(i.main) refers to spi.o(i.MX_SPI1_Init) for MX_SPI1_Init
    main.o(i.main) refers to spi.o(i.MX_SPI2_Init) for MX_SPI2_Init
    main.o(i.main) refers to tim.o(i.MX_TIM1_Init) for MX_TIM1_Init
    main.o(i.main) refers to usart.o(i.MX_USART1_UART_Init) for MX_USART1_UART_Init
    main.o(i.main) refers to usart.o(i.MX_USART2_UART_Init) for MX_USART2_UART_Init
    main.o(i.main) refers to sx1281.o(i.SX1281_Init) for SX1281_Init
    main.o(i.main) refers to sx1281.o(i.SX1281_SetTX) for SX1281_SetTX
    main.o(i.main) refers to lcd.o(i.LCD_Init) for LCD_Init
    main.o(i.main) refers to lcd.o(i.LCD_Clear) for LCD_Clear
    main.o(i.main) refers to lcd.o(i.LCD_DrawString) for LCD_DrawString
    main.o(i.main) refers to lcd.o(i.LCD_DrawBitmap) for LCD_DrawBitmap
    main.o(i.main) refers to sx1281.o(i.SX1281_Running) for SX1281_Running
    main.o(i.main) refers to stm32f1xx_hal.o(i.HAL_Delay) for HAL_Delay
    main.o(i.main) refers to usart.o(.bss) for huart2
    main.o(i.main) refers to main.o(.bss) for .bss
    main.o(i.main) refers to lcd.o(.constdata) for logo_M
    gpio.o(i.MX_GPIO_Init) refers to stm32f1xx_hal_gpio.o(i.HAL_GPIO_WritePin) for HAL_GPIO_WritePin
    gpio.o(i.MX_GPIO_Init) refers to stm32f1xx_hal_gpio.o(i.HAL_GPIO_Init) for HAL_GPIO_Init
    gpio.o(i.MX_GPIO_Init) refers to stm32f1xx_hal_cortex.o(i.HAL_NVIC_SetPriority) for HAL_NVIC_SetPriority
    gpio.o(i.MX_GPIO_Init) refers to stm32f1xx_hal_cortex.o(i.HAL_NVIC_EnableIRQ) for HAL_NVIC_EnableIRQ
    dma.o(i.MX_DMA_Init) refers to stm32f1xx_hal_cortex.o(i.HAL_NVIC_SetPriority) for HAL_NVIC_SetPriority
    dma.o(i.MX_DMA_Init) refers to stm32f1xx_hal_cortex.o(i.HAL_NVIC_EnableIRQ) for HAL_NVIC_EnableIRQ
    spi.o(i.HAL_SPI_MspDeInit) refers to stm32f1xx_hal_gpio.o(i.HAL_GPIO_DeInit) for HAL_GPIO_DeInit
    spi.o(i.HAL_SPI_MspDeInit) refers to stm32f1xx_hal_dma.o(i.HAL_DMA_DeInit) for HAL_DMA_DeInit
    spi.o(i.HAL_SPI_MspInit) refers to stm32f1xx_hal_gpio.o(i.HAL_GPIO_Init) for HAL_GPIO_Init
    spi.o(i.HAL_SPI_MspInit) refers to stm32f1xx_hal_dma.o(i.HAL_DMA_Init) for HAL_DMA_Init
    spi.o(i.HAL_SPI_MspInit) refers to main.o(i.Error_Handler) for Error_Handler
    spi.o(i.HAL_SPI_MspInit) refers to spi.o(.bss) for .bss
    spi.o(i.MX_SPI1_Init) refers to stm32f1xx_hal_spi.o(i.HAL_SPI_Init) for HAL_SPI_Init
    spi.o(i.MX_SPI1_Init) refers to main.o(i.Error_Handler) for Error_Handler
    spi.o(i.MX_SPI1_Init) refers to spi.o(.bss) for .bss
    spi.o(i.MX_SPI2_Init) refers to stm32f1xx_hal_spi.o(i.HAL_SPI_Init) for HAL_SPI_Init
    spi.o(i.MX_SPI2_Init) refers to main.o(i.Error_Handler) for Error_Handler
    spi.o(i.MX_SPI2_Init) refers to spi.o(.bss) for .bss
    tim.o(i.HAL_TIM_MspPostInit) refers to stm32f1xx_hal_gpio.o(i.HAL_GPIO_Init) for HAL_GPIO_Init
    tim.o(i.MX_TIM1_Init) refers to memseta.o(.text) for __aeabi_memclr4
    tim.o(i.MX_TIM1_Init) refers to stm32f1xx_hal_tim.o(i.HAL_TIM_Base_Init) for HAL_TIM_Base_Init
    tim.o(i.MX_TIM1_Init) refers to main.o(i.Error_Handler) for Error_Handler
    tim.o(i.MX_TIM1_Init) refers to stm32f1xx_hal_tim.o(i.HAL_TIM_ConfigClockSource) for HAL_TIM_ConfigClockSource
    tim.o(i.MX_TIM1_Init) refers to stm32f1xx_hal_tim.o(i.HAL_TIM_PWM_Init) for HAL_TIM_PWM_Init
    tim.o(i.MX_TIM1_Init) refers to stm32f1xx_hal_tim_ex.o(i.HAL_TIMEx_MasterConfigSynchronization) for HAL_TIMEx_MasterConfigSynchronization
    tim.o(i.MX_TIM1_Init) refers to stm32f1xx_hal_tim.o(i.HAL_TIM_PWM_ConfigChannel) for HAL_TIM_PWM_ConfigChannel
    tim.o(i.MX_TIM1_Init) refers to stm32f1xx_hal_tim_ex.o(i.HAL_TIMEx_ConfigBreakDeadTime) for HAL_TIMEx_ConfigBreakDeadTime
    tim.o(i.MX_TIM1_Init) refers to tim.o(i.HAL_TIM_MspPostInit) for HAL_TIM_MspPostInit
    tim.o(i.MX_TIM1_Init) refers to tim.o(.bss) for .bss
    usart.o(i.HAL_UART_MspDeInit) refers to stm32f1xx_hal_gpio.o(i.HAL_GPIO_DeInit) for HAL_GPIO_DeInit
    usart.o(i.HAL_UART_MspDeInit) refers to stm32f1xx_hal_dma.o(i.HAL_DMA_DeInit) for HAL_DMA_DeInit
    usart.o(i.HAL_UART_MspDeInit) refers to stm32f1xx_hal_cortex.o(i.HAL_NVIC_DisableIRQ) for HAL_NVIC_DisableIRQ
    usart.o(i.HAL_UART_MspInit) refers to stm32f1xx_hal_gpio.o(i.HAL_GPIO_Init) for HAL_GPIO_Init
    usart.o(i.HAL_UART_MspInit) refers to stm32f1xx_hal_dma.o(i.HAL_DMA_Init) for HAL_DMA_Init
    usart.o(i.HAL_UART_MspInit) refers to main.o(i.Error_Handler) for Error_Handler
    usart.o(i.HAL_UART_MspInit) refers to stm32f1xx_hal_cortex.o(i.HAL_NVIC_SetPriority) for HAL_NVIC_SetPriority
    usart.o(i.HAL_UART_MspInit) refers to stm32f1xx_hal_cortex.o(i.HAL_NVIC_EnableIRQ) for HAL_NVIC_EnableIRQ
    usart.o(i.HAL_UART_MspInit) refers to usart.o(.bss) for .bss
    usart.o(i.MX_USART1_UART_Init) refers to stm32f1xx_hal_uart.o(i.HAL_HalfDuplex_Init) for HAL_HalfDuplex_Init
    usart.o(i.MX_USART1_UART_Init) refers to main.o(i.Error_Handler) for Error_Handler
    usart.o(i.MX_USART1_UART_Init) refers to usart.o(.bss) for .bss
    usart.o(i.MX_USART2_UART_Init) refers to stm32f1xx_hal_uart.o(i.HAL_UART_Init) for HAL_UART_Init
    usart.o(i.MX_USART2_UART_Init) refers to main.o(i.Error_Handler) for Error_Handler
    usart.o(i.MX_USART2_UART_Init) refers to usart.o(.bss) for .bss
    usart.o(i.USAR_UART_IDLECallback) refers to stm32f1xx_hal_uart.o(i.HAL_UART_DMAStop) for HAL_UART_DMAStop
    usart.o(i.USAR_UART_IDLECallback) refers to printfa.o(i.__0printf) for __2printf
    usart.o(i.USAR_UART_IDLECallback) refers to stm32f1xx_hal_uart.o(i.HAL_UART_Transmit) for HAL_UART_Transmit
    usart.o(i.USAR_UART_IDLECallback) refers to strcpy.o(.text) for strcpy
    usart.o(i.USAR_UART_IDLECallback) refers to memseta.o(.text) for __aeabi_memclr4
    usart.o(i.USAR_UART_IDLECallback) refers to stm32f1xx_hal_uart.o(i.HAL_UART_Receive_DMA) for HAL_UART_Receive_DMA
    usart.o(i.USAR_UART_IDLECallback) refers to usart.o(.bss) for .bss
    usart.o(i.USER_UART_IRQHandler) refers to printfa.o(i.__0printf) for __2printf
    usart.o(i.USER_UART_IRQHandler) refers to usart.o(i.USAR_UART_IDLECallback) for USAR_UART_IDLECallback
    stm32f1xx_it.o(i.DMA1_Channel2_IRQHandler) refers to stm32f1xx_hal_dma.o(i.HAL_DMA_IRQHandler) for HAL_DMA_IRQHandler
    stm32f1xx_it.o(i.DMA1_Channel2_IRQHandler) refers to spi.o(.bss) for hdma_spi1_rx
    stm32f1xx_it.o(i.DMA1_Channel3_IRQHandler) refers to stm32f1xx_hal_dma.o(i.HAL_DMA_IRQHandler) for HAL_DMA_IRQHandler
    stm32f1xx_it.o(i.DMA1_Channel3_IRQHandler) refers to spi.o(.bss) for hdma_spi1_tx
    stm32f1xx_it.o(i.DMA1_Channel5_IRQHandler) refers to stm32f1xx_hal_dma.o(i.HAL_DMA_IRQHandler) for HAL_DMA_IRQHandler
    stm32f1xx_it.o(i.DMA1_Channel5_IRQHandler) refers to spi.o(.bss) for hdma_spi2_tx
    stm32f1xx_it.o(i.DMA1_Channel6_IRQHandler) refers to stm32f1xx_hal_dma.o(i.HAL_DMA_IRQHandler) for HAL_DMA_IRQHandler
    stm32f1xx_it.o(i.DMA1_Channel6_IRQHandler) refers to usart.o(.bss) for hdma_usart2_rx
    stm32f1xx_it.o(i.DMA1_Channel7_IRQHandler) refers to stm32f1xx_hal_dma.o(i.HAL_DMA_IRQHandler) for HAL_DMA_IRQHandler
    stm32f1xx_it.o(i.DMA1_Channel7_IRQHandler) refers to usart.o(.bss) for hdma_usart2_tx
    stm32f1xx_it.o(i.EXTI15_10_IRQHandler) refers to stm32f1xx_hal_gpio.o(i.HAL_GPIO_EXTI_IRQHandler) for HAL_GPIO_EXTI_IRQHandler
    stm32f1xx_it.o(i.EXTI9_5_IRQHandler) refers to stm32f1xx_hal_gpio.o(i.HAL_GPIO_EXTI_IRQHandler) for HAL_GPIO_EXTI_IRQHandler
    stm32f1xx_it.o(i.SysTick_Handler) refers to stm32f1xx_hal.o(i.HAL_IncTick) for HAL_IncTick
    stm32f1xx_it.o(i.USART2_IRQHandler) refers to stm32f1xx_hal_uart.o(i.HAL_UART_IRQHandler) for HAL_UART_IRQHandler
    stm32f1xx_it.o(i.USART2_IRQHandler) refers to usart.o(i.USER_UART_IRQHandler) for USER_UART_IRQHandler
    stm32f1xx_it.o(i.USART2_IRQHandler) refers to usart.o(.bss) for huart2
    stm32f1xx_hal_spi.o(i.HAL_SPI_Abort) refers to stm32f1xx_hal_dma.o(i.HAL_DMA_Abort) for HAL_DMA_Abort
    stm32f1xx_hal_spi.o(i.HAL_SPI_Abort) refers to system_stm32f1xx.o(.data) for SystemCoreClock
    stm32f1xx_hal_spi.o(i.HAL_SPI_Abort) refers to stm32f1xx_hal_spi.o(i.SPI_AbortTx_ISR) for SPI_AbortTx_ISR
    stm32f1xx_hal_spi.o(i.HAL_SPI_Abort) refers to stm32f1xx_hal_spi.o(i.SPI_AbortRx_ISR) for SPI_AbortRx_ISR
    stm32f1xx_hal_spi.o(i.HAL_SPI_Abort_IT) refers to stm32f1xx_hal_dma.o(i.HAL_DMA_Abort_IT) for HAL_DMA_Abort_IT
    stm32f1xx_hal_spi.o(i.HAL_SPI_Abort_IT) refers to spi_1.o(i.HAL_SPI_AbortCpltCallback) for HAL_SPI_AbortCpltCallback
    stm32f1xx_hal_spi.o(i.HAL_SPI_Abort_IT) refers to system_stm32f1xx.o(.data) for SystemCoreClock
    stm32f1xx_hal_spi.o(i.HAL_SPI_Abort_IT) refers to stm32f1xx_hal_spi.o(i.SPI_AbortTx_ISR) for SPI_AbortTx_ISR
    stm32f1xx_hal_spi.o(i.HAL_SPI_Abort_IT) refers to stm32f1xx_hal_spi.o(i.SPI_AbortRx_ISR) for SPI_AbortRx_ISR
    stm32f1xx_hal_spi.o(i.HAL_SPI_Abort_IT) refers to stm32f1xx_hal_spi.o(i.SPI_DMATxAbortCallback) for SPI_DMATxAbortCallback
    stm32f1xx_hal_spi.o(i.HAL_SPI_Abort_IT) refers to stm32f1xx_hal_spi.o(i.SPI_DMARxAbortCallback) for SPI_DMARxAbortCallback
    stm32f1xx_hal_spi.o(i.HAL_SPI_DMAStop) refers to stm32f1xx_hal_dma.o(i.HAL_DMA_Abort) for HAL_DMA_Abort
    stm32f1xx_hal_spi.o(i.HAL_SPI_DeInit) refers to spi.o(i.HAL_SPI_MspDeInit) for HAL_SPI_MspDeInit
    stm32f1xx_hal_spi.o(i.HAL_SPI_IRQHandler) refers to stm32f1xx_hal_dma.o(i.HAL_DMA_Abort_IT) for HAL_DMA_Abort_IT
    stm32f1xx_hal_spi.o(i.HAL_SPI_IRQHandler) refers to spi_1.o(i.HAL_SPI_ErrorCallback) for HAL_SPI_ErrorCallback
    stm32f1xx_hal_spi.o(i.HAL_SPI_IRQHandler) refers to stm32f1xx_hal_spi.o(i.SPI_DMAAbortOnError) for SPI_DMAAbortOnError
    stm32f1xx_hal_spi.o(i.HAL_SPI_Init) refers to spi.o(i.HAL_SPI_MspInit) for HAL_SPI_MspInit
    stm32f1xx_hal_spi.o(i.HAL_SPI_Receive) refers to stm32f1xx_hal.o(i.HAL_GetTick) for HAL_GetTick
    stm32f1xx_hal_spi.o(i.HAL_SPI_Receive) refers to stm32f1xx_hal_spi.o(i.HAL_SPI_TransmitReceive) for HAL_SPI_TransmitReceive
    stm32f1xx_hal_spi.o(i.HAL_SPI_Receive) refers to stm32f1xx_hal_spi.o(i.SPI_EndRxTransaction) for SPI_EndRxTransaction
    stm32f1xx_hal_spi.o(i.HAL_SPI_Receive_DMA) refers to stm32f1xx_hal_spi.o(i.HAL_SPI_TransmitReceive_DMA) for HAL_SPI_TransmitReceive_DMA
    stm32f1xx_hal_spi.o(i.HAL_SPI_Receive_DMA) refers to stm32f1xx_hal_dma.o(i.HAL_DMA_Start_IT) for HAL_DMA_Start_IT
    stm32f1xx_hal_spi.o(i.HAL_SPI_Receive_DMA) refers to stm32f1xx_hal_spi.o(i.SPI_DMAHalfReceiveCplt) for SPI_DMAHalfReceiveCplt
    stm32f1xx_hal_spi.o(i.HAL_SPI_Receive_DMA) refers to stm32f1xx_hal_spi.o(i.SPI_DMAReceiveCplt) for SPI_DMAReceiveCplt
    stm32f1xx_hal_spi.o(i.HAL_SPI_Receive_DMA) refers to stm32f1xx_hal_spi.o(i.SPI_DMAError) for SPI_DMAError
    stm32f1xx_hal_spi.o(i.HAL_SPI_Receive_IT) refers to stm32f1xx_hal_spi.o(i.HAL_SPI_TransmitReceive_IT) for HAL_SPI_TransmitReceive_IT
    stm32f1xx_hal_spi.o(i.HAL_SPI_Receive_IT) refers to stm32f1xx_hal_spi.o(i.SPI_RxISR_16BIT) for SPI_RxISR_16BIT
    stm32f1xx_hal_spi.o(i.HAL_SPI_Receive_IT) refers to stm32f1xx_hal_spi.o(i.SPI_RxISR_8BIT) for SPI_RxISR_8BIT
    stm32f1xx_hal_spi.o(i.HAL_SPI_Transmit) refers to stm32f1xx_hal.o(i.HAL_GetTick) for HAL_GetTick
    stm32f1xx_hal_spi.o(i.HAL_SPI_Transmit) refers to stm32f1xx_hal_spi.o(i.SPI_EndRxTxTransaction) for SPI_EndRxTxTransaction
    stm32f1xx_hal_spi.o(i.HAL_SPI_TransmitReceive) refers to stm32f1xx_hal.o(i.HAL_GetTick) for HAL_GetTick
    stm32f1xx_hal_spi.o(i.HAL_SPI_TransmitReceive) refers to stm32f1xx_hal_spi.o(i.SPI_EndRxTxTransaction) for SPI_EndRxTxTransaction
    stm32f1xx_hal_spi.o(i.HAL_SPI_TransmitReceive_DMA) refers to stm32f1xx_hal_dma.o(i.HAL_DMA_Start_IT) for HAL_DMA_Start_IT
    stm32f1xx_hal_spi.o(i.HAL_SPI_TransmitReceive_DMA) refers to stm32f1xx_hal_spi.o(i.SPI_DMAHalfTransmitReceiveCplt) for SPI_DMAHalfTransmitReceiveCplt
    stm32f1xx_hal_spi.o(i.HAL_SPI_TransmitReceive_DMA) refers to stm32f1xx_hal_spi.o(i.SPI_DMATransmitReceiveCplt) for SPI_DMATransmitReceiveCplt
    stm32f1xx_hal_spi.o(i.HAL_SPI_TransmitReceive_DMA) refers to stm32f1xx_hal_spi.o(i.SPI_DMAError) for SPI_DMAError
    stm32f1xx_hal_spi.o(i.HAL_SPI_TransmitReceive_DMA) refers to stm32f1xx_hal_spi.o(i.SPI_DMAHalfReceiveCplt) for SPI_DMAHalfReceiveCplt
    stm32f1xx_hal_spi.o(i.HAL_SPI_TransmitReceive_DMA) refers to stm32f1xx_hal_spi.o(i.SPI_DMAReceiveCplt) for SPI_DMAReceiveCplt
    stm32f1xx_hal_spi.o(i.HAL_SPI_TransmitReceive_IT) refers to stm32f1xx_hal_spi.o(i.SPI_2linesRxISR_16BIT) for SPI_2linesRxISR_16BIT
    stm32f1xx_hal_spi.o(i.HAL_SPI_TransmitReceive_IT) refers to stm32f1xx_hal_spi.o(i.SPI_2linesTxISR_16BIT) for SPI_2linesTxISR_16BIT
    stm32f1xx_hal_spi.o(i.HAL_SPI_TransmitReceive_IT) refers to stm32f1xx_hal_spi.o(i.SPI_2linesRxISR_8BIT) for SPI_2linesRxISR_8BIT
    stm32f1xx_hal_spi.o(i.HAL_SPI_TransmitReceive_IT) refers to stm32f1xx_hal_spi.o(i.SPI_2linesTxISR_8BIT) for SPI_2linesTxISR_8BIT
    stm32f1xx_hal_spi.o(i.HAL_SPI_Transmit_DMA) refers to stm32f1xx_hal_dma.o(i.HAL_DMA_Start_IT) for HAL_DMA_Start_IT
    stm32f1xx_hal_spi.o(i.HAL_SPI_Transmit_DMA) refers to stm32f1xx_hal_spi.o(i.SPI_DMAHalfTransmitCplt) for SPI_DMAHalfTransmitCplt
    stm32f1xx_hal_spi.o(i.HAL_SPI_Transmit_DMA) refers to stm32f1xx_hal_spi.o(i.SPI_DMATransmitCplt) for SPI_DMATransmitCplt
    stm32f1xx_hal_spi.o(i.HAL_SPI_Transmit_DMA) refers to stm32f1xx_hal_spi.o(i.SPI_DMAError) for SPI_DMAError
    stm32f1xx_hal_spi.o(i.HAL_SPI_Transmit_IT) refers to stm32f1xx_hal_spi.o(i.SPI_TxISR_16BIT) for SPI_TxISR_16BIT
    stm32f1xx_hal_spi.o(i.HAL_SPI_Transmit_IT) refers to stm32f1xx_hal_spi.o(i.SPI_TxISR_8BIT) for SPI_TxISR_8BIT
    stm32f1xx_hal_spi.o(i.SPI_2linesRxISR_16BIT) refers to stm32f1xx_hal_spi.o(i.SPI_CloseRxTx_ISR) for SPI_CloseRxTx_ISR
    stm32f1xx_hal_spi.o(i.SPI_2linesRxISR_8BIT) refers to stm32f1xx_hal_spi.o(i.SPI_CloseRxTx_ISR) for SPI_CloseRxTx_ISR
    stm32f1xx_hal_spi.o(i.SPI_2linesTxISR_16BIT) refers to stm32f1xx_hal_spi.o(i.SPI_CloseRxTx_ISR) for SPI_CloseRxTx_ISR
    stm32f1xx_hal_spi.o(i.SPI_2linesTxISR_8BIT) refers to stm32f1xx_hal_spi.o(i.SPI_CloseRxTx_ISR) for SPI_CloseRxTx_ISR
    stm32f1xx_hal_spi.o(i.SPI_AbortRx_ISR) refers to system_stm32f1xx.o(.data) for SystemCoreClock
    stm32f1xx_hal_spi.o(i.SPI_CloseRxTx_ISR) refers to stm32f1xx_hal.o(i.HAL_GetTick) for HAL_GetTick
    stm32f1xx_hal_spi.o(i.SPI_CloseRxTx_ISR) refers to stm32f1xx_hal_spi.o(i.SPI_EndRxTxTransaction) for SPI_EndRxTxTransaction
    stm32f1xx_hal_spi.o(i.SPI_CloseRxTx_ISR) refers to spi_1.o(i.HAL_SPI_ErrorCallback) for HAL_SPI_ErrorCallback
    stm32f1xx_hal_spi.o(i.SPI_CloseRxTx_ISR) refers to spi_1.o(i.HAL_SPI_TxRxCpltCallback) for HAL_SPI_TxRxCpltCallback
    stm32f1xx_hal_spi.o(i.SPI_CloseRxTx_ISR) refers to spi_1.o(i.HAL_SPI_RxCpltCallback) for HAL_SPI_RxCpltCallback
    stm32f1xx_hal_spi.o(i.SPI_CloseRxTx_ISR) refers to system_stm32f1xx.o(.data) for SystemCoreClock
    stm32f1xx_hal_spi.o(i.SPI_CloseRx_ISR) refers to stm32f1xx_hal.o(i.HAL_GetTick) for HAL_GetTick
    stm32f1xx_hal_spi.o(i.SPI_CloseRx_ISR) refers to stm32f1xx_hal_spi.o(i.SPI_EndRxTransaction) for SPI_EndRxTransaction
    stm32f1xx_hal_spi.o(i.SPI_CloseRx_ISR) refers to spi_1.o(i.HAL_SPI_ErrorCallback) for HAL_SPI_ErrorCallback
    stm32f1xx_hal_spi.o(i.SPI_CloseRx_ISR) refers to spi_1.o(i.HAL_SPI_RxCpltCallback) for HAL_SPI_RxCpltCallback
    stm32f1xx_hal_spi.o(i.SPI_CloseTx_ISR) refers to stm32f1xx_hal.o(i.HAL_GetTick) for HAL_GetTick
    stm32f1xx_hal_spi.o(i.SPI_CloseTx_ISR) refers to stm32f1xx_hal_spi.o(i.SPI_EndRxTxTransaction) for SPI_EndRxTxTransaction
    stm32f1xx_hal_spi.o(i.SPI_CloseTx_ISR) refers to spi_1.o(i.HAL_SPI_ErrorCallback) for HAL_SPI_ErrorCallback
    stm32f1xx_hal_spi.o(i.SPI_CloseTx_ISR) refers to spi_1.o(i.HAL_SPI_TxCpltCallback) for HAL_SPI_TxCpltCallback
    stm32f1xx_hal_spi.o(i.SPI_CloseTx_ISR) refers to system_stm32f1xx.o(.data) for SystemCoreClock
    stm32f1xx_hal_spi.o(i.SPI_DMAAbortOnError) refers to spi_1.o(i.HAL_SPI_ErrorCallback) for HAL_SPI_ErrorCallback
    stm32f1xx_hal_spi.o(i.SPI_DMAError) refers to spi_1.o(i.HAL_SPI_ErrorCallback) for HAL_SPI_ErrorCallback
    stm32f1xx_hal_spi.o(i.SPI_DMAHalfReceiveCplt) refers to spi_1.o(i.HAL_SPI_RxHalfCpltCallback) for HAL_SPI_RxHalfCpltCallback
    stm32f1xx_hal_spi.o(i.SPI_DMAHalfTransmitCplt) refers to spi_1.o(i.HAL_SPI_TxHalfCpltCallback) for HAL_SPI_TxHalfCpltCallback
    stm32f1xx_hal_spi.o(i.SPI_DMAHalfTransmitReceiveCplt) refers to spi_1.o(i.HAL_SPI_TxRxHalfCpltCallback) for HAL_SPI_TxRxHalfCpltCallback
    stm32f1xx_hal_spi.o(i.SPI_DMAReceiveCplt) refers to stm32f1xx_hal.o(i.HAL_GetTick) for HAL_GetTick
    stm32f1xx_hal_spi.o(i.SPI_DMAReceiveCplt) refers to stm32f1xx_hal_spi.o(i.SPI_EndRxTransaction) for SPI_EndRxTransaction
    stm32f1xx_hal_spi.o(i.SPI_DMAReceiveCplt) refers to spi_1.o(i.HAL_SPI_ErrorCallback) for HAL_SPI_ErrorCallback
    stm32f1xx_hal_spi.o(i.SPI_DMAReceiveCplt) refers to spi_1.o(i.HAL_SPI_RxCpltCallback) for HAL_SPI_RxCpltCallback
    stm32f1xx_hal_spi.o(i.SPI_DMARxAbortCallback) refers to stm32f1xx_hal.o(i.HAL_GetTick) for HAL_GetTick
    stm32f1xx_hal_spi.o(i.SPI_DMARxAbortCallback) refers to stm32f1xx_hal_spi.o(i.SPI_EndRxTxTransaction) for SPI_EndRxTxTransaction
    stm32f1xx_hal_spi.o(i.SPI_DMARxAbortCallback) refers to spi_1.o(i.HAL_SPI_AbortCpltCallback) for HAL_SPI_AbortCpltCallback
    stm32f1xx_hal_spi.o(i.SPI_DMATransmitCplt) refers to stm32f1xx_hal.o(i.HAL_GetTick) for HAL_GetTick
    stm32f1xx_hal_spi.o(i.SPI_DMATransmitCplt) refers to stm32f1xx_hal_spi.o(i.SPI_EndRxTxTransaction) for SPI_EndRxTxTransaction
    stm32f1xx_hal_spi.o(i.SPI_DMATransmitCplt) refers to spi_1.o(i.HAL_SPI_ErrorCallback) for HAL_SPI_ErrorCallback
    stm32f1xx_hal_spi.o(i.SPI_DMATransmitCplt) refers to spi_1.o(i.HAL_SPI_TxCpltCallback) for HAL_SPI_TxCpltCallback
    stm32f1xx_hal_spi.o(i.SPI_DMATransmitReceiveCplt) refers to stm32f1xx_hal.o(i.HAL_GetTick) for HAL_GetTick
    stm32f1xx_hal_spi.o(i.SPI_DMATransmitReceiveCplt) refers to stm32f1xx_hal_spi.o(i.SPI_EndRxTxTransaction) for SPI_EndRxTxTransaction
    stm32f1xx_hal_spi.o(i.SPI_DMATransmitReceiveCplt) refers to spi_1.o(i.HAL_SPI_ErrorCallback) for HAL_SPI_ErrorCallback
    stm32f1xx_hal_spi.o(i.SPI_DMATransmitReceiveCplt) refers to spi_1.o(i.HAL_SPI_TxRxCpltCallback) for HAL_SPI_TxRxCpltCallback
    stm32f1xx_hal_spi.o(i.SPI_DMATxAbortCallback) refers to spi_1.o(i.HAL_SPI_AbortCpltCallback) for HAL_SPI_AbortCpltCallback
    stm32f1xx_hal_spi.o(i.SPI_DMATxAbortCallback) refers to system_stm32f1xx.o(.data) for SystemCoreClock
    stm32f1xx_hal_spi.o(i.SPI_EndRxTransaction) refers to stm32f1xx_hal_spi.o(i.SPI_WaitFlagStateUntilTimeout) for SPI_WaitFlagStateUntilTimeout
    stm32f1xx_hal_spi.o(i.SPI_EndRxTxTransaction) refers to stm32f1xx_hal_spi.o(i.SPI_WaitFlagStateUntilTimeout) for SPI_WaitFlagStateUntilTimeout
    stm32f1xx_hal_spi.o(i.SPI_RxISR_16BIT) refers to stm32f1xx_hal_spi.o(i.SPI_CloseRx_ISR) for SPI_CloseRx_ISR
    stm32f1xx_hal_spi.o(i.SPI_RxISR_8BIT) refers to stm32f1xx_hal_spi.o(i.SPI_CloseRx_ISR) for SPI_CloseRx_ISR
    stm32f1xx_hal_spi.o(i.SPI_TxISR_16BIT) refers to stm32f1xx_hal_spi.o(i.SPI_CloseTx_ISR) for SPI_CloseTx_ISR
    stm32f1xx_hal_spi.o(i.SPI_TxISR_8BIT) refers to stm32f1xx_hal_spi.o(i.SPI_CloseTx_ISR) for SPI_CloseTx_ISR
    stm32f1xx_hal_spi.o(i.SPI_WaitFlagStateUntilTimeout) refers to stm32f1xx_hal.o(i.HAL_GetTick) for HAL_GetTick
    stm32f1xx_hal_spi.o(i.SPI_WaitFlagStateUntilTimeout) refers to system_stm32f1xx.o(.data) for SystemCoreClock
    stm32f1xx_hal.o(i.HAL_DeInit) refers to stm32f1xx_hal.o(i.HAL_MspDeInit) for HAL_MspDeInit
    stm32f1xx_hal.o(i.HAL_Delay) refers to stm32f1xx_hal.o(i.HAL_GetTick) for HAL_GetTick
    stm32f1xx_hal.o(i.HAL_Delay) refers to stm32f1xx_hal.o(.data) for .data
    stm32f1xx_hal.o(i.HAL_GetTick) refers to stm32f1xx_hal.o(.data) for .data
    stm32f1xx_hal.o(i.HAL_GetTickFreq) refers to stm32f1xx_hal.o(.data) for .data
    stm32f1xx_hal.o(i.HAL_GetTickPrio) refers to stm32f1xx_hal.o(.data) for .data
    stm32f1xx_hal.o(i.HAL_IncTick) refers to stm32f1xx_hal.o(.data) for .data
    stm32f1xx_hal.o(i.HAL_Init) refers to stm32f1xx_hal_cortex.o(i.HAL_NVIC_SetPriorityGrouping) for HAL_NVIC_SetPriorityGrouping
    stm32f1xx_hal.o(i.HAL_Init) refers to stm32f1xx_hal.o(i.HAL_InitTick) for HAL_InitTick
    stm32f1xx_hal.o(i.HAL_Init) refers to stm32f1xx_hal_msp.o(i.HAL_MspInit) for HAL_MspInit
    stm32f1xx_hal.o(i.HAL_InitTick) refers to stm32f1xx_hal_cortex.o(i.HAL_SYSTICK_Config) for HAL_SYSTICK_Config
    stm32f1xx_hal.o(i.HAL_InitTick) refers to stm32f1xx_hal_cortex.o(i.HAL_NVIC_SetPriority) for HAL_NVIC_SetPriority
    stm32f1xx_hal.o(i.HAL_InitTick) refers to stm32f1xx_hal.o(.data) for .data
    stm32f1xx_hal.o(i.HAL_InitTick) refers to system_stm32f1xx.o(.data) for SystemCoreClock
    stm32f1xx_hal.o(i.HAL_SetTickFreq) refers to stm32f1xx_hal.o(i.HAL_InitTick) for HAL_InitTick
    stm32f1xx_hal.o(i.HAL_SetTickFreq) refers to stm32f1xx_hal.o(.data) for .data
    stm32f1xx_hal_rcc.o(i.HAL_RCC_ClockConfig) refers to stm32f1xx_hal.o(i.HAL_GetTick) for HAL_GetTick
    stm32f1xx_hal_rcc.o(i.HAL_RCC_ClockConfig) refers to stm32f1xx_hal_rcc.o(i.HAL_RCC_GetSysClockFreq) for HAL_RCC_GetSysClockFreq
    stm32f1xx_hal_rcc.o(i.HAL_RCC_ClockConfig) refers to stm32f1xx_hal.o(i.HAL_InitTick) for HAL_InitTick
    stm32f1xx_hal_rcc.o(i.HAL_RCC_ClockConfig) refers to system_stm32f1xx.o(.constdata) for AHBPrescTable
    stm32f1xx_hal_rcc.o(i.HAL_RCC_ClockConfig) refers to system_stm32f1xx.o(.data) for SystemCoreClock
    stm32f1xx_hal_rcc.o(i.HAL_RCC_ClockConfig) refers to stm32f1xx_hal.o(.data) for uwTickPrio
    stm32f1xx_hal_rcc.o(i.HAL_RCC_DeInit) refers to stm32f1xx_hal.o(i.HAL_GetTick) for HAL_GetTick
    stm32f1xx_hal_rcc.o(i.HAL_RCC_DeInit) refers to stm32f1xx_hal.o(i.HAL_InitTick) for HAL_InitTick
    stm32f1xx_hal_rcc.o(i.HAL_RCC_DeInit) refers to system_stm32f1xx.o(.data) for SystemCoreClock
    stm32f1xx_hal_rcc.o(i.HAL_RCC_DeInit) refers to stm32f1xx_hal.o(.data) for uwTickPrio
    stm32f1xx_hal_rcc.o(i.HAL_RCC_GetHCLKFreq) refers to system_stm32f1xx.o(.data) for SystemCoreClock
    stm32f1xx_hal_rcc.o(i.HAL_RCC_GetPCLK1Freq) refers to system_stm32f1xx.o(.data) for SystemCoreClock
    stm32f1xx_hal_rcc.o(i.HAL_RCC_GetPCLK1Freq) refers to system_stm32f1xx.o(.constdata) for APBPrescTable
    stm32f1xx_hal_rcc.o(i.HAL_RCC_GetPCLK2Freq) refers to system_stm32f1xx.o(.data) for SystemCoreClock
    stm32f1xx_hal_rcc.o(i.HAL_RCC_GetPCLK2Freq) refers to system_stm32f1xx.o(.constdata) for APBPrescTable
    stm32f1xx_hal_rcc.o(i.HAL_RCC_GetSysClockFreq) refers to stm32f1xx_hal_rcc.o(.constdata) for .constdata
    stm32f1xx_hal_rcc.o(i.HAL_RCC_MCOConfig) refers to stm32f1xx_hal_gpio.o(i.HAL_GPIO_Init) for HAL_GPIO_Init
    stm32f1xx_hal_rcc.o(i.HAL_RCC_NMI_IRQHandler) refers to stm32f1xx_hal_rcc.o(i.HAL_RCC_CSSCallback) for HAL_RCC_CSSCallback
    stm32f1xx_hal_rcc.o(i.HAL_RCC_OscConfig) refers to stm32f1xx_hal.o(i.HAL_GetTick) for HAL_GetTick
    stm32f1xx_hal_rcc.o(i.HAL_RCC_OscConfig) refers to system_stm32f1xx.o(.data) for SystemCoreClock
    stm32f1xx_hal_rcc_ex.o(i.HAL_RCCEx_GetPeriphCLKFreq) refers to stm32f1xx_hal_rcc.o(i.HAL_RCC_GetPCLK2Freq) for HAL_RCC_GetPCLK2Freq
    stm32f1xx_hal_rcc_ex.o(i.HAL_RCCEx_GetPeriphCLKFreq) refers to stm32f1xx_hal_rcc_ex.o(.constdata) for .constdata
    stm32f1xx_hal_rcc_ex.o(i.HAL_RCCEx_PeriphCLKConfig) refers to stm32f1xx_hal.o(i.HAL_GetTick) for HAL_GetTick
    stm32f1xx_hal_gpio.o(i.HAL_GPIO_EXTI_IRQHandler) refers to gpio_1.o(i.HAL_GPIO_EXTI_Callback) for HAL_GPIO_EXTI_Callback
    stm32f1xx_hal_dma.o(i.HAL_DMA_PollForTransfer) refers to stm32f1xx_hal.o(i.HAL_GetTick) for HAL_GetTick
    stm32f1xx_hal_dma.o(i.HAL_DMA_Start) refers to stm32f1xx_hal_dma.o(i.DMA_SetConfig) for DMA_SetConfig
    stm32f1xx_hal_dma.o(i.HAL_DMA_Start_IT) refers to stm32f1xx_hal_dma.o(i.DMA_SetConfig) for DMA_SetConfig
    stm32f1xx_hal_cortex.o(i.HAL_NVIC_SetPriority) refers to stm32f1xx_hal_cortex.o(i.__NVIC_SetPriority) for __NVIC_SetPriority
    stm32f1xx_hal_cortex.o(i.HAL_SYSTICK_Config) refers to stm32f1xx_hal_cortex.o(i.__NVIC_SetPriority) for __NVIC_SetPriority
    stm32f1xx_hal_cortex.o(i.HAL_SYSTICK_IRQHandler) refers to stm32f1xx_hal_cortex.o(i.HAL_SYSTICK_Callback) for HAL_SYSTICK_Callback
    stm32f1xx_hal_pwr.o(i.HAL_PWR_EnterSTOPMode) refers to stm32f1xx_hal_pwr.o(i.PWR_OverloadWfe) for PWR_OverloadWfe
    stm32f1xx_hal_pwr.o(i.HAL_PWR_PVD_IRQHandler) refers to stm32f1xx_hal_pwr.o(i.HAL_PWR_PVDCallback) for HAL_PWR_PVDCallback
    stm32f1xx_hal_flash.o(i.FLASH_Program_HalfWord) refers to stm32f1xx_hal_flash.o(.bss) for .bss
    stm32f1xx_hal_flash.o(i.FLASH_SetErrorCode) refers to stm32f1xx_hal_flash.o(.bss) for .bss
    stm32f1xx_hal_flash.o(i.FLASH_WaitForLastOperation) refers to stm32f1xx_hal.o(i.HAL_GetTick) for HAL_GetTick
    stm32f1xx_hal_flash.o(i.FLASH_WaitForLastOperation) refers to stm32f1xx_hal_flash.o(i.FLASH_SetErrorCode) for FLASH_SetErrorCode
    stm32f1xx_hal_flash.o(i.HAL_FLASH_GetError) refers to stm32f1xx_hal_flash.o(.bss) for .bss
    stm32f1xx_hal_flash.o(i.HAL_FLASH_IRQHandler) refers to stm32f1xx_hal_flash.o(i.FLASH_SetErrorCode) for FLASH_SetErrorCode
    stm32f1xx_hal_flash.o(i.HAL_FLASH_IRQHandler) refers to stm32f1xx_hal_flash.o(i.HAL_FLASH_OperationErrorCallback) for HAL_FLASH_OperationErrorCallback
    stm32f1xx_hal_flash.o(i.HAL_FLASH_IRQHandler) refers to stm32f1xx_hal_flash.o(i.FLASH_Program_HalfWord) for FLASH_Program_HalfWord
    stm32f1xx_hal_flash.o(i.HAL_FLASH_IRQHandler) refers to stm32f1xx_hal_flash.o(i.HAL_FLASH_EndOfOperationCallback) for HAL_FLASH_EndOfOperationCallback
    stm32f1xx_hal_flash.o(i.HAL_FLASH_IRQHandler) refers to stm32f1xx_hal_flash_ex.o(i.FLASH_PageErase) for FLASH_PageErase
    stm32f1xx_hal_flash.o(i.HAL_FLASH_IRQHandler) refers to stm32f1xx_hal_flash.o(.bss) for .bss
    stm32f1xx_hal_flash.o(i.HAL_FLASH_OB_Launch) refers to stm32f1xx_hal_cortex.o(i.HAL_NVIC_SystemReset) for HAL_NVIC_SystemReset
    stm32f1xx_hal_flash.o(i.HAL_FLASH_Program) refers to stm32f1xx_hal_flash.o(i.FLASH_WaitForLastOperation) for FLASH_WaitForLastOperation
    stm32f1xx_hal_flash.o(i.HAL_FLASH_Program) refers to llushr.o(.text) for __aeabi_llsr
    stm32f1xx_hal_flash.o(i.HAL_FLASH_Program) refers to stm32f1xx_hal_flash.o(i.FLASH_Program_HalfWord) for FLASH_Program_HalfWord
    stm32f1xx_hal_flash.o(i.HAL_FLASH_Program) refers to stm32f1xx_hal_flash.o(.bss) for .bss
    stm32f1xx_hal_flash.o(i.HAL_FLASH_Program_IT) refers to stm32f1xx_hal_flash.o(i.FLASH_Program_HalfWord) for FLASH_Program_HalfWord
    stm32f1xx_hal_flash.o(i.HAL_FLASH_Program_IT) refers to stm32f1xx_hal_flash.o(.bss) for .bss
    stm32f1xx_hal_flash_ex.o(i.FLASH_MassErase) refers to stm32f1xx_hal_flash.o(.bss) for pFlash
    stm32f1xx_hal_flash_ex.o(i.FLASH_OB_DisableWRP) refers to stm32f1xx_hal_flash.o(i.FLASH_WaitForLastOperation) for FLASH_WaitForLastOperation
    stm32f1xx_hal_flash_ex.o(i.FLASH_OB_DisableWRP) refers to stm32f1xx_hal_flash_ex.o(i.HAL_FLASHEx_OBErase) for HAL_FLASHEx_OBErase
    stm32f1xx_hal_flash_ex.o(i.FLASH_OB_DisableWRP) refers to stm32f1xx_hal_flash.o(.bss) for pFlash
    stm32f1xx_hal_flash_ex.o(i.FLASH_OB_EnableWRP) refers to stm32f1xx_hal_flash.o(i.FLASH_WaitForLastOperation) for FLASH_WaitForLastOperation
    stm32f1xx_hal_flash_ex.o(i.FLASH_OB_EnableWRP) refers to stm32f1xx_hal_flash_ex.o(i.HAL_FLASHEx_OBErase) for HAL_FLASHEx_OBErase
    stm32f1xx_hal_flash_ex.o(i.FLASH_OB_EnableWRP) refers to stm32f1xx_hal_flash.o(.bss) for pFlash
    stm32f1xx_hal_flash_ex.o(i.FLASH_OB_RDP_LevelConfig) refers to stm32f1xx_hal_flash.o(i.FLASH_WaitForLastOperation) for FLASH_WaitForLastOperation
    stm32f1xx_hal_flash_ex.o(i.FLASH_OB_RDP_LevelConfig) refers to stm32f1xx_hal_flash.o(.bss) for pFlash
    stm32f1xx_hal_flash_ex.o(i.FLASH_PageErase) refers to stm32f1xx_hal_flash.o(.bss) for pFlash
    stm32f1xx_hal_flash_ex.o(i.HAL_FLASHEx_Erase) refers to stm32f1xx_hal_flash.o(i.FLASH_WaitForLastOperation) for FLASH_WaitForLastOperation
    stm32f1xx_hal_flash_ex.o(i.HAL_FLASHEx_Erase) refers to stm32f1xx_hal_flash_ex.o(i.FLASH_MassErase) for FLASH_MassErase
    stm32f1xx_hal_flash_ex.o(i.HAL_FLASHEx_Erase) refers to stm32f1xx_hal_flash_ex.o(i.FLASH_PageErase) for FLASH_PageErase
    stm32f1xx_hal_flash_ex.o(i.HAL_FLASHEx_Erase) refers to stm32f1xx_hal_flash.o(.bss) for pFlash
    stm32f1xx_hal_flash_ex.o(i.HAL_FLASHEx_Erase_IT) refers to stm32f1xx_hal_flash_ex.o(i.FLASH_PageErase) for FLASH_PageErase
    stm32f1xx_hal_flash_ex.o(i.HAL_FLASHEx_Erase_IT) refers to stm32f1xx_hal_flash_ex.o(i.FLASH_MassErase) for FLASH_MassErase
    stm32f1xx_hal_flash_ex.o(i.HAL_FLASHEx_Erase_IT) refers to stm32f1xx_hal_flash.o(.bss) for pFlash
    stm32f1xx_hal_flash_ex.o(i.HAL_FLASHEx_OBErase) refers to stm32f1xx_hal_flash_ex.o(i.FLASH_OB_GetRDP) for FLASH_OB_GetRDP
    stm32f1xx_hal_flash_ex.o(i.HAL_FLASHEx_OBErase) refers to stm32f1xx_hal_flash.o(i.FLASH_WaitForLastOperation) for FLASH_WaitForLastOperation
    stm32f1xx_hal_flash_ex.o(i.HAL_FLASHEx_OBErase) refers to stm32f1xx_hal_flash_ex.o(i.FLASH_OB_RDP_LevelConfig) for FLASH_OB_RDP_LevelConfig
    stm32f1xx_hal_flash_ex.o(i.HAL_FLASHEx_OBErase) refers to stm32f1xx_hal_flash.o(.bss) for pFlash
    stm32f1xx_hal_flash_ex.o(i.HAL_FLASHEx_OBGetConfig) refers to stm32f1xx_hal_flash_ex.o(i.FLASH_OB_GetRDP) for FLASH_OB_GetRDP
    stm32f1xx_hal_flash_ex.o(i.HAL_FLASHEx_OBProgram) refers to stm32f1xx_hal_flash_ex.o(i.FLASH_OB_DisableWRP) for FLASH_OB_DisableWRP
    stm32f1xx_hal_flash_ex.o(i.HAL_FLASHEx_OBProgram) refers to stm32f1xx_hal_flash_ex.o(i.FLASH_OB_EnableWRP) for FLASH_OB_EnableWRP
    stm32f1xx_hal_flash_ex.o(i.HAL_FLASHEx_OBProgram) refers to stm32f1xx_hal_flash_ex.o(i.FLASH_OB_RDP_LevelConfig) for FLASH_OB_RDP_LevelConfig
    stm32f1xx_hal_flash_ex.o(i.HAL_FLASHEx_OBProgram) refers to stm32f1xx_hal_flash.o(i.FLASH_WaitForLastOperation) for FLASH_WaitForLastOperation
    stm32f1xx_hal_flash_ex.o(i.HAL_FLASHEx_OBProgram) refers to stm32f1xx_hal_flash.o(.bss) for pFlash
    stm32f1xx_hal_tim.o(i.HAL_TIM_Base_DeInit) refers to tim.o(i.HAL_TIM_Base_MspDeInit) for HAL_TIM_Base_MspDeInit
    stm32f1xx_hal_tim.o(i.HAL_TIM_Base_Init) refers to tim.o(i.HAL_TIM_Base_MspInit) for HAL_TIM_Base_MspInit
    stm32f1xx_hal_tim.o(i.HAL_TIM_Base_Init) refers to stm32f1xx_hal_tim.o(i.TIM_Base_SetConfig) for TIM_Base_SetConfig
    stm32f1xx_hal_tim.o(i.HAL_TIM_Base_Start_DMA) refers to stm32f1xx_hal_dma.o(i.HAL_DMA_Start_IT) for HAL_DMA_Start_IT
    stm32f1xx_hal_tim.o(i.HAL_TIM_Base_Start_DMA) refers to stm32f1xx_hal_tim.o(i.TIM_DMAPeriodElapsedCplt) for TIM_DMAPeriodElapsedCplt
    stm32f1xx_hal_tim.o(i.HAL_TIM_Base_Start_DMA) refers to stm32f1xx_hal_tim.o(i.TIM_DMAPeriodElapsedHalfCplt) for TIM_DMAPeriodElapsedHalfCplt
    stm32f1xx_hal_tim.o(i.HAL_TIM_Base_Start_DMA) refers to stm32f1xx_hal_tim.o(i.TIM_DMAError) for TIM_DMAError
    stm32f1xx_hal_tim.o(i.HAL_TIM_Base_Stop_DMA) refers to stm32f1xx_hal_dma.o(i.HAL_DMA_Abort_IT) for HAL_DMA_Abort_IT
    stm32f1xx_hal_tim.o(i.HAL_TIM_ConfigClockSource) refers to stm32f1xx_hal_tim.o(i.TIM_ETR_SetConfig) for TIM_ETR_SetConfig
    stm32f1xx_hal_tim.o(i.HAL_TIM_ConfigClockSource) refers to stm32f1xx_hal_tim.o(i.TIM_TI1_ConfigInputStage) for TIM_TI1_ConfigInputStage
    stm32f1xx_hal_tim.o(i.HAL_TIM_ConfigClockSource) refers to stm32f1xx_hal_tim.o(i.TIM_TI2_ConfigInputStage) for TIM_TI2_ConfigInputStage
    stm32f1xx_hal_tim.o(i.HAL_TIM_ConfigClockSource) refers to stm32f1xx_hal_tim.o(i.TIM_ITRx_SetConfig) for TIM_ITRx_SetConfig
    stm32f1xx_hal_tim.o(i.HAL_TIM_ConfigOCrefClear) refers to stm32f1xx_hal_tim.o(i.TIM_ETR_SetConfig) for TIM_ETR_SetConfig
    stm32f1xx_hal_tim.o(i.HAL_TIM_DMABurst_MultiReadStart) refers to stm32f1xx_hal_dma.o(i.HAL_DMA_Start_IT) for HAL_DMA_Start_IT
    stm32f1xx_hal_tim.o(i.HAL_TIM_DMABurst_MultiReadStart) refers to stm32f1xx_hal_tim.o(i.TIM_DMAError) for TIM_DMAError
    stm32f1xx_hal_tim.o(i.HAL_TIM_DMABurst_MultiReadStart) refers to stm32f1xx_hal_tim.o(i.TIM_DMACaptureCplt) for TIM_DMACaptureCplt
    stm32f1xx_hal_tim.o(i.HAL_TIM_DMABurst_MultiReadStart) refers to stm32f1xx_hal_tim.o(i.TIM_DMACaptureHalfCplt) for TIM_DMACaptureHalfCplt
    stm32f1xx_hal_tim.o(i.HAL_TIM_DMABurst_MultiReadStart) refers to stm32f1xx_hal_tim.o(i.TIM_DMAPeriodElapsedCplt) for TIM_DMAPeriodElapsedCplt
    stm32f1xx_hal_tim.o(i.HAL_TIM_DMABurst_MultiReadStart) refers to stm32f1xx_hal_tim.o(i.TIM_DMAPeriodElapsedHalfCplt) for TIM_DMAPeriodElapsedHalfCplt
    stm32f1xx_hal_tim.o(i.HAL_TIM_DMABurst_MultiReadStart) refers to stm32f1xx_hal_tim_ex.o(i.TIMEx_DMACommutationCplt) for TIMEx_DMACommutationCplt
    stm32f1xx_hal_tim.o(i.HAL_TIM_DMABurst_MultiReadStart) refers to stm32f1xx_hal_tim_ex.o(i.TIMEx_DMACommutationHalfCplt) for TIMEx_DMACommutationHalfCplt
    stm32f1xx_hal_tim.o(i.HAL_TIM_DMABurst_MultiReadStart) refers to stm32f1xx_hal_tim.o(i.TIM_DMATriggerCplt) for TIM_DMATriggerCplt
    stm32f1xx_hal_tim.o(i.HAL_TIM_DMABurst_MultiReadStart) refers to stm32f1xx_hal_tim.o(i.TIM_DMATriggerHalfCplt) for TIM_DMATriggerHalfCplt
    stm32f1xx_hal_tim.o(i.HAL_TIM_DMABurst_MultiWriteStart) refers to stm32f1xx_hal_dma.o(i.HAL_DMA_Start_IT) for HAL_DMA_Start_IT
    stm32f1xx_hal_tim.o(i.HAL_TIM_DMABurst_MultiWriteStart) refers to stm32f1xx_hal_tim.o(i.TIM_DMAError) for TIM_DMAError
    stm32f1xx_hal_tim.o(i.HAL_TIM_DMABurst_MultiWriteStart) refers to stm32f1xx_hal_tim.o(i.TIM_DMADelayPulseCplt) for TIM_DMADelayPulseCplt
    stm32f1xx_hal_tim.o(i.HAL_TIM_DMABurst_MultiWriteStart) refers to stm32f1xx_hal_tim.o(i.TIM_DMADelayPulseHalfCplt) for TIM_DMADelayPulseHalfCplt
    stm32f1xx_hal_tim.o(i.HAL_TIM_DMABurst_MultiWriteStart) refers to stm32f1xx_hal_tim.o(i.TIM_DMAPeriodElapsedCplt) for TIM_DMAPeriodElapsedCplt
    stm32f1xx_hal_tim.o(i.HAL_TIM_DMABurst_MultiWriteStart) refers to stm32f1xx_hal_tim.o(i.TIM_DMAPeriodElapsedHalfCplt) for TIM_DMAPeriodElapsedHalfCplt
    stm32f1xx_hal_tim.o(i.HAL_TIM_DMABurst_MultiWriteStart) refers to stm32f1xx_hal_tim_ex.o(i.TIMEx_DMACommutationCplt) for TIMEx_DMACommutationCplt
    stm32f1xx_hal_tim.o(i.HAL_TIM_DMABurst_MultiWriteStart) refers to stm32f1xx_hal_tim_ex.o(i.TIMEx_DMACommutationHalfCplt) for TIMEx_DMACommutationHalfCplt
    stm32f1xx_hal_tim.o(i.HAL_TIM_DMABurst_MultiWriteStart) refers to stm32f1xx_hal_tim.o(i.TIM_DMATriggerCplt) for TIM_DMATriggerCplt
    stm32f1xx_hal_tim.o(i.HAL_TIM_DMABurst_MultiWriteStart) refers to stm32f1xx_hal_tim.o(i.TIM_DMATriggerHalfCplt) for TIM_DMATriggerHalfCplt
    stm32f1xx_hal_tim.o(i.HAL_TIM_DMABurst_ReadStart) refers to stm32f1xx_hal_tim.o(i.HAL_TIM_DMABurst_MultiReadStart) for HAL_TIM_DMABurst_MultiReadStart
    stm32f1xx_hal_tim.o(i.HAL_TIM_DMABurst_ReadStop) refers to stm32f1xx_hal_dma.o(i.HAL_DMA_Abort_IT) for HAL_DMA_Abort_IT
    stm32f1xx_hal_tim.o(i.HAL_TIM_DMABurst_WriteStart) refers to stm32f1xx_hal_tim.o(i.HAL_TIM_DMABurst_MultiWriteStart) for HAL_TIM_DMABurst_MultiWriteStart
    stm32f1xx_hal_tim.o(i.HAL_TIM_DMABurst_WriteStop) refers to stm32f1xx_hal_dma.o(i.HAL_DMA_Abort_IT) for HAL_DMA_Abort_IT
    stm32f1xx_hal_tim.o(i.HAL_TIM_Encoder_DeInit) refers to stm32f1xx_hal_tim.o(i.HAL_TIM_Encoder_MspDeInit) for HAL_TIM_Encoder_MspDeInit
    stm32f1xx_hal_tim.o(i.HAL_TIM_Encoder_Init) refers to stm32f1xx_hal_tim.o(i.HAL_TIM_Encoder_MspInit) for HAL_TIM_Encoder_MspInit
    stm32f1xx_hal_tim.o(i.HAL_TIM_Encoder_Init) refers to stm32f1xx_hal_tim.o(i.TIM_Base_SetConfig) for TIM_Base_SetConfig
    stm32f1xx_hal_tim.o(i.HAL_TIM_Encoder_Start) refers to stm32f1xx_hal_tim.o(i.TIM_CCxChannelCmd) for TIM_CCxChannelCmd
    stm32f1xx_hal_tim.o(i.HAL_TIM_Encoder_Start_DMA) refers to stm32f1xx_hal_dma.o(i.HAL_DMA_Start_IT) for HAL_DMA_Start_IT
    stm32f1xx_hal_tim.o(i.HAL_TIM_Encoder_Start_DMA) refers to stm32f1xx_hal_tim.o(i.TIM_CCxChannelCmd) for TIM_CCxChannelCmd
    stm32f1xx_hal_tim.o(i.HAL_TIM_Encoder_Start_DMA) refers to stm32f1xx_hal_tim.o(i.TIM_DMACaptureCplt) for TIM_DMACaptureCplt
    stm32f1xx_hal_tim.o(i.HAL_TIM_Encoder_Start_DMA) refers to stm32f1xx_hal_tim.o(i.TIM_DMACaptureHalfCplt) for TIM_DMACaptureHalfCplt
    stm32f1xx_hal_tim.o(i.HAL_TIM_Encoder_Start_DMA) refers to stm32f1xx_hal_tim.o(i.TIM_DMAError) for TIM_DMAError
    stm32f1xx_hal_tim.o(i.HAL_TIM_Encoder_Start_IT) refers to stm32f1xx_hal_tim.o(i.TIM_CCxChannelCmd) for TIM_CCxChannelCmd
    stm32f1xx_hal_tim.o(i.HAL_TIM_Encoder_Stop) refers to stm32f1xx_hal_tim.o(i.TIM_CCxChannelCmd) for TIM_CCxChannelCmd
    stm32f1xx_hal_tim.o(i.HAL_TIM_Encoder_Stop_DMA) refers to stm32f1xx_hal_tim.o(i.TIM_CCxChannelCmd) for TIM_CCxChannelCmd
    stm32f1xx_hal_tim.o(i.HAL_TIM_Encoder_Stop_DMA) refers to stm32f1xx_hal_dma.o(i.HAL_DMA_Abort_IT) for HAL_DMA_Abort_IT
    stm32f1xx_hal_tim.o(i.HAL_TIM_Encoder_Stop_IT) refers to stm32f1xx_hal_tim.o(i.TIM_CCxChannelCmd) for TIM_CCxChannelCmd
    stm32f1xx_hal_tim.o(i.HAL_TIM_IC_ConfigChannel) refers to stm32f1xx_hal_tim.o(i.TIM_TI1_SetConfig) for TIM_TI1_SetConfig
    stm32f1xx_hal_tim.o(i.HAL_TIM_IC_ConfigChannel) refers to stm32f1xx_hal_tim.o(i.TIM_TI2_SetConfig) for TIM_TI2_SetConfig
    stm32f1xx_hal_tim.o(i.HAL_TIM_IC_DeInit) refers to stm32f1xx_hal_tim.o(i.HAL_TIM_IC_MspDeInit) for HAL_TIM_IC_MspDeInit
    stm32f1xx_hal_tim.o(i.HAL_TIM_IC_Init) refers to stm32f1xx_hal_tim.o(i.HAL_TIM_IC_MspInit) for HAL_TIM_IC_MspInit
    stm32f1xx_hal_tim.o(i.HAL_TIM_IC_Init) refers to stm32f1xx_hal_tim.o(i.TIM_Base_SetConfig) for TIM_Base_SetConfig
    stm32f1xx_hal_tim.o(i.HAL_TIM_IC_Start) refers to stm32f1xx_hal_tim.o(i.TIM_CCxChannelCmd) for TIM_CCxChannelCmd
    stm32f1xx_hal_tim.o(i.HAL_TIM_IC_Start_DMA) refers to stm32f1xx_hal_tim.o(i.TIM_CCxChannelCmd) for TIM_CCxChannelCmd
    stm32f1xx_hal_tim.o(i.HAL_TIM_IC_Start_DMA) refers to stm32f1xx_hal_dma.o(i.HAL_DMA_Start_IT) for HAL_DMA_Start_IT
    stm32f1xx_hal_tim.o(i.HAL_TIM_IC_Start_DMA) refers to stm32f1xx_hal_tim.o(i.TIM_DMACaptureCplt) for TIM_DMACaptureCplt
    stm32f1xx_hal_tim.o(i.HAL_TIM_IC_Start_DMA) refers to stm32f1xx_hal_tim.o(i.TIM_DMACaptureHalfCplt) for TIM_DMACaptureHalfCplt
    stm32f1xx_hal_tim.o(i.HAL_TIM_IC_Start_DMA) refers to stm32f1xx_hal_tim.o(i.TIM_DMAError) for TIM_DMAError
    stm32f1xx_hal_tim.o(i.HAL_TIM_IC_Start_IT) refers to stm32f1xx_hal_tim.o(i.TIM_CCxChannelCmd) for TIM_CCxChannelCmd
    stm32f1xx_hal_tim.o(i.HAL_TIM_IC_Stop) refers to stm32f1xx_hal_tim.o(i.TIM_CCxChannelCmd) for TIM_CCxChannelCmd
    stm32f1xx_hal_tim.o(i.HAL_TIM_IC_Stop_DMA) refers to stm32f1xx_hal_tim.o(i.TIM_CCxChannelCmd) for TIM_CCxChannelCmd
    stm32f1xx_hal_tim.o(i.HAL_TIM_IC_Stop_DMA) refers to stm32f1xx_hal_dma.o(i.HAL_DMA_Abort_IT) for HAL_DMA_Abort_IT
    stm32f1xx_hal_tim.o(i.HAL_TIM_IC_Stop_IT) refers to stm32f1xx_hal_tim.o(i.TIM_CCxChannelCmd) for TIM_CCxChannelCmd
    stm32f1xx_hal_tim.o(i.HAL_TIM_IRQHandler) refers to stm32f1xx_hal_tim.o(i.HAL_TIM_IC_CaptureCallback) for HAL_TIM_IC_CaptureCallback
    stm32f1xx_hal_tim.o(i.HAL_TIM_IRQHandler) refers to stm32f1xx_hal_tim.o(i.HAL_TIM_OC_DelayElapsedCallback) for HAL_TIM_OC_DelayElapsedCallback
    stm32f1xx_hal_tim.o(i.HAL_TIM_IRQHandler) refers to stm32f1xx_hal_tim.o(i.HAL_TIM_PWM_PulseFinishedCallback) for HAL_TIM_PWM_PulseFinishedCallback
    stm32f1xx_hal_tim.o(i.HAL_TIM_IRQHandler) refers to stm32f1xx_hal_tim.o(i.HAL_TIM_PeriodElapsedCallback) for HAL_TIM_PeriodElapsedCallback
    stm32f1xx_hal_tim.o(i.HAL_TIM_IRQHandler) refers to stm32f1xx_hal_tim_ex.o(i.HAL_TIMEx_BreakCallback) for HAL_TIMEx_BreakCallback
    stm32f1xx_hal_tim.o(i.HAL_TIM_IRQHandler) refers to stm32f1xx_hal_tim.o(i.HAL_TIM_TriggerCallback) for HAL_TIM_TriggerCallback
    stm32f1xx_hal_tim.o(i.HAL_TIM_IRQHandler) refers to stm32f1xx_hal_tim_ex.o(i.HAL_TIMEx_CommutCallback) for HAL_TIMEx_CommutCallback
    stm32f1xx_hal_tim.o(i.HAL_TIM_OC_ConfigChannel) refers to stm32f1xx_hal_tim.o(i.TIM_OC1_SetConfig) for TIM_OC1_SetConfig
    stm32f1xx_hal_tim.o(i.HAL_TIM_OC_ConfigChannel) refers to stm32f1xx_hal_tim.o(i.TIM_OC2_SetConfig) for TIM_OC2_SetConfig
    stm32f1xx_hal_tim.o(i.HAL_TIM_OC_ConfigChannel) refers to stm32f1xx_hal_tim.o(i.TIM_OC3_SetConfig) for TIM_OC3_SetConfig
    stm32f1xx_hal_tim.o(i.HAL_TIM_OC_ConfigChannel) refers to stm32f1xx_hal_tim.o(i.TIM_OC4_SetConfig) for TIM_OC4_SetConfig
    stm32f1xx_hal_tim.o(i.HAL_TIM_OC_DeInit) refers to stm32f1xx_hal_tim.o(i.HAL_TIM_OC_MspDeInit) for HAL_TIM_OC_MspDeInit
    stm32f1xx_hal_tim.o(i.HAL_TIM_OC_Init) refers to stm32f1xx_hal_tim.o(i.HAL_TIM_OC_MspInit) for HAL_TIM_OC_MspInit
    stm32f1xx_hal_tim.o(i.HAL_TIM_OC_Init) refers to stm32f1xx_hal_tim.o(i.TIM_Base_SetConfig) for TIM_Base_SetConfig
    stm32f1xx_hal_tim.o(i.HAL_TIM_OC_Start) refers to stm32f1xx_hal_tim.o(i.TIM_CCxChannelCmd) for TIM_CCxChannelCmd
    stm32f1xx_hal_tim.o(i.HAL_TIM_OC_Start_DMA) refers to stm32f1xx_hal_dma.o(i.HAL_DMA_Start_IT) for HAL_DMA_Start_IT
    stm32f1xx_hal_tim.o(i.HAL_TIM_OC_Start_DMA) refers to stm32f1xx_hal_tim.o(i.TIM_CCxChannelCmd) for TIM_CCxChannelCmd
    stm32f1xx_hal_tim.o(i.HAL_TIM_OC_Start_DMA) refers to stm32f1xx_hal_tim.o(i.TIM_DMADelayPulseCplt) for TIM_DMADelayPulseCplt
    stm32f1xx_hal_tim.o(i.HAL_TIM_OC_Start_DMA) refers to stm32f1xx_hal_tim.o(i.TIM_DMADelayPulseHalfCplt) for TIM_DMADelayPulseHalfCplt
    stm32f1xx_hal_tim.o(i.HAL_TIM_OC_Start_DMA) refers to stm32f1xx_hal_tim.o(i.TIM_DMAError) for TIM_DMAError
    stm32f1xx_hal_tim.o(i.HAL_TIM_OC_Start_IT) refers to stm32f1xx_hal_tim.o(i.TIM_CCxChannelCmd) for TIM_CCxChannelCmd
    stm32f1xx_hal_tim.o(i.HAL_TIM_OC_Stop) refers to stm32f1xx_hal_tim.o(i.TIM_CCxChannelCmd) for TIM_CCxChannelCmd
    stm32f1xx_hal_tim.o(i.HAL_TIM_OC_Stop_DMA) refers to stm32f1xx_hal_dma.o(i.HAL_DMA_Abort_IT) for HAL_DMA_Abort_IT
    stm32f1xx_hal_tim.o(i.HAL_TIM_OC_Stop_DMA) refers to stm32f1xx_hal_tim.o(i.TIM_CCxChannelCmd) for TIM_CCxChannelCmd
    stm32f1xx_hal_tim.o(i.HAL_TIM_OC_Stop_IT) refers to stm32f1xx_hal_tim.o(i.TIM_CCxChannelCmd) for TIM_CCxChannelCmd
    stm32f1xx_hal_tim.o(i.HAL_TIM_OnePulse_ConfigChannel) refers to stm32f1xx_hal_tim.o(i.TIM_OC1_SetConfig) for TIM_OC1_SetConfig
    stm32f1xx_hal_tim.o(i.HAL_TIM_OnePulse_ConfigChannel) refers to stm32f1xx_hal_tim.o(i.TIM_OC2_SetConfig) for TIM_OC2_SetConfig
    stm32f1xx_hal_tim.o(i.HAL_TIM_OnePulse_ConfigChannel) refers to stm32f1xx_hal_tim.o(i.TIM_TI1_SetConfig) for TIM_TI1_SetConfig
    stm32f1xx_hal_tim.o(i.HAL_TIM_OnePulse_ConfigChannel) refers to stm32f1xx_hal_tim.o(i.TIM_TI2_SetConfig) for TIM_TI2_SetConfig
    stm32f1xx_hal_tim.o(i.HAL_TIM_OnePulse_DeInit) refers to stm32f1xx_hal_tim.o(i.HAL_TIM_OnePulse_MspDeInit) for HAL_TIM_OnePulse_MspDeInit
    stm32f1xx_hal_tim.o(i.HAL_TIM_OnePulse_Init) refers to stm32f1xx_hal_tim.o(i.HAL_TIM_OnePulse_MspInit) for HAL_TIM_OnePulse_MspInit
    stm32f1xx_hal_tim.o(i.HAL_TIM_OnePulse_Init) refers to stm32f1xx_hal_tim.o(i.TIM_Base_SetConfig) for TIM_Base_SetConfig
    stm32f1xx_hal_tim.o(i.HAL_TIM_OnePulse_Start) refers to stm32f1xx_hal_tim.o(i.TIM_CCxChannelCmd) for TIM_CCxChannelCmd
    stm32f1xx_hal_tim.o(i.HAL_TIM_OnePulse_Start_IT) refers to stm32f1xx_hal_tim.o(i.TIM_CCxChannelCmd) for TIM_CCxChannelCmd
    stm32f1xx_hal_tim.o(i.HAL_TIM_OnePulse_Stop) refers to stm32f1xx_hal_tim.o(i.TIM_CCxChannelCmd) for TIM_CCxChannelCmd
    stm32f1xx_hal_tim.o(i.HAL_TIM_OnePulse_Stop_IT) refers to stm32f1xx_hal_tim.o(i.TIM_CCxChannelCmd) for TIM_CCxChannelCmd
    stm32f1xx_hal_tim.o(i.HAL_TIM_PWM_ConfigChannel) refers to stm32f1xx_hal_tim.o(i.TIM_OC1_SetConfig) for TIM_OC1_SetConfig
    stm32f1xx_hal_tim.o(i.HAL_TIM_PWM_ConfigChannel) refers to stm32f1xx_hal_tim.o(i.TIM_OC2_SetConfig) for TIM_OC2_SetConfig
    stm32f1xx_hal_tim.o(i.HAL_TIM_PWM_ConfigChannel) refers to stm32f1xx_hal_tim.o(i.TIM_OC3_SetConfig) for TIM_OC3_SetConfig
    stm32f1xx_hal_tim.o(i.HAL_TIM_PWM_ConfigChannel) refers to stm32f1xx_hal_tim.o(i.TIM_OC4_SetConfig) for TIM_OC4_SetConfig
    stm32f1xx_hal_tim.o(i.HAL_TIM_PWM_DeInit) refers to stm32f1xx_hal_tim.o(i.HAL_TIM_PWM_MspDeInit) for HAL_TIM_PWM_MspDeInit
    stm32f1xx_hal_tim.o(i.HAL_TIM_PWM_Init) refers to stm32f1xx_hal_tim.o(i.HAL_TIM_PWM_MspInit) for HAL_TIM_PWM_MspInit
    stm32f1xx_hal_tim.o(i.HAL_TIM_PWM_Init) refers to stm32f1xx_hal_tim.o(i.TIM_Base_SetConfig) for TIM_Base_SetConfig
    stm32f1xx_hal_tim.o(i.HAL_TIM_PWM_Start) refers to stm32f1xx_hal_tim.o(i.TIM_CCxChannelCmd) for TIM_CCxChannelCmd
    stm32f1xx_hal_tim.o(i.HAL_TIM_PWM_Start_DMA) refers to stm32f1xx_hal_dma.o(i.HAL_DMA_Start_IT) for HAL_DMA_Start_IT
    stm32f1xx_hal_tim.o(i.HAL_TIM_PWM_Start_DMA) refers to stm32f1xx_hal_tim.o(i.TIM_CCxChannelCmd) for TIM_CCxChannelCmd
    stm32f1xx_hal_tim.o(i.HAL_TIM_PWM_Start_DMA) refers to stm32f1xx_hal_tim.o(i.TIM_DMADelayPulseCplt) for TIM_DMADelayPulseCplt
    stm32f1xx_hal_tim.o(i.HAL_TIM_PWM_Start_DMA) refers to stm32f1xx_hal_tim.o(i.TIM_DMADelayPulseHalfCplt) for TIM_DMADelayPulseHalfCplt
    stm32f1xx_hal_tim.o(i.HAL_TIM_PWM_Start_DMA) refers to stm32f1xx_hal_tim.o(i.TIM_DMAError) for TIM_DMAError
    stm32f1xx_hal_tim.o(i.HAL_TIM_PWM_Start_IT) refers to stm32f1xx_hal_tim.o(i.TIM_CCxChannelCmd) for TIM_CCxChannelCmd
    stm32f1xx_hal_tim.o(i.HAL_TIM_PWM_Stop) refers to stm32f1xx_hal_tim.o(i.TIM_CCxChannelCmd) for TIM_CCxChannelCmd
    stm32f1xx_hal_tim.o(i.HAL_TIM_PWM_Stop_DMA) refers to stm32f1xx_hal_dma.o(i.HAL_DMA_Abort_IT) for HAL_DMA_Abort_IT
    stm32f1xx_hal_tim.o(i.HAL_TIM_PWM_Stop_DMA) refers to stm32f1xx_hal_tim.o(i.TIM_CCxChannelCmd) for TIM_CCxChannelCmd
    stm32f1xx_hal_tim.o(i.HAL_TIM_PWM_Stop_IT) refers to stm32f1xx_hal_tim.o(i.TIM_CCxChannelCmd) for TIM_CCxChannelCmd
    stm32f1xx_hal_tim.o(i.HAL_TIM_SlaveConfigSynchro) refers to stm32f1xx_hal_tim.o(i.TIM_SlaveTimer_SetConfig) for TIM_SlaveTimer_SetConfig
    stm32f1xx_hal_tim.o(i.HAL_TIM_SlaveConfigSynchro_IT) refers to stm32f1xx_hal_tim.o(i.TIM_SlaveTimer_SetConfig) for TIM_SlaveTimer_SetConfig
    stm32f1xx_hal_tim.o(i.TIM_DMACaptureCplt) refers to stm32f1xx_hal_tim.o(i.HAL_TIM_IC_CaptureCallback) for HAL_TIM_IC_CaptureCallback
    stm32f1xx_hal_tim.o(i.TIM_DMACaptureHalfCplt) refers to stm32f1xx_hal_tim.o(i.HAL_TIM_IC_CaptureHalfCpltCallback) for HAL_TIM_IC_CaptureHalfCpltCallback
    stm32f1xx_hal_tim.o(i.TIM_DMADelayPulseCplt) refers to stm32f1xx_hal_tim.o(i.HAL_TIM_PWM_PulseFinishedCallback) for HAL_TIM_PWM_PulseFinishedCallback
    stm32f1xx_hal_tim.o(i.TIM_DMADelayPulseHalfCplt) refers to stm32f1xx_hal_tim.o(i.HAL_TIM_PWM_PulseFinishedHalfCpltCallback) for HAL_TIM_PWM_PulseFinishedHalfCpltCallback
    stm32f1xx_hal_tim.o(i.TIM_DMAError) refers to stm32f1xx_hal_tim.o(i.HAL_TIM_ErrorCallback) for HAL_TIM_ErrorCallback
    stm32f1xx_hal_tim.o(i.TIM_DMAPeriodElapsedCplt) refers to stm32f1xx_hal_tim.o(i.HAL_TIM_PeriodElapsedCallback) for HAL_TIM_PeriodElapsedCallback
    stm32f1xx_hal_tim.o(i.TIM_DMAPeriodElapsedHalfCplt) refers to stm32f1xx_hal_tim.o(i.HAL_TIM_PeriodElapsedHalfCpltCallback) for HAL_TIM_PeriodElapsedHalfCpltCallback
    stm32f1xx_hal_tim.o(i.TIM_DMATriggerCplt) refers to stm32f1xx_hal_tim.o(i.HAL_TIM_TriggerCallback) for HAL_TIM_TriggerCallback
    stm32f1xx_hal_tim.o(i.TIM_DMATriggerHalfCplt) refers to stm32f1xx_hal_tim.o(i.HAL_TIM_TriggerHalfCpltCallback) for HAL_TIM_TriggerHalfCpltCallback
    stm32f1xx_hal_tim.o(i.TIM_SlaveTimer_SetConfig) refers to stm32f1xx_hal_tim.o(i.TIM_ETR_SetConfig) for TIM_ETR_SetConfig
    stm32f1xx_hal_tim.o(i.TIM_SlaveTimer_SetConfig) refers to stm32f1xx_hal_tim.o(i.TIM_TI1_ConfigInputStage) for TIM_TI1_ConfigInputStage
    stm32f1xx_hal_tim.o(i.TIM_SlaveTimer_SetConfig) refers to stm32f1xx_hal_tim.o(i.TIM_TI2_ConfigInputStage) for TIM_TI2_ConfigInputStage
    stm32f1xx_hal_tim_ex.o(i.HAL_TIMEx_ConfigCommutEvent_DMA) refers to stm32f1xx_hal_tim_ex.o(i.TIMEx_DMACommutationCplt) for TIMEx_DMACommutationCplt
    stm32f1xx_hal_tim_ex.o(i.HAL_TIMEx_ConfigCommutEvent_DMA) refers to stm32f1xx_hal_tim_ex.o(i.TIMEx_DMACommutationHalfCplt) for TIMEx_DMACommutationHalfCplt
    stm32f1xx_hal_tim_ex.o(i.HAL_TIMEx_ConfigCommutEvent_DMA) refers to stm32f1xx_hal_tim.o(i.TIM_DMAError) for TIM_DMAError
    stm32f1xx_hal_tim_ex.o(i.HAL_TIMEx_HallSensor_DeInit) refers to stm32f1xx_hal_tim_ex.o(i.HAL_TIMEx_HallSensor_MspDeInit) for HAL_TIMEx_HallSensor_MspDeInit
    stm32f1xx_hal_tim_ex.o(i.HAL_TIMEx_HallSensor_Init) refers to stm32f1xx_hal_tim_ex.o(i.HAL_TIMEx_HallSensor_MspInit) for HAL_TIMEx_HallSensor_MspInit
    stm32f1xx_hal_tim_ex.o(i.HAL_TIMEx_HallSensor_Init) refers to stm32f1xx_hal_tim.o(i.TIM_Base_SetConfig) for TIM_Base_SetConfig
    stm32f1xx_hal_tim_ex.o(i.HAL_TIMEx_HallSensor_Init) refers to stm32f1xx_hal_tim.o(i.TIM_TI1_SetConfig) for TIM_TI1_SetConfig
    stm32f1xx_hal_tim_ex.o(i.HAL_TIMEx_HallSensor_Init) refers to stm32f1xx_hal_tim.o(i.TIM_OC2_SetConfig) for TIM_OC2_SetConfig
    stm32f1xx_hal_tim_ex.o(i.HAL_TIMEx_HallSensor_Start) refers to stm32f1xx_hal_tim.o(i.TIM_CCxChannelCmd) for TIM_CCxChannelCmd
    stm32f1xx_hal_tim_ex.o(i.HAL_TIMEx_HallSensor_Start_DMA) refers to stm32f1xx_hal_tim.o(i.TIM_CCxChannelCmd) for TIM_CCxChannelCmd
    stm32f1xx_hal_tim_ex.o(i.HAL_TIMEx_HallSensor_Start_DMA) refers to stm32f1xx_hal_dma.o(i.HAL_DMA_Start_IT) for HAL_DMA_Start_IT
    stm32f1xx_hal_tim_ex.o(i.HAL_TIMEx_HallSensor_Start_DMA) refers to stm32f1xx_hal_tim.o(i.TIM_DMACaptureCplt) for TIM_DMACaptureCplt
    stm32f1xx_hal_tim_ex.o(i.HAL_TIMEx_HallSensor_Start_DMA) refers to stm32f1xx_hal_tim.o(i.TIM_DMACaptureHalfCplt) for TIM_DMACaptureHalfCplt
    stm32f1xx_hal_tim_ex.o(i.HAL_TIMEx_HallSensor_Start_DMA) refers to stm32f1xx_hal_tim.o(i.TIM_DMAError) for TIM_DMAError
    stm32f1xx_hal_tim_ex.o(i.HAL_TIMEx_HallSensor_Start_IT) refers to stm32f1xx_hal_tim.o(i.TIM_CCxChannelCmd) for TIM_CCxChannelCmd
    stm32f1xx_hal_tim_ex.o(i.HAL_TIMEx_HallSensor_Stop) refers to stm32f1xx_hal_tim.o(i.TIM_CCxChannelCmd) for TIM_CCxChannelCmd
    stm32f1xx_hal_tim_ex.o(i.HAL_TIMEx_HallSensor_Stop_DMA) refers to stm32f1xx_hal_tim.o(i.TIM_CCxChannelCmd) for TIM_CCxChannelCmd
    stm32f1xx_hal_tim_ex.o(i.HAL_TIMEx_HallSensor_Stop_DMA) refers to stm32f1xx_hal_dma.o(i.HAL_DMA_Abort_IT) for HAL_DMA_Abort_IT
    stm32f1xx_hal_tim_ex.o(i.HAL_TIMEx_HallSensor_Stop_IT) refers to stm32f1xx_hal_tim.o(i.TIM_CCxChannelCmd) for TIM_CCxChannelCmd
    stm32f1xx_hal_tim_ex.o(i.HAL_TIMEx_OCN_Start) refers to stm32f1xx_hal_tim_ex.o(i.TIM_CCxNChannelCmd) for TIM_CCxNChannelCmd
    stm32f1xx_hal_tim_ex.o(i.HAL_TIMEx_OCN_Start_DMA) refers to stm32f1xx_hal_dma.o(i.HAL_DMA_Start_IT) for HAL_DMA_Start_IT
    stm32f1xx_hal_tim_ex.o(i.HAL_TIMEx_OCN_Start_DMA) refers to stm32f1xx_hal_tim_ex.o(i.TIM_CCxNChannelCmd) for TIM_CCxNChannelCmd
    stm32f1xx_hal_tim_ex.o(i.HAL_TIMEx_OCN_Start_DMA) refers to stm32f1xx_hal_tim_ex.o(i.TIM_DMADelayPulseNCplt) for TIM_DMADelayPulseNCplt
    stm32f1xx_hal_tim_ex.o(i.HAL_TIMEx_OCN_Start_DMA) refers to stm32f1xx_hal_tim.o(i.TIM_DMADelayPulseHalfCplt) for TIM_DMADelayPulseHalfCplt
    stm32f1xx_hal_tim_ex.o(i.HAL_TIMEx_OCN_Start_DMA) refers to stm32f1xx_hal_tim_ex.o(i.TIM_DMAErrorCCxN) for TIM_DMAErrorCCxN
    stm32f1xx_hal_tim_ex.o(i.HAL_TIMEx_OCN_Start_IT) refers to stm32f1xx_hal_tim_ex.o(i.TIM_CCxNChannelCmd) for TIM_CCxNChannelCmd
    stm32f1xx_hal_tim_ex.o(i.HAL_TIMEx_OCN_Stop) refers to stm32f1xx_hal_tim_ex.o(i.TIM_CCxNChannelCmd) for TIM_CCxNChannelCmd
    stm32f1xx_hal_tim_ex.o(i.HAL_TIMEx_OCN_Stop_DMA) refers to stm32f1xx_hal_dma.o(i.HAL_DMA_Abort_IT) for HAL_DMA_Abort_IT
    stm32f1xx_hal_tim_ex.o(i.HAL_TIMEx_OCN_Stop_DMA) refers to stm32f1xx_hal_tim_ex.o(i.TIM_CCxNChannelCmd) for TIM_CCxNChannelCmd
    stm32f1xx_hal_tim_ex.o(i.HAL_TIMEx_OCN_Stop_IT) refers to stm32f1xx_hal_tim_ex.o(i.TIM_CCxNChannelCmd) for TIM_CCxNChannelCmd
    stm32f1xx_hal_tim_ex.o(i.HAL_TIMEx_OnePulseN_Start) refers to stm32f1xx_hal_tim_ex.o(i.TIM_CCxNChannelCmd) for TIM_CCxNChannelCmd
    stm32f1xx_hal_tim_ex.o(i.HAL_TIMEx_OnePulseN_Start) refers to stm32f1xx_hal_tim.o(i.TIM_CCxChannelCmd) for TIM_CCxChannelCmd
    stm32f1xx_hal_tim_ex.o(i.HAL_TIMEx_OnePulseN_Start_IT) refers to stm32f1xx_hal_tim_ex.o(i.TIM_CCxNChannelCmd) for TIM_CCxNChannelCmd
    stm32f1xx_hal_tim_ex.o(i.HAL_TIMEx_OnePulseN_Start_IT) refers to stm32f1xx_hal_tim.o(i.TIM_CCxChannelCmd) for TIM_CCxChannelCmd
    stm32f1xx_hal_tim_ex.o(i.HAL_TIMEx_OnePulseN_Stop) refers to stm32f1xx_hal_tim_ex.o(i.TIM_CCxNChannelCmd) for TIM_CCxNChannelCmd
    stm32f1xx_hal_tim_ex.o(i.HAL_TIMEx_OnePulseN_Stop) refers to stm32f1xx_hal_tim.o(i.TIM_CCxChannelCmd) for TIM_CCxChannelCmd
    stm32f1xx_hal_tim_ex.o(i.HAL_TIMEx_OnePulseN_Stop_IT) refers to stm32f1xx_hal_tim_ex.o(i.TIM_CCxNChannelCmd) for TIM_CCxNChannelCmd
    stm32f1xx_hal_tim_ex.o(i.HAL_TIMEx_OnePulseN_Stop_IT) refers to stm32f1xx_hal_tim.o(i.TIM_CCxChannelCmd) for TIM_CCxChannelCmd
    stm32f1xx_hal_tim_ex.o(i.HAL_TIMEx_PWMN_Start) refers to stm32f1xx_hal_tim_ex.o(i.TIM_CCxNChannelCmd) for TIM_CCxNChannelCmd
    stm32f1xx_hal_tim_ex.o(i.HAL_TIMEx_PWMN_Start_DMA) refers to stm32f1xx_hal_dma.o(i.HAL_DMA_Start_IT) for HAL_DMA_Start_IT
    stm32f1xx_hal_tim_ex.o(i.HAL_TIMEx_PWMN_Start_DMA) refers to stm32f1xx_hal_tim_ex.o(i.TIM_CCxNChannelCmd) for TIM_CCxNChannelCmd
    stm32f1xx_hal_tim_ex.o(i.HAL_TIMEx_PWMN_Start_DMA) refers to stm32f1xx_hal_tim_ex.o(i.TIM_DMADelayPulseNCplt) for TIM_DMADelayPulseNCplt
    stm32f1xx_hal_tim_ex.o(i.HAL_TIMEx_PWMN_Start_DMA) refers to stm32f1xx_hal_tim.o(i.TIM_DMADelayPulseHalfCplt) for TIM_DMADelayPulseHalfCplt
    stm32f1xx_hal_tim_ex.o(i.HAL_TIMEx_PWMN_Start_DMA) refers to stm32f1xx_hal_tim_ex.o(i.TIM_DMAErrorCCxN) for TIM_DMAErrorCCxN
    stm32f1xx_hal_tim_ex.o(i.HAL_TIMEx_PWMN_Start_IT) refers to stm32f1xx_hal_tim_ex.o(i.TIM_CCxNChannelCmd) for TIM_CCxNChannelCmd
    stm32f1xx_hal_tim_ex.o(i.HAL_TIMEx_PWMN_Stop) refers to stm32f1xx_hal_tim_ex.o(i.TIM_CCxNChannelCmd) for TIM_CCxNChannelCmd
    stm32f1xx_hal_tim_ex.o(i.HAL_TIMEx_PWMN_Stop_DMA) refers to stm32f1xx_hal_dma.o(i.HAL_DMA_Abort_IT) for HAL_DMA_Abort_IT
    stm32f1xx_hal_tim_ex.o(i.HAL_TIMEx_PWMN_Stop_DMA) refers to stm32f1xx_hal_tim_ex.o(i.TIM_CCxNChannelCmd) for TIM_CCxNChannelCmd
    stm32f1xx_hal_tim_ex.o(i.HAL_TIMEx_PWMN_Stop_IT) refers to stm32f1xx_hal_tim_ex.o(i.TIM_CCxNChannelCmd) for TIM_CCxNChannelCmd
    stm32f1xx_hal_tim_ex.o(i.TIMEx_DMACommutationCplt) refers to stm32f1xx_hal_tim_ex.o(i.HAL_TIMEx_CommutCallback) for HAL_TIMEx_CommutCallback
    stm32f1xx_hal_tim_ex.o(i.TIMEx_DMACommutationHalfCplt) refers to stm32f1xx_hal_tim_ex.o(i.HAL_TIMEx_CommutHalfCpltCallback) for HAL_TIMEx_CommutHalfCpltCallback
    stm32f1xx_hal_tim_ex.o(i.TIM_DMADelayPulseNCplt) refers to stm32f1xx_hal_tim.o(i.HAL_TIM_PWM_PulseFinishedCallback) for HAL_TIM_PWM_PulseFinishedCallback
    stm32f1xx_hal_tim_ex.o(i.TIM_DMAErrorCCxN) refers to stm32f1xx_hal_tim.o(i.HAL_TIM_ErrorCallback) for HAL_TIM_ErrorCallback
    stm32f1xx_hal_uart.o(i.HAL_HalfDuplex_Init) refers to usart.o(i.HAL_UART_MspInit) for HAL_UART_MspInit
    stm32f1xx_hal_uart.o(i.HAL_HalfDuplex_Init) refers to stm32f1xx_hal_uart.o(i.UART_SetConfig) for UART_SetConfig
    stm32f1xx_hal_uart.o(i.HAL_LIN_Init) refers to usart.o(i.HAL_UART_MspInit) for HAL_UART_MspInit
    stm32f1xx_hal_uart.o(i.HAL_LIN_Init) refers to stm32f1xx_hal_uart.o(i.UART_SetConfig) for UART_SetConfig
    stm32f1xx_hal_uart.o(i.HAL_MultiProcessor_Init) refers to usart.o(i.HAL_UART_MspInit) for HAL_UART_MspInit
    stm32f1xx_hal_uart.o(i.HAL_MultiProcessor_Init) refers to stm32f1xx_hal_uart.o(i.UART_SetConfig) for UART_SetConfig
    stm32f1xx_hal_uart.o(i.HAL_UARTEx_ReceiveToIdle) refers to stm32f1xx_hal.o(i.HAL_GetTick) for HAL_GetTick
    stm32f1xx_hal_uart.o(i.HAL_UARTEx_ReceiveToIdle_DMA) refers to stm32f1xx_hal_uart.o(i.UART_Start_Receive_DMA) for UART_Start_Receive_DMA
    stm32f1xx_hal_uart.o(i.HAL_UARTEx_ReceiveToIdle_IT) refers to stm32f1xx_hal_uart.o(i.UART_Start_Receive_IT) for UART_Start_Receive_IT
    stm32f1xx_hal_uart.o(i.HAL_UART_Abort) refers to stm32f1xx_hal_dma.o(i.HAL_DMA_Abort) for HAL_DMA_Abort
    stm32f1xx_hal_uart.o(i.HAL_UART_Abort) refers to stm32f1xx_hal_dma.o(i.HAL_DMA_GetError) for HAL_DMA_GetError
    stm32f1xx_hal_uart.o(i.HAL_UART_AbortReceive) refers to stm32f1xx_hal_dma.o(i.HAL_DMA_Abort) for HAL_DMA_Abort
    stm32f1xx_hal_uart.o(i.HAL_UART_AbortReceive) refers to stm32f1xx_hal_dma.o(i.HAL_DMA_GetError) for HAL_DMA_GetError
    stm32f1xx_hal_uart.o(i.HAL_UART_AbortReceive_IT) refers to stm32f1xx_hal_dma.o(i.HAL_DMA_Abort_IT) for HAL_DMA_Abort_IT
    stm32f1xx_hal_uart.o(i.HAL_UART_AbortReceive_IT) refers to uart.o(i.HAL_UART_AbortReceiveCpltCallback) for HAL_UART_AbortReceiveCpltCallback
    stm32f1xx_hal_uart.o(i.HAL_UART_AbortReceive_IT) refers to stm32f1xx_hal_uart.o(i.UART_DMARxOnlyAbortCallback) for UART_DMARxOnlyAbortCallback
    stm32f1xx_hal_uart.o(i.HAL_UART_AbortTransmit) refers to stm32f1xx_hal_dma.o(i.HAL_DMA_Abort) for HAL_DMA_Abort
    stm32f1xx_hal_uart.o(i.HAL_UART_AbortTransmit) refers to stm32f1xx_hal_dma.o(i.HAL_DMA_GetError) for HAL_DMA_GetError
    stm32f1xx_hal_uart.o(i.HAL_UART_AbortTransmit_IT) refers to stm32f1xx_hal_dma.o(i.HAL_DMA_Abort_IT) for HAL_DMA_Abort_IT
    stm32f1xx_hal_uart.o(i.HAL_UART_AbortTransmit_IT) refers to uart.o(i.HAL_UART_AbortTransmitCpltCallback) for HAL_UART_AbortTransmitCpltCallback
    stm32f1xx_hal_uart.o(i.HAL_UART_AbortTransmit_IT) refers to stm32f1xx_hal_uart.o(i.UART_DMATxOnlyAbortCallback) for UART_DMATxOnlyAbortCallback
    stm32f1xx_hal_uart.o(i.HAL_UART_Abort_IT) refers to stm32f1xx_hal_dma.o(i.HAL_DMA_Abort_IT) for HAL_DMA_Abort_IT
    stm32f1xx_hal_uart.o(i.HAL_UART_Abort_IT) refers to uart.o(i.HAL_UART_AbortCpltCallback) for HAL_UART_AbortCpltCallback
    stm32f1xx_hal_uart.o(i.HAL_UART_Abort_IT) refers to stm32f1xx_hal_uart.o(i.UART_DMATxAbortCallback) for UART_DMATxAbortCallback
    stm32f1xx_hal_uart.o(i.HAL_UART_Abort_IT) refers to stm32f1xx_hal_uart.o(i.UART_DMARxAbortCallback) for UART_DMARxAbortCallback
    stm32f1xx_hal_uart.o(i.HAL_UART_DMAStop) refers to stm32f1xx_hal_dma.o(i.HAL_DMA_Abort) for HAL_DMA_Abort
    stm32f1xx_hal_uart.o(i.HAL_UART_DMAStop) refers to stm32f1xx_hal_uart.o(i.UART_EndTxTransfer) for UART_EndTxTransfer
    stm32f1xx_hal_uart.o(i.HAL_UART_DMAStop) refers to stm32f1xx_hal_uart.o(i.UART_EndRxTransfer) for UART_EndRxTransfer
    stm32f1xx_hal_uart.o(i.HAL_UART_DeInit) refers to usart.o(i.HAL_UART_MspDeInit) for HAL_UART_MspDeInit
    stm32f1xx_hal_uart.o(i.HAL_UART_IRQHandler) refers to stm32f1xx_hal_uart.o(i.UART_Receive_IT) for UART_Receive_IT
    stm32f1xx_hal_uart.o(i.HAL_UART_IRQHandler) refers to stm32f1xx_hal_uart.o(i.UART_EndRxTransfer) for UART_EndRxTransfer
    stm32f1xx_hal_uart.o(i.HAL_UART_IRQHandler) refers to stm32f1xx_hal_dma.o(i.HAL_DMA_Abort_IT) for HAL_DMA_Abort_IT
    stm32f1xx_hal_uart.o(i.HAL_UART_IRQHandler) refers to uart.o(i.HAL_UART_ErrorCallback) for HAL_UART_ErrorCallback
    stm32f1xx_hal_uart.o(i.HAL_UART_IRQHandler) refers to stm32f1xx_hal_dma.o(i.HAL_DMA_Abort) for HAL_DMA_Abort
    stm32f1xx_hal_uart.o(i.HAL_UART_IRQHandler) refers to stm32f1xx_hal_uart.o(i.HAL_UARTEx_RxEventCallback) for HAL_UARTEx_RxEventCallback
    stm32f1xx_hal_uart.o(i.HAL_UART_IRQHandler) refers to uart.o(i.HAL_UART_TxCpltCallback) for HAL_UART_TxCpltCallback
    stm32f1xx_hal_uart.o(i.HAL_UART_IRQHandler) refers to stm32f1xx_hal_uart.o(i.UART_DMAAbortOnError) for UART_DMAAbortOnError
    stm32f1xx_hal_uart.o(i.HAL_UART_Init) refers to usart.o(i.HAL_UART_MspInit) for HAL_UART_MspInit
    stm32f1xx_hal_uart.o(i.HAL_UART_Init) refers to stm32f1xx_hal_uart.o(i.UART_SetConfig) for UART_SetConfig
    stm32f1xx_hal_uart.o(i.HAL_UART_Receive) refers to stm32f1xx_hal.o(i.HAL_GetTick) for HAL_GetTick
    stm32f1xx_hal_uart.o(i.HAL_UART_Receive) refers to stm32f1xx_hal_uart.o(i.UART_WaitOnFlagUntilTimeout) for UART_WaitOnFlagUntilTimeout
    stm32f1xx_hal_uart.o(i.HAL_UART_Receive_DMA) refers to stm32f1xx_hal_uart.o(i.UART_Start_Receive_DMA) for UART_Start_Receive_DMA
    stm32f1xx_hal_uart.o(i.HAL_UART_Receive_IT) refers to stm32f1xx_hal_uart.o(i.UART_Start_Receive_IT) for UART_Start_Receive_IT
    stm32f1xx_hal_uart.o(i.HAL_UART_Transmit) refers to stm32f1xx_hal.o(i.HAL_GetTick) for HAL_GetTick
    stm32f1xx_hal_uart.o(i.HAL_UART_Transmit) refers to stm32f1xx_hal_uart.o(i.UART_WaitOnFlagUntilTimeout) for UART_WaitOnFlagUntilTimeout
    stm32f1xx_hal_uart.o(i.HAL_UART_Transmit_DMA) refers to stm32f1xx_hal_dma.o(i.HAL_DMA_Start_IT) for HAL_DMA_Start_IT
    stm32f1xx_hal_uart.o(i.HAL_UART_Transmit_DMA) refers to stm32f1xx_hal_uart.o(i.UART_DMATransmitCplt) for UART_DMATransmitCplt
    stm32f1xx_hal_uart.o(i.HAL_UART_Transmit_DMA) refers to stm32f1xx_hal_uart.o(i.UART_DMATxHalfCplt) for UART_DMATxHalfCplt
    stm32f1xx_hal_uart.o(i.HAL_UART_Transmit_DMA) refers to stm32f1xx_hal_uart.o(i.UART_DMAError) for UART_DMAError
    stm32f1xx_hal_uart.o(i.UART_DMAAbortOnError) refers to uart.o(i.HAL_UART_ErrorCallback) for HAL_UART_ErrorCallback
    stm32f1xx_hal_uart.o(i.UART_DMAError) refers to stm32f1xx_hal_uart.o(i.UART_EndTxTransfer) for UART_EndTxTransfer
    stm32f1xx_hal_uart.o(i.UART_DMAError) refers to stm32f1xx_hal_uart.o(i.UART_EndRxTransfer) for UART_EndRxTransfer
    stm32f1xx_hal_uart.o(i.UART_DMAError) refers to uart.o(i.HAL_UART_ErrorCallback) for HAL_UART_ErrorCallback
    stm32f1xx_hal_uart.o(i.UART_DMAReceiveCplt) refers to uart.o(i.HAL_UART_RxCpltCallback) for HAL_UART_RxCpltCallback
    stm32f1xx_hal_uart.o(i.UART_DMAReceiveCplt) refers to stm32f1xx_hal_uart.o(i.HAL_UARTEx_RxEventCallback) for HAL_UARTEx_RxEventCallback
    stm32f1xx_hal_uart.o(i.UART_DMARxAbortCallback) refers to uart.o(i.HAL_UART_AbortCpltCallback) for HAL_UART_AbortCpltCallback
    stm32f1xx_hal_uart.o(i.UART_DMARxHalfCplt) refers to uart.o(i.HAL_UART_RxHalfCpltCallback) for HAL_UART_RxHalfCpltCallback
    stm32f1xx_hal_uart.o(i.UART_DMARxHalfCplt) refers to stm32f1xx_hal_uart.o(i.HAL_UARTEx_RxEventCallback) for HAL_UARTEx_RxEventCallback
    stm32f1xx_hal_uart.o(i.UART_DMARxOnlyAbortCallback) refers to uart.o(i.HAL_UART_AbortReceiveCpltCallback) for HAL_UART_AbortReceiveCpltCallback
    stm32f1xx_hal_uart.o(i.UART_DMATransmitCplt) refers to uart.o(i.HAL_UART_TxCpltCallback) for HAL_UART_TxCpltCallback
    stm32f1xx_hal_uart.o(i.UART_DMATxAbortCallback) refers to uart.o(i.HAL_UART_AbortCpltCallback) for HAL_UART_AbortCpltCallback
    stm32f1xx_hal_uart.o(i.UART_DMATxHalfCplt) refers to uart.o(i.HAL_UART_TxHalfCpltCallback) for HAL_UART_TxHalfCpltCallback
    stm32f1xx_hal_uart.o(i.UART_DMATxOnlyAbortCallback) refers to uart.o(i.HAL_UART_AbortTransmitCpltCallback) for HAL_UART_AbortTransmitCpltCallback
    stm32f1xx_hal_uart.o(i.UART_Receive_IT) refers to uart.o(i.HAL_UART_RxCpltCallback) for HAL_UART_RxCpltCallback
    stm32f1xx_hal_uart.o(i.UART_Receive_IT) refers to stm32f1xx_hal_uart.o(i.HAL_UARTEx_RxEventCallback) for HAL_UARTEx_RxEventCallback
    stm32f1xx_hal_uart.o(i.UART_SetConfig) refers to stm32f1xx_hal_rcc.o(i.HAL_RCC_GetPCLK2Freq) for HAL_RCC_GetPCLK2Freq
    stm32f1xx_hal_uart.o(i.UART_SetConfig) refers to stm32f1xx_hal_rcc.o(i.HAL_RCC_GetPCLK1Freq) for HAL_RCC_GetPCLK1Freq
    stm32f1xx_hal_uart.o(i.UART_Start_Receive_DMA) refers to stm32f1xx_hal_dma.o(i.HAL_DMA_Start_IT) for HAL_DMA_Start_IT
    stm32f1xx_hal_uart.o(i.UART_Start_Receive_DMA) refers to stm32f1xx_hal_uart.o(i.UART_DMAReceiveCplt) for UART_DMAReceiveCplt
    stm32f1xx_hal_uart.o(i.UART_Start_Receive_DMA) refers to stm32f1xx_hal_uart.o(i.UART_DMARxHalfCplt) for UART_DMARxHalfCplt
    stm32f1xx_hal_uart.o(i.UART_Start_Receive_DMA) refers to stm32f1xx_hal_uart.o(i.UART_DMAError) for UART_DMAError
    stm32f1xx_hal_uart.o(i.UART_WaitOnFlagUntilTimeout) refers to stm32f1xx_hal.o(i.HAL_GetTick) for HAL_GetTick
    stm32f1xx_hal_uart.o(i.UART_WaitOnFlagUntilTimeout) refers to stm32f1xx_hal_uart.o(i.UART_EndRxTransfer) for UART_EndRxTransfer
    system_stm32f1xx.o(i.SystemCoreClockUpdate) refers to system_stm32f1xx.o(.data) for .data
    system_stm32f1xx.o(i.SystemCoreClockUpdate) refers to system_stm32f1xx.o(.constdata) for .constdata
    sx1281.o(i.OnCadDone) refers to sx1281.o(i.SX1281_Callback) for SX1281_Callback
    sx1281.o(i.OnCadDone) refers to sx1281.o(.data) for .data
    sx1281.o(i.OnRxDone) refers to sx1281.o(i.SX1281_Callback) for SX1281_Callback
    sx1281.o(i.OnRxDone) refers to sx1281.o(.data) for .data
    sx1281.o(i.OnRxError) refers to sx1281.o(i.SX1281_Callback) for SX1281_Callback
    sx1281.o(i.OnRxError) refers to sx1281.o(.data) for .data
    sx1281.o(i.OnRxTimeout) refers to sx1281.o(i.SX1281_Callback) for SX1281_Callback
    sx1281.o(i.OnRxTimeout) refers to sx1281.o(.data) for .data
    sx1281.o(i.OnTxDone) refers to sx1281.o(i.SX1281_Callback) for SX1281_Callback
    sx1281.o(i.OnTxDone) refers to sx1281.o(.data) for .data
    sx1281.o(i.OnTxTimeout) refers to sx1281.o(i.SX1281_Callback) for SX1281_Callback
    sx1281.o(i.OnTxTimeout) refers to sx1281.o(.data) for .data
    sx1281.o(i.SX1281_Callback) refers to printfa.o(i.__0printf) for __2printf
    sx1281.o(i.SX1281_Callback) refers to sx1281.o(.data) for .data
    sx1281.o(i.SX1281_Callback) refers to sx1281_driver_hal.o(.constdata) for Radio
    sx1281.o(i.SX1281_Callback) refers to sx1281.o(.constdata) for .constdata
    sx1281.o(i.SX1281_Callback) refers to sx1281.o(.bss) for .bss
    sx1281.o(i.SX1281_GetState) refers to sx1281.o(.data) for .data
    sx1281.o(i.SX1281_Init) refers to sx1281_header.o(i.SX1281_BSPInit) for SX1281_BSPInit
    sx1281.o(i.SX1281_Init) refers to stm32f1xx_hal.o(i.HAL_Delay) for HAL_Delay
    sx1281.o(i.SX1281_Init) refers to printfa.o(i.__0printf) for __2printf
    sx1281.o(i.SX1281_Init) refers to sx1281_driver_hal.o(.constdata) for Radio
    sx1281.o(i.SX1281_Init) refers to sx1281.o(.data) for .data
    sx1281.o(i.SX1281_Init) refers to sx1281.o(.constdata) for .constdata
    sx1281.o(i.SX1281_Running) refers to sx1281_driver.o(i.SX1281ProcessIrqs) for SX1281ProcessIrqs
    sx1281.o(i.SX1281_Running) refers to sx1281.o(i.SX1281_GetState) for SX1281_GetState
    sx1281.o(i.SX1281_Running) refers to stm32f1xx_hal.o(i.HAL_Delay) for HAL_Delay
    sx1281.o(i.SX1281_SetBLEBaudrate) refers to sx1281_driver_hal.o(.constdata) for Radio
    sx1281.o(i.SX1281_SetBLEBaudrate) refers to sx1281.o(.constdata) for .constdata
    sx1281.o(i.SX1281_SetFLRCBaudrate) refers to sx1281_driver_hal.o(.constdata) for Radio
    sx1281.o(i.SX1281_SetFLRCBaudrate) refers to sx1281.o(.constdata) for .constdata
    sx1281.o(i.SX1281_SetGFSKBaudrate) refers to sx1281_driver_hal.o(.constdata) for Radio
    sx1281.o(i.SX1281_SetGFSKBaudrate) refers to sx1281.o(.constdata) for .constdata
    sx1281.o(i.SX1281_SetLORABaudrate) refers to sx1281_driver_hal.o(.constdata) for Radio
    sx1281.o(i.SX1281_SetLORABaudrate) refers to sx1281.o(.constdata) for .constdata
    sx1281.o(i.SX1281_SetMode) refers to sx1281_driver_hal.o(.constdata) for Radio
    sx1281.o(i.SX1281_SetPacketConfig) refers to sx1281_driver_hal.o(.constdata) for Radio
    sx1281.o(i.SX1281_SetRFFrequency) refers to sx1281_driver_hal.o(.constdata) for Radio
    sx1281.o(i.SX1281_SetRXSingle) refers to sx1281_driver_hal.o(.constdata) for Radio
    sx1281.o(i.SX1281_SetRXSingle) refers to sx1281.o(.data) for .data
    sx1281.o(i.SX1281_SetRXSingle) refers to sx1281.o(.constdata) for .constdata
    sx1281.o(i.SX1281_SetRXSuccessive) refers to sx1281_driver_hal.o(.constdata) for Radio
    sx1281.o(i.SX1281_SetRXSuccessive) refers to sx1281.o(.data) for .data
    sx1281.o(i.SX1281_SetRXSuccessive) refers to sx1281.o(.constdata) for .constdata
    sx1281.o(i.SX1281_SetTX) refers to sx1281_driver_hal.o(.constdata) for Radio
    sx1281.o(i.SX1281_SetTX) refers to sx1281.o(.data) for .data
    sx1281.o(i.SX1281_SetTX) refers to sx1281.o(.constdata) for .constdata
    sx1281.o(.data) refers to sx1281.o(i.OnTxDone) for OnTxDone
    sx1281.o(.data) refers to sx1281.o(i.OnRxDone) for OnRxDone
    sx1281.o(.data) refers to sx1281.o(i.OnTxTimeout) for OnTxTimeout
    sx1281.o(.data) refers to sx1281.o(i.OnRxTimeout) for OnRxTimeout
    sx1281.o(.data) refers to sx1281.o(i.OnRxError) for OnRxError
    sx1281_driver.o(i.SX1281Calibrate) refers to sx1281_driver_hal.o(i.SX1281HalWriteCommand) for SX1281HalWriteCommand
    sx1281_driver.o(i.SX1281ClearIrqStatus) refers to sx1281_driver_hal.o(i.SX1281HalWriteCommand) for SX1281HalWriteCommand
    sx1281_driver.o(i.SX1281GetFirmwareVersion) refers to sx1281_driver_hal.o(i.SX1281HalReadRegister) for SX1281HalReadRegister
    sx1281_driver.o(i.SX1281GetFrequencyError) refers to sx1281_driver_hal.o(i.SX1281HalReadRegister) for SX1281HalReadRegister
    sx1281_driver.o(i.SX1281GetFrequencyError) refers to sx1281_driver.o(i.SX1281GetLoRaBandwidth) for SX1281GetLoRaBandwidth
    sx1281_driver.o(i.SX1281GetFrequencyError) refers to dflti.o(.text) for __aeabi_i2d
    sx1281_driver.o(i.SX1281GetFrequencyError) refers to ddiv.o(.text) for __aeabi_ddiv
    sx1281_driver.o(i.SX1281GetFrequencyError) refers to dmul.o(.text) for __aeabi_dmul
    sx1281_driver.o(i.SX1281GetFrequencyError) refers to sx1281_driver.o(.data) for .data
    sx1281_driver.o(i.SX1281GetHexFileLineFields) refers to _scanf_int.o(.text) for _scanf_int
    sx1281_driver.o(i.SX1281GetHexFileLineFields) refers to strlen.o(.text) for strlen
    sx1281_driver.o(i.SX1281GetHexFileLineFields) refers to __0sscanf.o(.text) for __0sscanf
    sx1281_driver.o(i.SX1281GetIrqStatus) refers to sx1281_driver_hal.o(i.SX1281HalReadCommand) for SX1281HalReadCommand
    sx1281_driver.o(i.SX1281GetLoRaBandwidth) refers to sx1281_driver.o(.data) for .data
    sx1281_driver.o(i.SX1281GetOpMode) refers to sx1281_driver.o(.data) for .data
    sx1281_driver.o(i.SX1281GetPacketStatus) refers to sx1281_driver_hal.o(i.SX1281HalReadCommand) for SX1281HalReadCommand
    sx1281_driver.o(i.SX1281GetPacketStatus) refers to sx1281_driver.o(.data) for .data
    sx1281_driver.o(i.SX1281GetPacketType) refers to sx1281_driver.o(.data) for .data
    sx1281_driver.o(i.SX1281GetPayload) refers to sx1281_driver.o(i.SX1281GetRxBufferStatus) for SX1281GetRxBufferStatus
    sx1281_driver.o(i.SX1281GetPayload) refers to sx1281_driver_hal.o(i.SX1281HalReadBuffer) for SX1281HalReadBuffer
    sx1281_driver.o(i.SX1281GetRssiInst) refers to sx1281_driver_hal.o(i.SX1281HalReadCommand) for SX1281HalReadCommand
    sx1281_driver.o(i.SX1281GetRxBufferStatus) refers to sx1281_driver_hal.o(i.SX1281HalReadCommand) for SX1281HalReadCommand
    sx1281_driver.o(i.SX1281GetRxBufferStatus) refers to sx1281_driver_hal.o(i.SX1281HalReadRegister) for SX1281HalReadRegister
    sx1281_driver.o(i.SX1281GetRxBufferStatus) refers to sx1281_driver.o(.data) for .data
    sx1281_driver.o(i.SX1281GetStatus) refers to sx1281_driver_hal.o(i.SX1281HalReadCommand) for SX1281HalReadCommand
    sx1281_driver.o(i.SX1281Init) refers to sx1281_driver_hal.o(i.SX1281HalInit) for SX1281HalInit
    sx1281_driver.o(i.SX1281Init) refers to sx1281_driver.o(.data) for .data
    sx1281_driver.o(i.SX1281OnDioIrq) refers to sx1281_driver.o(i.SX1281ProcessIrqs) for SX1281ProcessIrqs
    sx1281_driver.o(i.SX1281OnDioIrq) refers to sx1281_driver.o(.data) for .data
    sx1281_driver.o(i.SX1281ParseHexFileLine) refers to sx1281_driver.o(i.SX1281GetHexFileLineFields) for SX1281GetHexFileLineFields
    sx1281_driver.o(i.SX1281ParseHexFileLine) refers to sx1281_driver_hal.o(i.SX1281HalWriteRegisters) for SX1281HalWriteRegisters
    sx1281_driver.o(i.SX1281ProcessIrqs) refers to sx1281_driver.o(i.SX1281GetIrqStatus) for SX1281GetIrqStatus
    sx1281_driver.o(i.SX1281ProcessIrqs) refers to sx1281_driver.o(i.SX1281ClearIrqStatus) for SX1281ClearIrqStatus
    sx1281_driver.o(i.SX1281ProcessIrqs) refers to sx1281_driver.o(.data) for .data
    sx1281_driver.o(i.SX1281SendPayload) refers to sx1281_driver.o(i.SX1281SetPayload) for SX1281SetPayload
    sx1281_driver.o(i.SX1281SendPayload) refers to sx1281_driver.o(i.SX1281SetTx) for SX1281SetTx
    sx1281_driver.o(i.SX1281SetAutoFS) refers to sx1281_driver_hal.o(i.SX1281HalWriteCommand) for SX1281HalWriteCommand
    sx1281_driver.o(i.SX1281SetAutoTx) refers to sx1281_driver_hal.o(i.SX1281HalWriteCommand) for SX1281HalWriteCommand
    sx1281_driver.o(i.SX1281SetBleAccessAddress) refers to sx1281_driver_hal.o(i.SX1281HalWriteRegister) for SX1281HalWriteRegister
    sx1281_driver.o(i.SX1281SetBleAdvertizerAccessAddress) refers to sx1281_driver.o(i.SX1281SetBleAccessAddress) for SX1281SetBleAccessAddress
    sx1281_driver.o(i.SX1281SetBufferBaseAddresses) refers to sx1281_driver_hal.o(i.SX1281HalWriteCommand) for SX1281HalWriteCommand
    sx1281_driver.o(i.SX1281SetCad) refers to sx1281_driver_hal.o(i.SX1281HalWriteCommand) for SX1281HalWriteCommand
    sx1281_driver.o(i.SX1281SetCad) refers to sx1281_driver.o(.data) for .data
    sx1281_driver.o(i.SX1281SetCadParams) refers to sx1281_driver_hal.o(i.SX1281HalWriteCommand) for SX1281HalWriteCommand
    sx1281_driver.o(i.SX1281SetCadParams) refers to sx1281_driver.o(.data) for .data
    sx1281_driver.o(i.SX1281SetCrcPolynomial) refers to sx1281_driver_hal.o(i.SX1281HalWriteRegisters) for SX1281HalWriteRegisters
    sx1281_driver.o(i.SX1281SetCrcPolynomial) refers to sx1281_driver.o(.data) for .data
    sx1281_driver.o(i.SX1281SetCrcSeed) refers to sx1281_driver_hal.o(i.SX1281HalWriteRegisters) for SX1281HalWriteRegisters
    sx1281_driver.o(i.SX1281SetCrcSeed) refers to sx1281_driver.o(.data) for .data
    sx1281_driver.o(i.SX1281SetDioIrqParams) refers to sx1281_driver_hal.o(i.SX1281HalWriteCommand) for SX1281HalWriteCommand
    sx1281_driver.o(i.SX1281SetFs) refers to sx1281_driver_hal.o(i.SX1281HalWriteCommand) for SX1281HalWriteCommand
    sx1281_driver.o(i.SX1281SetFs) refers to sx1281_driver.o(.data) for .data
    sx1281_driver.o(i.SX1281SetInterruptMode) refers to sx1281_driver.o(.data) for .data
    sx1281_driver.o(i.SX1281SetLongPreamble) refers to sx1281_driver_hal.o(i.SX1281HalWriteCommand) for SX1281HalWriteCommand
    sx1281_driver.o(i.SX1281SetModulationParams) refers to sx1281_driver.o(i.SX1281SetPacketType) for SX1281SetPacketType
    sx1281_driver.o(i.SX1281SetModulationParams) refers to sx1281_driver_hal.o(i.SX1281HalWriteCommand) for SX1281HalWriteCommand
    sx1281_driver.o(i.SX1281SetModulationParams) refers to sx1281_driver.o(.data) for .data
    sx1281_driver.o(i.SX1281SetPacketParams) refers to sx1281_driver.o(i.SX1281SetPacketType) for SX1281SetPacketType
    sx1281_driver.o(i.SX1281SetPacketParams) refers to sx1281_driver_hal.o(i.SX1281HalWriteCommand) for SX1281HalWriteCommand
    sx1281_driver.o(i.SX1281SetPacketParams) refers to sx1281_driver.o(.data) for .data
    sx1281_driver.o(i.SX1281SetPacketType) refers to sx1281_driver_hal.o(i.SX1281HalWriteCommand) for SX1281HalWriteCommand
    sx1281_driver.o(i.SX1281SetPacketType) refers to sx1281_driver.o(.data) for .data
    sx1281_driver.o(i.SX1281SetPayload) refers to sx1281_driver_hal.o(i.SX1281HalWriteBuffer) for SX1281HalWriteBuffer
    sx1281_driver.o(i.SX1281SetPollingMode) refers to sx1281_driver.o(.data) for .data
    sx1281_driver.o(i.SX1281SetRegistersDefault) refers to sx1281_driver_hal.o(i.SX1281HalWriteRegister) for SX1281HalWriteRegister
    sx1281_driver.o(i.SX1281SetRegistersDefault) refers to sx1281_driver.o(.constdata) for .constdata
    sx1281_driver.o(i.SX1281SetRegulatorMode) refers to sx1281_driver_hal.o(i.SX1281HalWriteCommand) for SX1281HalWriteCommand
    sx1281_driver.o(i.SX1281SetRfFrequency) refers to dfltui.o(.text) for __aeabi_ui2d
    sx1281_driver.o(i.SX1281SetRfFrequency) refers to ddiv.o(.text) for __aeabi_ddiv
    sx1281_driver.o(i.SX1281SetRfFrequency) refers to dfixui.o(.text) for __aeabi_d2uiz
    sx1281_driver.o(i.SX1281SetRfFrequency) refers to sx1281_driver_hal.o(i.SX1281HalWriteCommand) for SX1281HalWriteCommand
    sx1281_driver.o(i.SX1281SetRx) refers to sx1281_driver.o(i.SX1281ClearIrqStatus) for SX1281ClearIrqStatus
    sx1281_driver.o(i.SX1281SetRx) refers to sx1281_driver_hal.o(i.SX1281HalWriteCommand) for SX1281HalWriteCommand
    sx1281_driver.o(i.SX1281SetRx) refers to sx1281_driver.o(.data) for .data
    sx1281_driver.o(i.SX1281SetRxDutyCycle) refers to sx1281_driver_hal.o(i.SX1281HalWriteCommand) for SX1281HalWriteCommand
    sx1281_driver.o(i.SX1281SetRxDutyCycle) refers to sx1281_driver.o(.data) for .data
    sx1281_driver.o(i.SX1281SetSaveContext) refers to sx1281_driver_hal.o(i.SX1281HalWriteCommand) for SX1281HalWriteCommand
    sx1281_driver.o(i.SX1281SetSleep) refers to sx1281_driver_hal.o(i.SX1281HalWriteCommand) for SX1281HalWriteCommand
    sx1281_driver.o(i.SX1281SetSleep) refers to sx1281_driver.o(.data) for .data
    sx1281_driver.o(i.SX1281SetStandby) refers to sx1281_driver_hal.o(i.SX1281HalWriteCommand) for SX1281HalWriteCommand
    sx1281_driver.o(i.SX1281SetStandby) refers to sx1281_driver.o(.data) for .data
    sx1281_driver.o(i.SX1281SetSyncWord) refers to sx1281_driver_hal.o(i.SX1281HalWriteRegisters) for SX1281HalWriteRegisters
    sx1281_driver.o(i.SX1281SetSyncWord) refers to sx1281_driver.o(.data) for .data
    sx1281_driver.o(i.SX1281SetSyncWordErrorTolerance) refers to sx1281_driver_hal.o(i.SX1281HalReadRegister) for SX1281HalReadRegister
    sx1281_driver.o(i.SX1281SetSyncWordErrorTolerance) refers to sx1281_driver_hal.o(i.SX1281HalWriteRegister) for SX1281HalWriteRegister
    sx1281_driver.o(i.SX1281SetTx) refers to sx1281_driver.o(i.SX1281ClearIrqStatus) for SX1281ClearIrqStatus
    sx1281_driver.o(i.SX1281SetTx) refers to sx1281_driver_hal.o(i.SX1281HalWriteCommand) for SX1281HalWriteCommand
    sx1281_driver.o(i.SX1281SetTx) refers to sx1281_driver.o(.data) for .data
    sx1281_driver.o(i.SX1281SetTxContinuousPreamble) refers to sx1281_driver_hal.o(i.SX1281HalWriteCommand) for SX1281HalWriteCommand
    sx1281_driver.o(i.SX1281SetTxContinuousWave) refers to sx1281_driver_hal.o(i.SX1281HalWriteCommand) for SX1281HalWriteCommand
    sx1281_driver.o(i.SX1281SetTxParams) refers to sx1281_driver_hal.o(i.SX1281HalWriteCommand) for SX1281HalWriteCommand
    sx1281_driver.o(i.SX1281SetWhiteningSeed) refers to sx1281_driver_hal.o(i.SX1281HalWriteRegister) for SX1281HalWriteRegister
    sx1281_driver.o(i.SX1281SetWhiteningSeed) refers to sx1281_driver.o(.data) for .data
    sx1281_driver.o(.data) refers to sx1281_driver.o(i.SX1281OnDioIrq) for SX1281OnDioIrq
    sx1281_driver_gpio.o(i.GpioLaunchIrqHandler) refers to sx1281_driver_gpio.o(i.GpioGetBitPos) for GpioGetBitPos
    sx1281_driver_gpio.o(i.GpioLaunchIrqHandler) refers to sx1281_driver_gpio.o(.bss) for .bss
    sx1281_driver_gpio.o(i.GpioRead) refers to stm32f1xx_hal_gpio.o(i.HAL_GPIO_ReadPin) for HAL_GPIO_ReadPin
    sx1281_driver_gpio.o(i.GpioSetIrq) refers to sx1281_driver_gpio.o(i.GpioGetBitPos) for GpioGetBitPos
    sx1281_driver_gpio.o(i.GpioSetIrq) refers to sx1281_driver_gpio.o(i.MSP_GetIRQn) for MSP_GetIRQn
    sx1281_driver_gpio.o(i.GpioSetIrq) refers to stm32f1xx_hal_cortex.o(i.HAL_NVIC_SetPriority) for HAL_NVIC_SetPriority
    sx1281_driver_gpio.o(i.GpioSetIrq) refers to stm32f1xx_hal_cortex.o(i.HAL_NVIC_EnableIRQ) for HAL_NVIC_EnableIRQ
    sx1281_driver_gpio.o(i.GpioSetIrq) refers to sx1281_driver_gpio.o(.bss) for .bss
    sx1281_driver_gpio.o(i.GpioWrite) refers to stm32f1xx_hal_gpio.o(i.HAL_GPIO_WritePin) for HAL_GPIO_WritePin
    sx1281_driver_gpio.o(i.MSP_GetIRQn) refers to sx1281_driver_gpio.o(i.GpioGetBitPos) for GpioGetBitPos
    sx1281_driver_hal.o(i.SX120HalWakeup) refers to sx1281_driver_gpio.o(i.GpioWrite) for GpioWrite
    sx1281_driver_hal.o(i.SX120HalWakeup) refers to sx1281_driver_spi.o(i.SpiIn) for SpiIn
    sx1281_driver_hal.o(i.SX120HalWakeup) refers to sx1281_driver_hal.o(i.SX1281HalWaitOnBusy) for SX1281HalWaitOnBusy
    sx1281_driver_hal.o(i.SX120HalWakeup) refers to sx1281_driver_hal.o(.bss) for .bss
    sx1281_driver_hal.o(i.SX1281HalClearInstructionRam) refers to sx1281_driver_hal.o(i.SX1281HalWaitOnBusy) for SX1281HalWaitOnBusy
    sx1281_driver_hal.o(i.SX1281HalClearInstructionRam) refers to sx1281_driver_gpio.o(i.GpioWrite) for GpioWrite
    sx1281_driver_hal.o(i.SX1281HalClearInstructionRam) refers to sx1281_driver_spi.o(i.SpiIn) for SpiIn
    sx1281_driver_hal.o(i.SX1281HalClearInstructionRam) refers to sx1281_driver_hal.o(.bss) for .bss
    sx1281_driver_hal.o(i.SX1281HalGetDioStatus) refers to sx1281_driver_gpio.o(i.GpioRead) for GpioRead
    sx1281_driver_hal.o(i.SX1281HalInit) refers to sx1281_driver_hal.o(i.SX1281HalReset) for SX1281HalReset
    sx1281_driver_hal.o(i.SX1281HalInit) refers to sx1281_driver_hal.o(i.SX1281HalIoIrqInit) for SX1281HalIoIrqInit
    sx1281_driver_hal.o(i.SX1281HalIoIrqInit) refers to sx1281_driver_gpio.o(i.GpioSetIrq) for GpioSetIrq
    sx1281_driver_hal.o(i.SX1281HalReadBuffer) refers to sx1281_driver_hal.o(i.SX1281HalWaitOnBusy) for SX1281HalWaitOnBusy
    sx1281_driver_hal.o(i.SX1281HalReadBuffer) refers to sx1281_driver_gpio.o(i.GpioWrite) for GpioWrite
    sx1281_driver_hal.o(i.SX1281HalReadBuffer) refers to sx1281_driver_spi.o(i.SpiInOut) for SpiInOut
    sx1281_driver_hal.o(i.SX1281HalReadBuffer) refers to memcpya.o(.text) for __aeabi_memcpy
    sx1281_driver_hal.o(i.SX1281HalReadBuffer) refers to sx1281_driver_hal.o(.bss) for .bss
    sx1281_driver_hal.o(i.SX1281HalReadCommand) refers to sx1281_driver_hal.o(i.SX1281HalWaitOnBusy) for SX1281HalWaitOnBusy
    sx1281_driver_hal.o(i.SX1281HalReadCommand) refers to sx1281_driver_gpio.o(i.GpioWrite) for GpioWrite
    sx1281_driver_hal.o(i.SX1281HalReadCommand) refers to sx1281_driver_spi.o(i.SpiInOut) for SpiInOut
    sx1281_driver_hal.o(i.SX1281HalReadCommand) refers to memcpya.o(.text) for __aeabi_memcpy
    sx1281_driver_hal.o(i.SX1281HalReadCommand) refers to sx1281_driver_hal.o(.bss) for .bss
    sx1281_driver_hal.o(i.SX1281HalReadRegister) refers to sx1281_driver_hal.o(i.SX1281HalReadRegisters) for SX1281HalReadRegisters
    sx1281_driver_hal.o(i.SX1281HalReadRegisters) refers to sx1281_driver_hal.o(i.SX1281HalWaitOnBusy) for SX1281HalWaitOnBusy
    sx1281_driver_hal.o(i.SX1281HalReadRegisters) refers to sx1281_driver_gpio.o(i.GpioWrite) for GpioWrite
    sx1281_driver_hal.o(i.SX1281HalReadRegisters) refers to sx1281_driver_spi.o(i.SpiInOut) for SpiInOut
    sx1281_driver_hal.o(i.SX1281HalReadRegisters) refers to memcpya.o(.text) for __aeabi_memcpy
    sx1281_driver_hal.o(i.SX1281HalReadRegisters) refers to sx1281_driver_hal.o(.bss) for .bss
    sx1281_driver_hal.o(i.SX1281HalReset) refers to stm32f1xx_hal.o(i.HAL_Delay) for HAL_Delay
    sx1281_driver_hal.o(i.SX1281HalReset) refers to sx1281_driver_gpio.o(i.GpioWrite) for GpioWrite
    sx1281_driver_hal.o(i.SX1281HalWaitOnBusy) refers to stm32f1xx_hal_gpio.o(i.HAL_GPIO_ReadPin) for HAL_GPIO_ReadPin
    sx1281_driver_hal.o(i.SX1281HalWriteBuffer) refers to memcpya.o(.text) for __aeabi_memcpy
    sx1281_driver_hal.o(i.SX1281HalWriteBuffer) refers to sx1281_driver_hal.o(i.SX1281HalWaitOnBusy) for SX1281HalWaitOnBusy
    sx1281_driver_hal.o(i.SX1281HalWriteBuffer) refers to sx1281_driver_gpio.o(i.GpioWrite) for GpioWrite
    sx1281_driver_hal.o(i.SX1281HalWriteBuffer) refers to sx1281_driver_spi.o(i.SpiIn) for SpiIn
    sx1281_driver_hal.o(i.SX1281HalWriteBuffer) refers to sx1281_driver_hal.o(.bss) for .bss
    sx1281_driver_hal.o(i.SX1281HalWriteCommand) refers to sx1281_driver_hal.o(i.SX1281HalWaitOnBusy) for SX1281HalWaitOnBusy
    sx1281_driver_hal.o(i.SX1281HalWriteCommand) refers to sx1281_driver_gpio.o(i.GpioWrite) for GpioWrite
    sx1281_driver_hal.o(i.SX1281HalWriteCommand) refers to memcpya.o(.text) for __aeabi_memcpy
    sx1281_driver_hal.o(i.SX1281HalWriteCommand) refers to sx1281_driver_spi.o(i.SpiIn) for SpiIn
    sx1281_driver_hal.o(i.SX1281HalWriteCommand) refers to sx1281_driver_hal.o(.bss) for .bss
    sx1281_driver_hal.o(i.SX1281HalWriteRegister) refers to sx1281_driver_hal.o(i.SX1281HalWriteRegisters) for SX1281HalWriteRegisters
    sx1281_driver_hal.o(i.SX1281HalWriteRegisters) refers to memcpya.o(.text) for __aeabi_memcpy
    sx1281_driver_hal.o(i.SX1281HalWriteRegisters) refers to sx1281_driver_hal.o(i.SX1281HalWaitOnBusy) for SX1281HalWaitOnBusy
    sx1281_driver_hal.o(i.SX1281HalWriteRegisters) refers to sx1281_driver_gpio.o(i.GpioWrite) for GpioWrite
    sx1281_driver_hal.o(i.SX1281HalWriteRegisters) refers to sx1281_driver_spi.o(i.SpiIn) for SpiIn
    sx1281_driver_hal.o(i.SX1281HalWriteRegisters) refers to sx1281_driver_hal.o(.bss) for .bss
    sx1281_driver_hal.o(.constdata) refers to sx1281_driver.o(i.SX1281Init) for SX1281Init
    sx1281_driver_hal.o(.constdata) refers to sx1281_driver_hal.o(i.SX1281HalReset) for SX1281HalReset
    sx1281_driver_hal.o(.constdata) refers to sx1281_driver.o(i.SX1281GetStatus) for SX1281GetStatus
    sx1281_driver_hal.o(.constdata) refers to sx1281_driver_hal.o(i.SX1281HalWriteCommand) for SX1281HalWriteCommand
    sx1281_driver_hal.o(.constdata) refers to sx1281_driver_hal.o(i.SX1281HalReadCommand) for SX1281HalReadCommand
    sx1281_driver_hal.o(.constdata) refers to sx1281_driver_hal.o(i.SX1281HalWriteRegisters) for SX1281HalWriteRegisters
    sx1281_driver_hal.o(.constdata) refers to sx1281_driver_hal.o(i.SX1281HalWriteRegister) for SX1281HalWriteRegister
    sx1281_driver_hal.o(.constdata) refers to sx1281_driver_hal.o(i.SX1281HalReadRegisters) for SX1281HalReadRegisters
    sx1281_driver_hal.o(.constdata) refers to sx1281_driver_hal.o(i.SX1281HalReadRegister) for SX1281HalReadRegister
    sx1281_driver_hal.o(.constdata) refers to sx1281_driver_hal.o(i.SX1281HalWriteBuffer) for SX1281HalWriteBuffer
    sx1281_driver_hal.o(.constdata) refers to sx1281_driver_hal.o(i.SX1281HalReadBuffer) for SX1281HalReadBuffer
    sx1281_driver_hal.o(.constdata) refers to sx1281_driver_hal.o(i.SX1281HalGetDioStatus) for SX1281HalGetDioStatus
    sx1281_driver_hal.o(.constdata) refers to sx1281_driver.o(i.SX1281GetFirmwareVersion) for SX1281GetFirmwareVersion
    sx1281_driver_hal.o(.constdata) refers to sx1281_driver.o(i.SX1281SetRegulatorMode) for SX1281SetRegulatorMode
    sx1281_driver_hal.o(.constdata) refers to sx1281_driver.o(i.SX1281SetStandby) for SX1281SetStandby
    sx1281_driver_hal.o(.constdata) refers to sx1281_driver.o(i.SX1281SetPacketType) for SX1281SetPacketType
    sx1281_driver_hal.o(.constdata) refers to sx1281_driver.o(i.SX1281SetModulationParams) for SX1281SetModulationParams
    sx1281_driver_hal.o(.constdata) refers to sx1281_driver.o(i.SX1281SetPacketParams) for SX1281SetPacketParams
    sx1281_driver_hal.o(.constdata) refers to sx1281_driver.o(i.SX1281SetRfFrequency) for SX1281SetRfFrequency
    sx1281_driver_hal.o(.constdata) refers to sx1281_driver.o(i.SX1281SetBufferBaseAddresses) for SX1281SetBufferBaseAddresses
    sx1281_driver_hal.o(.constdata) refers to sx1281_driver.o(i.SX1281SetTxParams) for SX1281SetTxParams
    sx1281_driver_hal.o(.constdata) refers to sx1281_driver.o(i.SX1281SetDioIrqParams) for SX1281SetDioIrqParams
    sx1281_driver_hal.o(.constdata) refers to sx1281_driver.o(i.SX1281SetSyncWord) for SX1281SetSyncWord
    sx1281_driver_hal.o(.constdata) refers to sx1281_driver.o(i.SX1281SetRx) for SX1281SetRx
    sx1281_driver_hal.o(.constdata) refers to sx1281_driver.o(i.SX1281GetPayload) for SX1281GetPayload
    sx1281_driver_hal.o(.constdata) refers to sx1281_driver.o(i.SX1281SendPayload) for SX1281SendPayload
    sx1281_driver_hal.o(.constdata) refers to sx1281_driver.o(i.SX1281SetPollingMode) for SX1281SetPollingMode
    sx1281_driver_hal.o(.constdata) refers to sx1281_driver.o(i.SX1281SetInterruptMode) for SX1281SetInterruptMode
    sx1281_driver_hal.o(.constdata) refers to sx1281_driver.o(i.SX1281SetRegistersDefault) for SX1281SetRegistersDefault
    sx1281_driver_hal.o(.constdata) refers to sx1281_driver.o(i.SX1281GetOpMode) for SX1281GetOpMode
    sx1281_driver_hal.o(.constdata) refers to sx1281_driver.o(i.SX1281SetSleep) for SX1281SetSleep
    sx1281_driver_hal.o(.constdata) refers to sx1281_driver.o(i.SX1281SetFs) for SX1281SetFs
    sx1281_driver_hal.o(.constdata) refers to sx1281_driver.o(i.SX1281SetTx) for SX1281SetTx
    sx1281_driver_hal.o(.constdata) refers to sx1281_driver.o(i.SX1281SetRxDutyCycle) for SX1281SetRxDutyCycle
    sx1281_driver_hal.o(.constdata) refers to sx1281_driver.o(i.SX1281SetCad) for SX1281SetCad
    sx1281_driver_hal.o(.constdata) refers to sx1281_driver.o(i.SX1281SetTxContinuousWave) for SX1281SetTxContinuousWave
    sx1281_driver_hal.o(.constdata) refers to sx1281_driver.o(i.SX1281SetTxContinuousPreamble) for SX1281SetTxContinuousPreamble
    sx1281_driver_hal.o(.constdata) refers to sx1281_driver.o(i.SX1281GetPacketType) for SX1281GetPacketType
    sx1281_driver_hal.o(.constdata) refers to sx1281_driver.o(i.SX1281SetCadParams) for SX1281SetCadParams
    sx1281_driver_hal.o(.constdata) refers to sx1281_driver.o(i.SX1281GetRxBufferStatus) for SX1281GetRxBufferStatus
    sx1281_driver_hal.o(.constdata) refers to sx1281_driver.o(i.SX1281GetPacketStatus) for SX1281GetPacketStatus
    sx1281_driver_hal.o(.constdata) refers to sx1281_driver.o(i.SX1281GetRssiInst) for SX1281GetRssiInst
    sx1281_driver_hal.o(.constdata) refers to sx1281_driver.o(i.SX1281GetIrqStatus) for SX1281GetIrqStatus
    sx1281_driver_hal.o(.constdata) refers to sx1281_driver.o(i.SX1281ClearIrqStatus) for SX1281ClearIrqStatus
    sx1281_driver_hal.o(.constdata) refers to sx1281_driver.o(i.SX1281Calibrate) for SX1281Calibrate
    sx1281_driver_hal.o(.constdata) refers to sx1281_driver.o(i.SX1281SetSaveContext) for SX1281SetSaveContext
    sx1281_driver_hal.o(.constdata) refers to sx1281_driver.o(i.SX1281SetAutoTx) for SX1281SetAutoTx
    sx1281_driver_hal.o(.constdata) refers to sx1281_driver.o(i.SX1281SetAutoFS) for SX1281SetAutoFS
    sx1281_driver_hal.o(.constdata) refers to sx1281_driver.o(i.SX1281SetLongPreamble) for SX1281SetLongPreamble
    sx1281_driver_hal.o(.constdata) refers to sx1281_driver.o(i.SX1281SetPayload) for SX1281SetPayload
    sx1281_driver_hal.o(.constdata) refers to sx1281_driver.o(i.SX1281SetSyncWordErrorTolerance) for SX1281SetSyncWordErrorTolerance
    sx1281_driver_hal.o(.constdata) refers to sx1281_driver.o(i.SX1281SetCrcSeed) for SX1281SetCrcSeed
    sx1281_driver_hal.o(.constdata) refers to sx1281_driver.o(i.SX1281SetBleAccessAddress) for SX1281SetBleAccessAddress
    sx1281_driver_hal.o(.constdata) refers to sx1281_driver.o(i.SX1281SetBleAdvertizerAccessAddress) for SX1281SetBleAdvertizerAccessAddress
    sx1281_driver_hal.o(.constdata) refers to sx1281_driver.o(i.SX1281SetCrcPolynomial) for SX1281SetCrcPolynomial
    sx1281_driver_hal.o(.constdata) refers to sx1281_driver.o(i.SX1281SetWhiteningSeed) for SX1281SetWhiteningSeed
    sx1281_driver_hal.o(.constdata) refers to sx1281_driver.o(i.SX1281GetFrequencyError) for SX1281GetFrequencyError
    sx1281_driver_spi.o(i.SpiIn) refers to spi_1.o(i.BSP_SPI_Transmit) for BSP_SPI_Transmit
    sx1281_driver_spi.o(i.SpiIn) refers to sx1281_driver_spi.o(.data) for .data
    sx1281_driver_spi.o(i.SpiInOut) refers to spi_1.o(i.BSP_SPI_TransmitReceive) for BSP_SPI_TransmitReceive
    sx1281_driver_spi.o(i.SpiInOut) refers to sx1281_driver_spi.o(.data) for .data
    sx1281_driver_spi.o(i.SpiInit) refers to spi_1.o(i.BSP_SPI_RegisterCallback) for BSP_SPI_RegisterCallback
    sx1281_driver_spi.o(i.SpiInit) refers to sx1281_driver_spi.o(i.txrx_cplt_cb) for txrx_cplt_cb
    sx1281_driver_spi.o(i.SpiInit) refers to sx1281_driver_spi.o(i.tx_cplt_cb) for tx_cplt_cb
    sx1281_driver_spi.o(i.tx_cplt_cb) refers to sx1281_driver_spi.o(.data) for .data
    sx1281_driver_spi.o(i.txrx_cplt_cb) refers to sx1281_driver_spi.o(.data) for .data
    sx1281_header.o(i.SX1281_BSPInit) refers to sx1281_driver_gpio.o(i.GpioInit) for GpioInit
    sx1281_header.o(i.SX1281_BSPInit) refers to sx1281_driver_spi.o(i.SpiInit) for SpiInit
    sx1281_header.o(i.fputc) refers to uart.o(i.BSP_UART_GetHandle) for BSP_UART_GetHandle
    sx1281_header.o(i.fputc) refers to stm32f1xx_hal_uart.o(i.HAL_UART_Transmit) for HAL_UART_Transmit
    gpio_1.o(i.BSP_GPIO_DisableIRQ) refers to stm32f1xx_hal_cortex.o(i.HAL_NVIC_DisableIRQ) for HAL_NVIC_DisableIRQ
    gpio_1.o(i.BSP_GPIO_EnableIRQ) refers to stm32f1xx_hal_cortex.o(i.HAL_NVIC_EnableIRQ) for HAL_NVIC_EnableIRQ
    gpio_1.o(i.BSP_GPIO_ReadPin) refers to stm32f1xx_hal_gpio.o(i.HAL_GPIO_ReadPin) for HAL_GPIO_ReadPin
    gpio_1.o(i.BSP_GPIO_ReadPin) refers to gpio_1.o(.constdata) for .constdata
    gpio_1.o(i.BSP_GPIO_RegisterCallback) refers to gpio_1.o(.constdata) for .constdata
    gpio_1.o(i.BSP_GPIO_RegisterCallback) refers to gpio_1.o(.bss) for .bss
    gpio_1.o(i.BSP_GPIO_TogglePin) refers to stm32f1xx_hal_gpio.o(i.HAL_GPIO_TogglePin) for HAL_GPIO_TogglePin
    gpio_1.o(i.BSP_GPIO_TogglePin) refers to gpio_1.o(.constdata) for .constdata
    gpio_1.o(i.BSP_GPIO_WritePin) refers to stm32f1xx_hal_gpio.o(i.HAL_GPIO_WritePin) for HAL_GPIO_WritePin
    gpio_1.o(i.BSP_GPIO_WritePin) refers to gpio_1.o(.constdata) for .constdata
    gpio_1.o(i.HAL_GPIO_EXTI_Callback) refers to gpio_1.o(.bss) for .bss
    spi_1.o(i.BSP_SPI_GetHandle) refers to spi.o(.bss) for hspi1
    spi_1.o(i.BSP_SPI_GetState) refers to spi_1.o(i.BSP_SPI_GetHandle) for BSP_SPI_GetHandle
    spi_1.o(i.BSP_SPI_GetState) refers to stm32f1xx_hal_spi.o(i.HAL_SPI_GetState) for HAL_SPI_GetState
    spi_1.o(i.BSP_SPI_MemRead) refers to spi_1.o(i.BSP_SPI_Transmit) for BSP_SPI_Transmit
    spi_1.o(i.BSP_SPI_MemRead) refers to spi_1.o(i.BSP_SPI_Receive) for BSP_SPI_Receive
    spi_1.o(i.BSP_SPI_MemReadByte) refers to spi_1.o(i.BSP_SPI_TransmitReceive) for BSP_SPI_TransmitReceive
    spi_1.o(i.BSP_SPI_MemWrite) refers to spi_1.o(i.BSP_SPI_Transmit) for BSP_SPI_Transmit
    spi_1.o(i.BSP_SPI_MemWriteByte) refers to spi_1.o(i.BSP_SPI_Transmit) for BSP_SPI_Transmit
    spi_1.o(i.BSP_SPI_Receive) refers to spi_1.o(i.BSP_SPI_GetHandle) for BSP_SPI_GetHandle
    spi_1.o(i.BSP_SPI_Receive) refers to stm32f1xx_hal_spi.o(i.HAL_SPI_Receive_DMA) for HAL_SPI_Receive_DMA
    spi_1.o(i.BSP_SPI_Receive) refers to stm32f1xx_hal_spi.o(i.HAL_SPI_Receive) for HAL_SPI_Receive
    spi_1.o(i.BSP_SPI_RegisterCallback) refers to spi_1.o(.bss) for .bss
    spi_1.o(i.BSP_SPI_Transmit) refers to spi_1.o(i.BSP_SPI_GetHandle) for BSP_SPI_GetHandle
    spi_1.o(i.BSP_SPI_Transmit) refers to stm32f1xx_hal_spi.o(i.HAL_SPI_Transmit_DMA) for HAL_SPI_Transmit_DMA
    spi_1.o(i.BSP_SPI_Transmit) refers to stm32f1xx_hal_spi.o(i.HAL_SPI_Transmit) for HAL_SPI_Transmit
    spi_1.o(i.BSP_SPI_TransmitReceive) refers to spi_1.o(i.BSP_SPI_GetHandle) for BSP_SPI_GetHandle
    spi_1.o(i.BSP_SPI_TransmitReceive) refers to stm32f1xx_hal_spi.o(i.HAL_SPI_TransmitReceive_DMA) for HAL_SPI_TransmitReceive_DMA
    spi_1.o(i.BSP_SPI_TransmitReceive) refers to stm32f1xx_hal_spi.o(i.HAL_SPI_TransmitReceive) for HAL_SPI_TransmitReceive
    spi_1.o(i.HAL_SPI_AbortCpltCallback) refers to spi_1.o(i.SPI_Get) for SPI_Get
    spi_1.o(i.HAL_SPI_AbortCpltCallback) refers to spi_1.o(.bss) for .bss
    spi_1.o(i.HAL_SPI_ErrorCallback) refers to spi_1.o(i.SPI_Get) for SPI_Get
    spi_1.o(i.HAL_SPI_ErrorCallback) refers to spi_1.o(.bss) for .bss
    spi_1.o(i.HAL_SPI_RxCpltCallback) refers to spi_1.o(i.SPI_Get) for SPI_Get
    spi_1.o(i.HAL_SPI_RxCpltCallback) refers to spi_1.o(.bss) for .bss
    spi_1.o(i.HAL_SPI_RxHalfCpltCallback) refers to spi_1.o(i.SPI_Get) for SPI_Get
    spi_1.o(i.HAL_SPI_RxHalfCpltCallback) refers to spi_1.o(.bss) for .bss
    spi_1.o(i.HAL_SPI_TxCpltCallback) refers to spi_1.o(i.SPI_Get) for SPI_Get
    spi_1.o(i.HAL_SPI_TxCpltCallback) refers to spi_1.o(.bss) for .bss
    spi_1.o(i.HAL_SPI_TxHalfCpltCallback) refers to spi_1.o(i.SPI_Get) for SPI_Get
    spi_1.o(i.HAL_SPI_TxHalfCpltCallback) refers to spi_1.o(.bss) for .bss
    spi_1.o(i.HAL_SPI_TxRxCpltCallback) refers to spi_1.o(i.SPI_Get) for SPI_Get
    spi_1.o(i.HAL_SPI_TxRxCpltCallback) refers to spi_1.o(.bss) for .bss
    spi_1.o(i.HAL_SPI_TxRxHalfCpltCallback) refers to spi_1.o(i.SPI_Get) for SPI_Get
    spi_1.o(i.HAL_SPI_TxRxHalfCpltCallback) refers to spi_1.o(.bss) for .bss
    uart.o(i.BSP_UART_GetHandle) refers to usart.o(.bss) for huart2
    uart.o(i.BSP_UART_IRQHandler) refers to uart.o(i.UART_Get) for UART_Get
    uart.o(i.BSP_UART_IRQHandler) refers to uart.o(.bss) for .bss
    uart.o(i.BSP_UART_Receive) refers to uart.o(i.BSP_UART_GetHandle) for BSP_UART_GetHandle
    uart.o(i.BSP_UART_Receive) refers to stm32f1xx_hal_uart.o(i.HAL_UART_Receive_DMA) for HAL_UART_Receive_DMA
    uart.o(i.BSP_UART_Receive) refers to stm32f1xx_hal_uart.o(i.HAL_UART_Receive_IT) for HAL_UART_Receive_IT
    uart.o(i.BSP_UART_RegisterCallback) refers to uart.o(.bss) for .bss
    uart.o(i.BSP_UART_Transmit) refers to uart.o(i.BSP_UART_GetHandle) for BSP_UART_GetHandle
    uart.o(i.BSP_UART_Transmit) refers to stm32f1xx_hal_uart.o(i.HAL_UART_Transmit_DMA) for HAL_UART_Transmit_DMA
    uart.o(i.BSP_UART_Transmit) refers to stm32f1xx_hal_uart.o(i.HAL_UART_Transmit_IT) for HAL_UART_Transmit_IT
    uart.o(i.HAL_UART_AbortCpltCallback) refers to uart.o(i.UART_Get) for UART_Get
    uart.o(i.HAL_UART_AbortCpltCallback) refers to uart.o(.bss) for .bss
    uart.o(i.HAL_UART_AbortReceiveCpltCallback) refers to uart.o(i.UART_Get) for UART_Get
    uart.o(i.HAL_UART_AbortReceiveCpltCallback) refers to uart.o(.bss) for .bss
    uart.o(i.HAL_UART_AbortTransmitCpltCallback) refers to uart.o(i.UART_Get) for UART_Get
    uart.o(i.HAL_UART_AbortTransmitCpltCallback) refers to uart.o(.bss) for .bss
    uart.o(i.HAL_UART_ErrorCallback) refers to uart.o(i.UART_Get) for UART_Get
    uart.o(i.HAL_UART_ErrorCallback) refers to uart.o(.bss) for .bss
    uart.o(i.HAL_UART_RxCpltCallback) refers to uart.o(i.UART_Get) for UART_Get
    uart.o(i.HAL_UART_RxCpltCallback) refers to uart.o(.bss) for .bss
    uart.o(i.HAL_UART_RxHalfCpltCallback) refers to uart.o(i.UART_Get) for UART_Get
    uart.o(i.HAL_UART_RxHalfCpltCallback) refers to uart.o(.bss) for .bss
    uart.o(i.HAL_UART_TxCpltCallback) refers to uart.o(i.UART_Get) for UART_Get
    uart.o(i.HAL_UART_TxCpltCallback) refers to uart.o(.bss) for .bss
    uart.o(i.HAL_UART_TxHalfCpltCallback) refers to uart.o(i.UART_Get) for UART_Get
    uart.o(i.HAL_UART_TxHalfCpltCallback) refers to uart.o(.bss) for .bss
    lcd.o(i.LCD_Clear) refers to lcd.o(i.LCD_SetAddressWindow) for LCD_SetAddressWindow
    lcd.o(i.LCD_Clear) refers to malloc.o(i.malloc) for malloc
    lcd.o(i.LCD_Clear) refers to lcd.o(i.LCD_WriteDataBuffer_DMA) for LCD_WriteDataBuffer_DMA
    lcd.o(i.LCD_Clear) refers to malloc.o(i.free) for free
    lcd.o(i.LCD_DrawBitmap) refers to lcd.o(i.LCD_DrawPoint) for LCD_DrawPoint
    lcd.o(i.LCD_DrawChar) refers to lcd.o(i.LCD_DrawPoint) for LCD_DrawPoint
    lcd.o(i.LCD_DrawChar) refers to lcd.o(.constdata) for .constdata
    lcd.o(i.LCD_DrawFloat) refers to f2d.o(.text) for __aeabi_f2d
    lcd.o(i.LCD_DrawFloat) refers to printfa.o(i.__0snprintf) for __2snprintf
    lcd.o(i.LCD_DrawFloat) refers to lcd.o(i.LCD_DrawString) for LCD_DrawString
    lcd.o(i.LCD_DrawHollowCircle) refers to lcd.o(i.LCD_DrawPoint) for LCD_DrawPoint
    lcd.o(i.LCD_DrawInteger) refers to printfa.o(i.__0snprintf) for __2snprintf
    lcd.o(i.LCD_DrawInteger) refers to lcd.o(i.LCD_DrawString) for LCD_DrawString
    lcd.o(i.LCD_DrawLine) refers to lcd.o(i.LCD_DrawPoint) for LCD_DrawPoint
    lcd.o(i.LCD_DrawPoint) refers to lcd.o(i.LCD_SetAddressWindow) for LCD_SetAddressWindow
    lcd.o(i.LCD_DrawPoint) refers to lcd.o(i.LCD_WriteDataBuffer) for LCD_WriteDataBuffer
    lcd.o(i.LCD_DrawPoint) refers to lcd.o(.data) for .data
    lcd.o(i.LCD_DrawRectangle) refers to lcd.o(i.LCD_DrawLine) for LCD_DrawLine
    lcd.o(i.LCD_DrawSolidCircle) refers to lcd.o(i.LCD_DrawLine) for LCD_DrawLine
    lcd.o(i.LCD_DrawSolidRectangle) refers to lcd.o(i.LCD_DrawLine) for LCD_DrawLine
    lcd.o(i.LCD_DrawString) refers to lcd.o(i.LCD_DrawChar) for LCD_DrawChar
    lcd.o(i.LCD_Init) refers to stm32f1xx_hal_gpio.o(i.HAL_GPIO_WritePin) for HAL_GPIO_WritePin
    lcd.o(i.LCD_Init) refers to stm32f1xx_hal.o(i.HAL_Delay) for HAL_Delay
    lcd.o(i.LCD_Init) refers to lcd.o(i.LCD_WriteCommand) for LCD_WriteCommand
    lcd.o(i.LCD_Init) refers to lcd.o(i.LCD_WriteData) for LCD_WriteData
    lcd.o(i.LCD_Init) refers to lcd.o(i.LCD_WriteDataBuffer) for LCD_WriteDataBuffer
    lcd.o(i.LCD_Init) refers to lcd.o(.data) for .data
    lcd.o(i.LCD_SetAddressWindow) refers to lcd.o(i.LCD_WriteCommand) for LCD_WriteCommand
    lcd.o(i.LCD_SetAddressWindow) refers to lcd.o(i.LCD_WriteDataBuffer) for LCD_WriteDataBuffer
    lcd.o(i.LCD_WriteCommand) refers to stm32f1xx_hal_gpio.o(i.HAL_GPIO_WritePin) for HAL_GPIO_WritePin
    lcd.o(i.LCD_WriteCommand) refers to spi_1.o(i.BSP_SPI_Transmit) for BSP_SPI_Transmit
    lcd.o(i.LCD_WriteData) refers to stm32f1xx_hal_gpio.o(i.HAL_GPIO_WritePin) for HAL_GPIO_WritePin
    lcd.o(i.LCD_WriteData) refers to spi_1.o(i.BSP_SPI_Transmit) for BSP_SPI_Transmit
    lcd.o(i.LCD_WriteDataBuffer) refers to lcd.o(i.LCD_WriteDataBuffer_DMA) for LCD_WriteDataBuffer_DMA
    lcd.o(i.LCD_WriteDataBuffer) refers to stm32f1xx_hal_gpio.o(i.HAL_GPIO_WritePin) for HAL_GPIO_WritePin
    lcd.o(i.LCD_WriteDataBuffer) refers to spi_1.o(i.BSP_SPI_Transmit) for BSP_SPI_Transmit
    lcd.o(i.LCD_WriteDataBuffer_DMA) refers to stm32f1xx_hal_gpio.o(i.HAL_GPIO_WritePin) for HAL_GPIO_WritePin
    lcd.o(i.LCD_WriteDataBuffer_DMA) refers to spi_1.o(i.BSP_SPI_Transmit) for BSP_SPI_Transmit
    lcd.o(i.LCD_WriteDataBuffer_DMA) refers to spi_1.o(i.BSP_SPI_GetState) for BSP_SPI_GetState
    crc8.o(i.CRC8_Calc) refers to crc8.o(.constdata) for .constdata
    crc8.o(i.CRC8_Verify) refers to crc8.o(i.CRC8_Calc) for CRC8_Calc
    crc16.o(i.CRC16_Calc) refers to crc16.o(.constdata) for .constdata
    crc16.o(i.CRC16_Verify) refers to crc16.o(i.CRC16_Calc) for CRC16_Calc
    entry.o(.ARM.Collect$$$$00000000) refers (Special) to entry10a.o(.ARM.Collect$$$$0000000F) for __rt_final_cpp
    entry.o(.ARM.Collect$$$$00000000) refers (Special) to entry11a.o(.ARM.Collect$$$$00000011) for __rt_final_exit
    entry.o(.ARM.Collect$$$$00000000) refers (Special) to entry12b.o(.ARM.Collect$$$$0000000E) for __rt_lib_shutdown_fini
    entry.o(.ARM.Collect$$$$00000000) refers (Special) to entry7b.o(.ARM.Collect$$$$00000008) for _main_clock
    entry.o(.ARM.Collect$$$$00000000) refers (Special) to entry8b.o(.ARM.Collect$$$$0000000A) for _main_cpp_init
    entry.o(.ARM.Collect$$$$00000000) refers (Special) to entry9a.o(.ARM.Collect$$$$0000000B) for _main_init
    entry.o(.ARM.Collect$$$$00000000) refers (Special) to entry5.o(.ARM.Collect$$$$00000004) for _main_scatterload
    entry.o(.ARM.Collect$$$$00000000) refers (Special) to entry2.o(.ARM.Collect$$$$00000001) for _main_stk
    printfb.o(i.__0fprintf$bare) refers to printfb.o(i._printf_core) for _printf_core
    printfb.o(i.__0fprintf$bare) refers to sx1281_header.o(i.fputc) for fputc
    printfb.o(i.__0printf$bare) refers to printfb.o(i._printf_core) for _printf_core
    printfb.o(i.__0printf$bare) refers to sx1281_header.o(i.fputc) for fputc
    printfb.o(i.__0printf$bare) refers to stdout.o(.data) for __stdout
    printfb.o(i.__0snprintf$bare) refers to printfb.o(i._printf_core) for _printf_core
    printfb.o(i.__0snprintf$bare) refers to printfb.o(i._snputc) for _snputc
    printfb.o(i.__0sprintf$bare) refers to printfb.o(i._printf_core) for _printf_core
    printfb.o(i.__0sprintf$bare) refers to printfb.o(i._sputc) for _sputc
    printfb.o(i.__0vfprintf$bare) refers to printfb.o(i._printf_core) for _printf_core
    printfb.o(i.__0vfprintf$bare) refers to sx1281_header.o(i.fputc) for fputc
    printfb.o(i.__0vprintf$bare) refers to printfb.o(i._printf_core) for _printf_core
    printfb.o(i.__0vprintf$bare) refers to sx1281_header.o(i.fputc) for fputc
    printfb.o(i.__0vprintf$bare) refers to stdout.o(.data) for __stdout
    printfb.o(i.__0vsnprintf$bare) refers to printfb.o(i._printf_core) for _printf_core
    printfb.o(i.__0vsnprintf$bare) refers to printfb.o(i._snputc) for _snputc
    printfb.o(i.__0vsprintf$bare) refers to printfb.o(i._printf_core) for _printf_core
    printfb.o(i.__0vsprintf$bare) refers to printfb.o(i._sputc) for _sputc
    printf0.o(i.__0fprintf$0) refers to printf0.o(i._printf_core) for _printf_core
    printf0.o(i.__0fprintf$0) refers to sx1281_header.o(i.fputc) for fputc
    printf0.o(i.__0printf$0) refers to printf0.o(i._printf_core) for _printf_core
    printf0.o(i.__0printf$0) refers to sx1281_header.o(i.fputc) for fputc
    printf0.o(i.__0printf$0) refers to stdout.o(.data) for __stdout
    printf0.o(i.__0snprintf$0) refers to printf0.o(i._printf_core) for _printf_core
    printf0.o(i.__0snprintf$0) refers to printf0.o(i._snputc) for _snputc
    printf0.o(i.__0sprintf$0) refers to printf0.o(i._printf_core) for _printf_core
    printf0.o(i.__0sprintf$0) refers to printf0.o(i._sputc) for _sputc
    printf0.o(i.__0vfprintf$0) refers to printf0.o(i._printf_core) for _printf_core
    printf0.o(i.__0vfprintf$0) refers to sx1281_header.o(i.fputc) for fputc
    printf0.o(i.__0vprintf$0) refers to printf0.o(i._printf_core) for _printf_core
    printf0.o(i.__0vprintf$0) refers to sx1281_header.o(i.fputc) for fputc
    printf0.o(i.__0vprintf$0) refers to stdout.o(.data) for __stdout
    printf0.o(i.__0vsnprintf$0) refers to printf0.o(i._printf_core) for _printf_core
    printf0.o(i.__0vsnprintf$0) refers to printf0.o(i._snputc) for _snputc
    printf0.o(i.__0vsprintf$0) refers to printf0.o(i._printf_core) for _printf_core
    printf0.o(i.__0vsprintf$0) refers to printf0.o(i._sputc) for _sputc
    printf1.o(i.__0fprintf$1) refers to printf1.o(i._printf_core) for _printf_core
    printf1.o(i.__0fprintf$1) refers to sx1281_header.o(i.fputc) for fputc
    printf1.o(i.__0printf$1) refers to printf1.o(i._printf_core) for _printf_core
    printf1.o(i.__0printf$1) refers to sx1281_header.o(i.fputc) for fputc
    printf1.o(i.__0printf$1) refers to stdout.o(.data) for __stdout
    printf1.o(i.__0snprintf$1) refers to printf1.o(i._printf_core) for _printf_core
    printf1.o(i.__0snprintf$1) refers to printf1.o(i._snputc) for _snputc
    printf1.o(i.__0sprintf$1) refers to printf1.o(i._printf_core) for _printf_core
    printf1.o(i.__0sprintf$1) refers to printf1.o(i._sputc) for _sputc
    printf1.o(i.__0vfprintf$1) refers to printf1.o(i._printf_core) for _printf_core
    printf1.o(i.__0vfprintf$1) refers to sx1281_header.o(i.fputc) for fputc
    printf1.o(i.__0vprintf$1) refers to printf1.o(i._printf_core) for _printf_core
    printf1.o(i.__0vprintf$1) refers to sx1281_header.o(i.fputc) for fputc
    printf1.o(i.__0vprintf$1) refers to stdout.o(.data) for __stdout
    printf1.o(i.__0vsnprintf$1) refers to printf1.o(i._printf_core) for _printf_core
    printf1.o(i.__0vsnprintf$1) refers to printf1.o(i._snputc) for _snputc
    printf1.o(i.__0vsprintf$1) refers to printf1.o(i._printf_core) for _printf_core
    printf1.o(i.__0vsprintf$1) refers to printf1.o(i._sputc) for _sputc
    printf1.o(i._printf_core) refers to uidiv.o(.text) for __aeabi_uidivmod
    printf2.o(i.__0fprintf$2) refers to printf2.o(i._printf_core) for _printf_core
    printf2.o(i.__0fprintf$2) refers to sx1281_header.o(i.fputc) for fputc
    printf2.o(i.__0printf$2) refers to printf2.o(i._printf_core) for _printf_core
    printf2.o(i.__0printf$2) refers to sx1281_header.o(i.fputc) for fputc
    printf2.o(i.__0printf$2) refers to stdout.o(.data) for __stdout
    printf2.o(i.__0snprintf$2) refers to printf2.o(i._printf_core) for _printf_core
    printf2.o(i.__0snprintf$2) refers to printf2.o(i._snputc) for _snputc
    printf2.o(i.__0sprintf$2) refers to printf2.o(i._printf_core) for _printf_core
    printf2.o(i.__0sprintf$2) refers to printf2.o(i._sputc) for _sputc
    printf2.o(i.__0vfprintf$2) refers to printf2.o(i._printf_core) for _printf_core
    printf2.o(i.__0vfprintf$2) refers to sx1281_header.o(i.fputc) for fputc
    printf2.o(i.__0vprintf$2) refers to printf2.o(i._printf_core) for _printf_core
    printf2.o(i.__0vprintf$2) refers to sx1281_header.o(i.fputc) for fputc
    printf2.o(i.__0vprintf$2) refers to stdout.o(.data) for __stdout
    printf2.o(i.__0vsnprintf$2) refers to printf2.o(i._printf_core) for _printf_core
    printf2.o(i.__0vsnprintf$2) refers to printf2.o(i._snputc) for _snputc
    printf2.o(i.__0vsprintf$2) refers to printf2.o(i._printf_core) for _printf_core
    printf2.o(i.__0vsprintf$2) refers to printf2.o(i._sputc) for _sputc
    printf3.o(i.__0fprintf$3) refers to printf3.o(i._printf_core) for _printf_core
    printf3.o(i.__0fprintf$3) refers to sx1281_header.o(i.fputc) for fputc
    printf3.o(i.__0printf$3) refers to printf3.o(i._printf_core) for _printf_core
    printf3.o(i.__0printf$3) refers to sx1281_header.o(i.fputc) for fputc
    printf3.o(i.__0printf$3) refers to stdout.o(.data) for __stdout
    printf3.o(i.__0snprintf$3) refers to printf3.o(i._printf_core) for _printf_core
    printf3.o(i.__0snprintf$3) refers to printf3.o(i._snputc) for _snputc
    printf3.o(i.__0sprintf$3) refers to printf3.o(i._printf_core) for _printf_core
    printf3.o(i.__0sprintf$3) refers to printf3.o(i._sputc) for _sputc
    printf3.o(i.__0vfprintf$3) refers to printf3.o(i._printf_core) for _printf_core
    printf3.o(i.__0vfprintf$3) refers to sx1281_header.o(i.fputc) for fputc
    printf3.o(i.__0vprintf$3) refers to printf3.o(i._printf_core) for _printf_core
    printf3.o(i.__0vprintf$3) refers to sx1281_header.o(i.fputc) for fputc
    printf3.o(i.__0vprintf$3) refers to stdout.o(.data) for __stdout
    printf3.o(i.__0vsnprintf$3) refers to printf3.o(i._printf_core) for _printf_core
    printf3.o(i.__0vsnprintf$3) refers to printf3.o(i._snputc) for _snputc
    printf3.o(i.__0vsprintf$3) refers to printf3.o(i._printf_core) for _printf_core
    printf3.o(i.__0vsprintf$3) refers to printf3.o(i._sputc) for _sputc
    printf3.o(i._printf_core) refers to uidiv.o(.text) for __aeabi_uidivmod
    printf4.o(i.__0fprintf$4) refers to printf4.o(i._printf_core) for _printf_core
    printf4.o(i.__0fprintf$4) refers to sx1281_header.o(i.fputc) for fputc
    printf4.o(i.__0printf$4) refers to printf4.o(i._printf_core) for _printf_core
    printf4.o(i.__0printf$4) refers to sx1281_header.o(i.fputc) for fputc
    printf4.o(i.__0printf$4) refers to stdout.o(.data) for __stdout
    printf4.o(i.__0snprintf$4) refers to printf4.o(i._printf_core) for _printf_core
    printf4.o(i.__0snprintf$4) refers to printf4.o(i._snputc) for _snputc
    printf4.o(i.__0sprintf$4) refers to printf4.o(i._printf_core) for _printf_core
    printf4.o(i.__0sprintf$4) refers to printf4.o(i._sputc) for _sputc
    printf4.o(i.__0vfprintf$4) refers to printf4.o(i._printf_core) for _printf_core
    printf4.o(i.__0vfprintf$4) refers to sx1281_header.o(i.fputc) for fputc
    printf4.o(i.__0vprintf$4) refers to printf4.o(i._printf_core) for _printf_core
    printf4.o(i.__0vprintf$4) refers to sx1281_header.o(i.fputc) for fputc
    printf4.o(i.__0vprintf$4) refers to stdout.o(.data) for __stdout
    printf4.o(i.__0vsnprintf$4) refers to printf4.o(i._printf_core) for _printf_core
    printf4.o(i.__0vsnprintf$4) refers to printf4.o(i._snputc) for _snputc
    printf4.o(i.__0vsprintf$4) refers to printf4.o(i._printf_core) for _printf_core
    printf4.o(i.__0vsprintf$4) refers to printf4.o(i._sputc) for _sputc
    printf4.o(i._printf_core) refers to uldiv.o(.text) for __aeabi_uldivmod
    printf5.o(i.__0fprintf$5) refers to printf5.o(i._printf_core) for _printf_core
    printf5.o(i.__0fprintf$5) refers to sx1281_header.o(i.fputc) for fputc
    printf5.o(i.__0printf$5) refers to printf5.o(i._printf_core) for _printf_core
    printf5.o(i.__0printf$5) refers to sx1281_header.o(i.fputc) for fputc
    printf5.o(i.__0printf$5) refers to stdout.o(.data) for __stdout
    printf5.o(i.__0snprintf$5) refers to printf5.o(i._printf_core) for _printf_core
    printf5.o(i.__0snprintf$5) refers to printf5.o(i._snputc) for _snputc
    printf5.o(i.__0sprintf$5) refers to printf5.o(i._printf_core) for _printf_core
    printf5.o(i.__0sprintf$5) refers to printf5.o(i._sputc) for _sputc
    printf5.o(i.__0vfprintf$5) refers to printf5.o(i._printf_core) for _printf_core
    printf5.o(i.__0vfprintf$5) refers to sx1281_header.o(i.fputc) for fputc
    printf5.o(i.__0vprintf$5) refers to printf5.o(i._printf_core) for _printf_core
    printf5.o(i.__0vprintf$5) refers to sx1281_header.o(i.fputc) for fputc
    printf5.o(i.__0vprintf$5) refers to stdout.o(.data) for __stdout
    printf5.o(i.__0vsnprintf$5) refers to printf5.o(i._printf_core) for _printf_core
    printf5.o(i.__0vsnprintf$5) refers to printf5.o(i._snputc) for _snputc
    printf5.o(i.__0vsprintf$5) refers to printf5.o(i._printf_core) for _printf_core
    printf5.o(i.__0vsprintf$5) refers to printf5.o(i._sputc) for _sputc
    printf5.o(i._printf_core) refers to uldiv.o(.text) for __aeabi_uldivmod
    printf6.o(i.__0fprintf$6) refers to printf6.o(i._printf_core) for _printf_core
    printf6.o(i.__0fprintf$6) refers to sx1281_header.o(i.fputc) for fputc
    printf6.o(i.__0printf$6) refers to printf6.o(i._printf_core) for _printf_core
    printf6.o(i.__0printf$6) refers to sx1281_header.o(i.fputc) for fputc
    printf6.o(i.__0printf$6) refers to stdout.o(.data) for __stdout
    printf6.o(i.__0snprintf$6) refers to printf6.o(i._printf_core) for _printf_core
    printf6.o(i.__0snprintf$6) refers to printf6.o(i._snputc) for _snputc
    printf6.o(i.__0sprintf$6) refers to printf6.o(i._printf_core) for _printf_core
    printf6.o(i.__0sprintf$6) refers to printf6.o(i._sputc) for _sputc
    printf6.o(i.__0vfprintf$6) refers to printf6.o(i._printf_core) for _printf_core
    printf6.o(i.__0vfprintf$6) refers to sx1281_header.o(i.fputc) for fputc
    printf6.o(i.__0vprintf$6) refers to printf6.o(i._printf_core) for _printf_core
    printf6.o(i.__0vprintf$6) refers to sx1281_header.o(i.fputc) for fputc
    printf6.o(i.__0vprintf$6) refers to stdout.o(.data) for __stdout
    printf6.o(i.__0vsnprintf$6) refers to printf6.o(i._printf_core) for _printf_core
    printf6.o(i.__0vsnprintf$6) refers to printf6.o(i._snputc) for _snputc
    printf6.o(i.__0vsprintf$6) refers to printf6.o(i._printf_core) for _printf_core
    printf6.o(i.__0vsprintf$6) refers to printf6.o(i._sputc) for _sputc
    printf6.o(i._printf_core) refers to printf6.o(i._printf_pre_padding) for _printf_pre_padding
    printf6.o(i._printf_core) refers to uidiv.o(.text) for __aeabi_uidivmod
    printf6.o(i._printf_core) refers to printf6.o(i._printf_post_padding) for _printf_post_padding
    printf7.o(i.__0fprintf$7) refers to printf7.o(i._printf_core) for _printf_core
    printf7.o(i.__0fprintf$7) refers to sx1281_header.o(i.fputc) for fputc
    printf7.o(i.__0printf$7) refers to printf7.o(i._printf_core) for _printf_core
    printf7.o(i.__0printf$7) refers to sx1281_header.o(i.fputc) for fputc
    printf7.o(i.__0printf$7) refers to stdout.o(.data) for __stdout
    printf7.o(i.__0snprintf$7) refers to printf7.o(i._printf_core) for _printf_core
    printf7.o(i.__0snprintf$7) refers to printf7.o(i._snputc) for _snputc
    printf7.o(i.__0sprintf$7) refers to printf7.o(i._printf_core) for _printf_core
    printf7.o(i.__0sprintf$7) refers to printf7.o(i._sputc) for _sputc
    printf7.o(i.__0vfprintf$7) refers to printf7.o(i._printf_core) for _printf_core
    printf7.o(i.__0vfprintf$7) refers to sx1281_header.o(i.fputc) for fputc
    printf7.o(i.__0vprintf$7) refers to printf7.o(i._printf_core) for _printf_core
    printf7.o(i.__0vprintf$7) refers to sx1281_header.o(i.fputc) for fputc
    printf7.o(i.__0vprintf$7) refers to stdout.o(.data) for __stdout
    printf7.o(i.__0vsnprintf$7) refers to printf7.o(i._printf_core) for _printf_core
    printf7.o(i.__0vsnprintf$7) refers to printf7.o(i._snputc) for _snputc
    printf7.o(i.__0vsprintf$7) refers to printf7.o(i._printf_core) for _printf_core
    printf7.o(i.__0vsprintf$7) refers to printf7.o(i._sputc) for _sputc
    printf7.o(i._printf_core) refers to printf7.o(i._printf_pre_padding) for _printf_pre_padding
    printf7.o(i._printf_core) refers to uldiv.o(.text) for __aeabi_uldivmod
    printf7.o(i._printf_core) refers to printf7.o(i._printf_post_padding) for _printf_post_padding
    printf8.o(i.__0fprintf$8) refers to printf8.o(i._printf_core) for _printf_core
    printf8.o(i.__0fprintf$8) refers to sx1281_header.o(i.fputc) for fputc
    printf8.o(i.__0printf$8) refers to printf8.o(i._printf_core) for _printf_core
    printf8.o(i.__0printf$8) refers to sx1281_header.o(i.fputc) for fputc
    printf8.o(i.__0printf$8) refers to stdout.o(.data) for __stdout
    printf8.o(i.__0snprintf$8) refers to printf8.o(i._printf_core) for _printf_core
    printf8.o(i.__0snprintf$8) refers to printf8.o(i._snputc) for _snputc
    printf8.o(i.__0sprintf$8) refers to printf8.o(i._printf_core) for _printf_core
    printf8.o(i.__0sprintf$8) refers to printf8.o(i._sputc) for _sputc
    printf8.o(i.__0vfprintf$8) refers to printf8.o(i._printf_core) for _printf_core
    printf8.o(i.__0vfprintf$8) refers to sx1281_header.o(i.fputc) for fputc
    printf8.o(i.__0vprintf$8) refers to printf8.o(i._printf_core) for _printf_core
    printf8.o(i.__0vprintf$8) refers to sx1281_header.o(i.fputc) for fputc
    printf8.o(i.__0vprintf$8) refers to stdout.o(.data) for __stdout
    printf8.o(i.__0vsnprintf$8) refers to printf8.o(i._printf_core) for _printf_core
    printf8.o(i.__0vsnprintf$8) refers to printf8.o(i._snputc) for _snputc
    printf8.o(i.__0vsprintf$8) refers to printf8.o(i._printf_core) for _printf_core
    printf8.o(i.__0vsprintf$8) refers to printf8.o(i._sputc) for _sputc
    printf8.o(i._printf_core) refers to printf8.o(i._printf_pre_padding) for _printf_pre_padding
    printf8.o(i._printf_core) refers to uldiv.o(.text) for __aeabi_uldivmod
    printf8.o(i._printf_core) refers to printf8.o(i._printf_post_padding) for _printf_post_padding
    printfa.o(i.__0fprintf) refers (Special) to iusefp.o(.text) for __I$use$fp
    printfa.o(i.__0fprintf) refers to printfa.o(i._printf_core) for _printf_core
    printfa.o(i.__0fprintf) refers to sx1281_header.o(i.fputc) for fputc
    printfa.o(i.__0printf) refers (Special) to iusefp.o(.text) for __I$use$fp
    printfa.o(i.__0printf) refers to printfa.o(i._printf_core) for _printf_core
    printfa.o(i.__0printf) refers to sx1281_header.o(i.fputc) for fputc
    printfa.o(i.__0printf) refers to stdout.o(.data) for __stdout
    printfa.o(i.__0snprintf) refers (Special) to iusefp.o(.text) for __I$use$fp
    printfa.o(i.__0snprintf) refers to printfa.o(i._printf_core) for _printf_core
    printfa.o(i.__0snprintf) refers to printfa.o(i._snputc) for _snputc
    printfa.o(i.__0sprintf) refers (Special) to iusefp.o(.text) for __I$use$fp
    printfa.o(i.__0sprintf) refers to printfa.o(i._printf_core) for _printf_core
    printfa.o(i.__0sprintf) refers to printfa.o(i._sputc) for _sputc
    printfa.o(i.__0vfprintf) refers (Special) to iusefp.o(.text) for __I$use$fp
    printfa.o(i.__0vfprintf) refers to printfa.o(i._printf_core) for _printf_core
    printfa.o(i.__0vfprintf) refers to sx1281_header.o(i.fputc) for fputc
    printfa.o(i.__0vprintf) refers (Special) to iusefp.o(.text) for __I$use$fp
    printfa.o(i.__0vprintf) refers to printfa.o(i._printf_core) for _printf_core
    printfa.o(i.__0vprintf) refers to sx1281_header.o(i.fputc) for fputc
    printfa.o(i.__0vprintf) refers to stdout.o(.data) for __stdout
    printfa.o(i.__0vsnprintf) refers (Special) to iusefp.o(.text) for __I$use$fp
    printfa.o(i.__0vsnprintf) refers to printfa.o(i._printf_core) for _printf_core
    printfa.o(i.__0vsnprintf) refers to printfa.o(i._snputc) for _snputc
    printfa.o(i.__0vsprintf) refers (Special) to iusefp.o(.text) for __I$use$fp
    printfa.o(i.__0vsprintf) refers to printfa.o(i._printf_core) for _printf_core
    printfa.o(i.__0vsprintf) refers to printfa.o(i._sputc) for _sputc
    printfa.o(i._fp_digits) refers (Special) to iusefp.o(.text) for __I$use$fp
    printfa.o(i._fp_digits) refers to dmul.o(.text) for __aeabi_dmul
    printfa.o(i._fp_digits) refers to ddiv.o(.text) for __aeabi_ddiv
    printfa.o(i._fp_digits) refers to cdrcmple.o(.text) for __aeabi_cdrcmple
    printfa.o(i._fp_digits) refers to dadd.o(.text) for __aeabi_dadd
    printfa.o(i._fp_digits) refers to dfixul.o(.text) for __aeabi_d2ulz
    printfa.o(i._fp_digits) refers to uldiv.o(.text) for __aeabi_uldivmod
    printfa.o(i._printf_core) refers (Special) to iusefp.o(.text) for __I$use$fp
    printfa.o(i._printf_core) refers to printfa.o(i._printf_pre_padding) for _printf_pre_padding
    printfa.o(i._printf_core) refers to uldiv.o(.text) for __aeabi_uldivmod
    printfa.o(i._printf_core) refers to printfa.o(i._printf_post_padding) for _printf_post_padding
    printfa.o(i._printf_core) refers to printfa.o(i._fp_digits) for _fp_digits
    printfa.o(i._printf_core) refers to uidiv.o(.text) for __aeabi_uidivmod
    printfa.o(i._printf_post_padding) refers (Special) to iusefp.o(.text) for __I$use$fp
    printfa.o(i._printf_pre_padding) refers (Special) to iusefp.o(.text) for __I$use$fp
    printfa.o(i._snputc) refers (Special) to iusefp.o(.text) for __I$use$fp
    printfa.o(i._sputc) refers (Special) to iusefp.o(.text) for __I$use$fp
    malloc.o(i.free) refers to mvars.o(.data) for __microlib_freelist
    malloc.o(i.malloc) refers to mvars.o(.data) for __microlib_freelist_initialised
    malloc.o(i.malloc) refers to mvars.o(.data) for __microlib_freelist
    malloc.o(i.malloc) refers to startup_stm32f103xb.o(HEAP) for __heap_base
    mallocr.o(i.__free$realloc) refers to mvars.o(.data) for __microlib_freelist
    mallocr.o(i.__malloc$realloc) refers to mallocr.o(i.internal_alloc) for internal_alloc
    mallocr.o(i.__malloc$realloc) refers to mvars.o(.data) for __microlib_freelist_initialised
    mallocr.o(i.__malloc$realloc) refers to startup_stm32f103xb.o(HEAP) for __heap_base
    mallocr.o(i.__malloc$realloc) refers to mvars.o(.data) for __microlib_freelist
    mallocr.o(i.internal_alloc) refers to memcpya.o(.text) for __aeabi_memcpy
    mallocr.o(i.internal_alloc) refers to mvars.o(.data) for __microlib_freelist
    mallocr.o(i.realloc) refers to mallocr.o(i.__free$realloc) for __free$realloc
    mallocr.o(i.realloc) refers to mallocr.o(i.internal_alloc) for internal_alloc
    mallocr.o(i.realloc) refers to mallocr.o(i.__malloc$realloc) for __malloc$realloc
    mallocr.o(i.realloc) refers to mvars.o(.data) for __microlib_freelist
    malloca.o(i.__aligned_malloc) refers to mvars.o(.data) for __microlib_freelist_initialised
    malloca.o(i.__aligned_malloc) refers to mvars.o(.data) for __microlib_freelist
    malloca.o(i.__aligned_malloc) refers to startup_stm32f103xb.o(HEAP) for __heap_base
    malloca.o(i.__free$memalign) refers to mvars.o(.data) for __microlib_freelist
    malloca.o(i.__malloc$memalign) refers to malloca.o(i.__aligned_malloc) for __aligned_malloc
    mallocra.o(i.__aligned_malloc$realloc) refers to mallocra.o(i.internal_alloc) for internal_alloc
    mallocra.o(i.__aligned_malloc$realloc) refers to mvars.o(.data) for __microlib_freelist_initialised
    mallocra.o(i.__aligned_malloc$realloc) refers to startup_stm32f103xb.o(HEAP) for __heap_base
    mallocra.o(i.__aligned_malloc$realloc) refers to mvars.o(.data) for __microlib_freelist
    mallocra.o(i.__free$realloc$memalign) refers to mvars.o(.data) for __microlib_freelist
    mallocra.o(i.__malloc$realloc$memalign) refers to mallocra.o(i.__aligned_malloc$realloc) for __aligned_malloc$realloc
    mallocra.o(i.__realloc$memalign) refers to mallocra.o(i.__free$realloc$memalign) for __free$realloc$memalign
    mallocra.o(i.__realloc$memalign) refers to mallocra.o(i.internal_alloc) for internal_alloc
    mallocra.o(i.__realloc$memalign) refers to mallocra.o(i.__malloc$realloc$memalign) for __malloc$realloc$memalign
    mallocra.o(i.__realloc$memalign) refers to mvars.o(.data) for __microlib_freelist
    mallocra.o(i.internal_alloc) refers to memcpya.o(.text) for __aeabi_memcpy
    mallocra.o(i.internal_alloc) refers to mvars.o(.data) for __microlib_freelist
    __0sscanf.o(.text) refers to scanf_char.o(.text) for __vfscanf_char
    __0sscanf.o(.text) refers to _sgetc.o(.text) for _sgetc
    _scanf_int.o(.text) refers to _chval.o(.text) for _chval
    fadd.o(.text) refers (Special) to iusefp.o(.text) for __I$use$fp
    fadd.o(.text) refers to fepilogue.o(.text) for _float_epilogue
    fmul.o(.text) refers (Special) to iusefp.o(.text) for __I$use$fp
    fdiv.o(.text) refers (Special) to iusefp.o(.text) for __I$use$fp
    fdiv.o(.text) refers to fepilogue.o(.text) for _float_round
    fscalb.o(.text) refers (Special) to iusefp.o(.text) for __I$use$fp
    dmul.o(.text) refers (Special) to iusefp.o(.text) for __I$use$fp
    dmul.o(.text) refers to depilogue.o(.text) for _double_epilogue
    ddiv.o(.text) refers (Special) to iusefp.o(.text) for __I$use$fp
    ddiv.o(.text) refers to depilogue.o(.text) for _double_round
    dflti.o(.text) refers (Special) to iusefp.o(.text) for __I$use$fp
    dflti.o(.text) refers to depilogue.o(.text) for _double_epilogue
    dfltui.o(.text) refers (Special) to iusefp.o(.text) for __I$use$fp
    dfltui.o(.text) refers to depilogue.o(.text) for _double_epilogue
    dfixui.o(.text) refers (Special) to iusefp.o(.text) for __I$use$fp
    dfixui.o(.text) refers to llushr.o(.text) for __aeabi_llsr
    f2d.o(.text) refers (Special) to iusefp.o(.text) for __I$use$fp
    cfcmple.o(.text) refers (Special) to iusefp.o(.text) for __I$use$fp
    cfrcmple.o(.text) refers (Special) to iusefp.o(.text) for __I$use$fp
    entry2.o(.ARM.Collect$$$$00000001) refers to entry2.o(.ARM.Collect$$$$00002712) for __lit__00000000
    entry2.o(.ARM.Collect$$$$00002712) refers to startup_stm32f103xb.o(STACK) for __initial_sp
    entry2.o(__vectab_stack_and_reset_area) refers to startup_stm32f103xb.o(STACK) for __initial_sp
    entry2.o(__vectab_stack_and_reset_area) refers to entry.o(.ARM.Collect$$$$00000000) for __main
    entry5.o(.ARM.Collect$$$$00000004) refers to init.o(.text) for __scatterload
    entry9a.o(.ARM.Collect$$$$0000000B) refers to main.o(i.main) for main
    entry9b.o(.ARM.Collect$$$$0000000C) refers to main.o(i.main) for main
    uldiv.o(.text) refers to llushr.o(.text) for __aeabi_llsr
    uldiv.o(.text) refers to llshl.o(.text) for __aeabi_llsl
    scanf_char.o(.text) refers to _scanf.o(.text) for __vfscanf
    scanf_char.o(.text) refers to isspace_c.o(.text) for isspace
    depilogue.o(.text) refers to llshl.o(.text) for __aeabi_llsl
    depilogue.o(.text) refers to llushr.o(.text) for __aeabi_llsr
    dadd.o(.text) refers to llshl.o(.text) for __aeabi_llsl
    dadd.o(.text) refers to llsshr.o(.text) for __aeabi_lasr
    dadd.o(.text) refers to depilogue.o(.text) for _double_epilogue
    dfixul.o(.text) refers to llushr.o(.text) for __aeabi_llsr
    dfixul.o(.text) refers to llshl.o(.text) for __aeabi_llsl
    init.o(.text) refers to entry5.o(.ARM.Collect$$$$00000004) for __main_after_scatterload
    isspace_c.o(.text) refers to ctype_c.o(.text) for __ctype_lookup
    _scanf.o(.text) refers (Weak) to _scanf_int.o(.text) for _scanf_int
    ctype_c.o(.text) refers to ctype_c.o(.constdata) for .constdata
    user_math.o(i.InvSqrt) refers to fscalb.o(.text) for __ARM_scalbnf
    user_math.o(i.InvSqrt) refers to fmul.o(.text) for __aeabi_fmul
    user_math.o(i.InvSqrt) refers to fadd.o(.text) for __aeabi_frsub
    user_math.o(i.AbsClip) refers to cfrcmple.o(.text) for __aeabi_cfrcmple
    user_math.o(i.Clip) refers to cfrcmple.o(.text) for __aeabi_cfrcmple
    user_math.o(i.Clip) refers to cfcmple.o(.text) for __aeabi_cfcmple
    user_math.o(i.CircleError) refers to fadd.o(.text) for __aeabi_fsub
    user_math.o(i.CircleError) refers to fscalb.o(.text) for __ARM_scalbnf
    user_math.o(i.CircleError) refers to cfrcmple.o(.text) for __aeabi_cfrcmple
    user_math.o(i.CircleAdd) refers to fadd.o(.text) for __aeabi_fadd
    user_math.o(i.CircleAdd) refers to cfrcmple.o(.text) for __aeabi_cfrcmple
    user_math.o(i.CircleReverse) refers to fadd.o(.text) for __aeabi_fsub
    user_math.o(i.CalculateRpm) refers to fmul.o(.text) for __aeabi_fmul
    user_math.o(i.CalculateRpm) refers to fdiv.o(.text) for __aeabi_fdiv


==============================================================================

Removing Unused input sections from the image.

    Removing main.o(.rev16_text), (4 bytes).
    Removing main.o(.revsh_text), (4 bytes).
    Removing main.o(.rrx_text), (6 bytes).
    Removing gpio.o(.rev16_text), (4 bytes).
    Removing gpio.o(.revsh_text), (4 bytes).
    Removing gpio.o(.rrx_text), (6 bytes).
    Removing dma.o(.rev16_text), (4 bytes).
    Removing dma.o(.revsh_text), (4 bytes).
    Removing dma.o(.rrx_text), (6 bytes).
    Removing spi.o(.rev16_text), (4 bytes).
    Removing spi.o(.revsh_text), (4 bytes).
    Removing spi.o(.rrx_text), (6 bytes).
    Removing spi.o(i.HAL_SPI_MspDeInit), (96 bytes).
    Removing tim.o(.rev16_text), (4 bytes).
    Removing tim.o(.revsh_text), (4 bytes).
    Removing tim.o(.rrx_text), (6 bytes).
    Removing tim.o(i.HAL_TIM_Base_MspDeInit), (28 bytes).
    Removing usart.o(.rev16_text), (4 bytes).
    Removing usart.o(.revsh_text), (4 bytes).
    Removing usart.o(.rrx_text), (6 bytes).
    Removing usart.o(i.HAL_UART_MspDeInit), (100 bytes).
    Removing stm32f1xx_it.o(.rev16_text), (4 bytes).
    Removing stm32f1xx_it.o(.revsh_text), (4 bytes).
    Removing stm32f1xx_it.o(.rrx_text), (6 bytes).
    Removing stm32f1xx_hal_msp.o(.rev16_text), (4 bytes).
    Removing stm32f1xx_hal_msp.o(.revsh_text), (4 bytes).
    Removing stm32f1xx_hal_msp.o(.rrx_text), (6 bytes).
    Removing stm32f1xx_hal_gpio_ex.o(.rev16_text), (4 bytes).
    Removing stm32f1xx_hal_gpio_ex.o(.revsh_text), (4 bytes).
    Removing stm32f1xx_hal_gpio_ex.o(.rrx_text), (6 bytes).
    Removing stm32f1xx_hal_gpio_ex.o(i.HAL_GPIOEx_ConfigEventout), (20 bytes).
    Removing stm32f1xx_hal_gpio_ex.o(i.HAL_GPIOEx_DisableEventout), (16 bytes).
    Removing stm32f1xx_hal_gpio_ex.o(i.HAL_GPIOEx_EnableEventout), (16 bytes).
    Removing stm32f1xx_hal_spi.o(.rev16_text), (4 bytes).
    Removing stm32f1xx_hal_spi.o(.revsh_text), (4 bytes).
    Removing stm32f1xx_hal_spi.o(.rrx_text), (6 bytes).
    Removing stm32f1xx_hal_spi.o(i.HAL_SPI_Abort), (288 bytes).
    Removing stm32f1xx_hal_spi.o(i.HAL_SPI_AbortCpltCallback), (2 bytes).
    Removing stm32f1xx_hal_spi.o(i.HAL_SPI_Abort_IT), (288 bytes).
    Removing stm32f1xx_hal_spi.o(i.HAL_SPI_DMAPause), (38 bytes).
    Removing stm32f1xx_hal_spi.o(i.HAL_SPI_DMAResume), (38 bytes).
    Removing stm32f1xx_hal_spi.o(i.HAL_SPI_DMAStop), (66 bytes).
    Removing stm32f1xx_hal_spi.o(i.HAL_SPI_DeInit), (46 bytes).
    Removing stm32f1xx_hal_spi.o(i.HAL_SPI_ErrorCallback), (2 bytes).
    Removing stm32f1xx_hal_spi.o(i.HAL_SPI_GetError), (4 bytes).
    Removing stm32f1xx_hal_spi.o(i.HAL_SPI_IRQHandler), (224 bytes).
    Removing stm32f1xx_hal_spi.o(i.HAL_SPI_MspDeInit), (2 bytes).
    Removing stm32f1xx_hal_spi.o(i.HAL_SPI_MspInit), (2 bytes).
    Removing stm32f1xx_hal_spi.o(i.HAL_SPI_Receive), (340 bytes).
    Removing stm32f1xx_hal_spi.o(i.HAL_SPI_Receive_DMA), (228 bytes).
    Removing stm32f1xx_hal_spi.o(i.HAL_SPI_Receive_IT), (168 bytes).
    Removing stm32f1xx_hal_spi.o(i.HAL_SPI_RxCpltCallback), (2 bytes).
    Removing stm32f1xx_hal_spi.o(i.HAL_SPI_RxHalfCpltCallback), (2 bytes).
    Removing stm32f1xx_hal_spi.o(i.HAL_SPI_TransmitReceive_IT), (156 bytes).
    Removing stm32f1xx_hal_spi.o(i.HAL_SPI_Transmit_IT), (144 bytes).
    Removing stm32f1xx_hal_spi.o(i.HAL_SPI_TxCpltCallback), (2 bytes).
    Removing stm32f1xx_hal_spi.o(i.HAL_SPI_TxHalfCpltCallback), (2 bytes).
    Removing stm32f1xx_hal_spi.o(i.HAL_SPI_TxRxCpltCallback), (2 bytes).
    Removing stm32f1xx_hal_spi.o(i.HAL_SPI_TxRxHalfCpltCallback), (2 bytes).
    Removing stm32f1xx_hal_spi.o(i.SPI_2linesRxISR_16BIT), (48 bytes).
    Removing stm32f1xx_hal_spi.o(i.SPI_2linesRxISR_8BIT), (48 bytes).
    Removing stm32f1xx_hal_spi.o(i.SPI_2linesTxISR_16BIT), (48 bytes).
    Removing stm32f1xx_hal_spi.o(i.SPI_2linesTxISR_8BIT), (48 bytes).
    Removing stm32f1xx_hal_spi.o(i.SPI_AbortRx_ISR), (88 bytes).
    Removing stm32f1xx_hal_spi.o(i.SPI_AbortTx_ISR), (28 bytes).
    Removing stm32f1xx_hal_spi.o(i.SPI_CloseRxTx_ISR), (144 bytes).
    Removing stm32f1xx_hal_spi.o(i.SPI_CloseRx_ISR), (76 bytes).
    Removing stm32f1xx_hal_spi.o(i.SPI_CloseTx_ISR), (124 bytes).
    Removing stm32f1xx_hal_spi.o(i.SPI_DMAAbortOnError), (16 bytes).
    Removing stm32f1xx_hal_spi.o(i.SPI_DMARxAbortCallback), (98 bytes).
    Removing stm32f1xx_hal_spi.o(i.SPI_DMATxAbortCallback), (112 bytes).
    Removing stm32f1xx_hal_spi.o(i.SPI_RxISR_16BIT), (32 bytes).
    Removing stm32f1xx_hal_spi.o(i.SPI_RxISR_8BIT), (32 bytes).
    Removing stm32f1xx_hal_spi.o(i.SPI_TxISR_16BIT), (32 bytes).
    Removing stm32f1xx_hal_spi.o(i.SPI_TxISR_8BIT), (32 bytes).
    Removing stm32f1xx_hal.o(.rev16_text), (4 bytes).
    Removing stm32f1xx_hal.o(.revsh_text), (4 bytes).
    Removing stm32f1xx_hal.o(.rrx_text), (6 bytes).
    Removing stm32f1xx_hal.o(i.HAL_DBGMCU_DisableDBGSleepMode), (16 bytes).
    Removing stm32f1xx_hal.o(i.HAL_DBGMCU_DisableDBGStandbyMode), (16 bytes).
    Removing stm32f1xx_hal.o(i.HAL_DBGMCU_DisableDBGStopMode), (16 bytes).
    Removing stm32f1xx_hal.o(i.HAL_DBGMCU_EnableDBGSleepMode), (16 bytes).
    Removing stm32f1xx_hal.o(i.HAL_DBGMCU_EnableDBGStandbyMode), (16 bytes).
    Removing stm32f1xx_hal.o(i.HAL_DBGMCU_EnableDBGStopMode), (16 bytes).
    Removing stm32f1xx_hal.o(i.HAL_DeInit), (32 bytes).
    Removing stm32f1xx_hal.o(i.HAL_GetDEVID), (16 bytes).
    Removing stm32f1xx_hal.o(i.HAL_GetHalVersion), (8 bytes).
    Removing stm32f1xx_hal.o(i.HAL_GetREVID), (12 bytes).
    Removing stm32f1xx_hal.o(i.HAL_GetTickFreq), (12 bytes).
    Removing stm32f1xx_hal.o(i.HAL_GetTickPrio), (12 bytes).
    Removing stm32f1xx_hal.o(i.HAL_GetUIDw0), (12 bytes).
    Removing stm32f1xx_hal.o(i.HAL_GetUIDw1), (12 bytes).
    Removing stm32f1xx_hal.o(i.HAL_GetUIDw2), (12 bytes).
    Removing stm32f1xx_hal.o(i.HAL_MspDeInit), (2 bytes).
    Removing stm32f1xx_hal.o(i.HAL_MspInit), (2 bytes).
    Removing stm32f1xx_hal.o(i.HAL_ResumeTick), (14 bytes).
    Removing stm32f1xx_hal.o(i.HAL_SetTickFreq), (36 bytes).
    Removing stm32f1xx_hal.o(i.HAL_SuspendTick), (14 bytes).
    Removing stm32f1xx_hal_rcc.o(.rev16_text), (4 bytes).
    Removing stm32f1xx_hal_rcc.o(.revsh_text), (4 bytes).
    Removing stm32f1xx_hal_rcc.o(.rrx_text), (6 bytes).
    Removing stm32f1xx_hal_rcc.o(i.HAL_RCC_CSSCallback), (2 bytes).
    Removing stm32f1xx_hal_rcc.o(i.HAL_RCC_DeInit), (220 bytes).
    Removing stm32f1xx_hal_rcc.o(i.HAL_RCC_DisableCSS), (12 bytes).
    Removing stm32f1xx_hal_rcc.o(i.HAL_RCC_EnableCSS), (12 bytes).
    Removing stm32f1xx_hal_rcc.o(i.HAL_RCC_GetClockConfig), (64 bytes).
    Removing stm32f1xx_hal_rcc.o(i.HAL_RCC_GetHCLKFreq), (12 bytes).
    Removing stm32f1xx_hal_rcc.o(i.HAL_RCC_GetOscConfig), (144 bytes).
    Removing stm32f1xx_hal_rcc.o(i.HAL_RCC_MCOConfig), (72 bytes).
    Removing stm32f1xx_hal_rcc.o(i.HAL_RCC_NMI_IRQHandler), (24 bytes).
    Removing stm32f1xx_hal_rcc_ex.o(.rev16_text), (4 bytes).
    Removing stm32f1xx_hal_rcc_ex.o(.revsh_text), (4 bytes).
    Removing stm32f1xx_hal_rcc_ex.o(.rrx_text), (6 bytes).
    Removing stm32f1xx_hal_rcc_ex.o(i.HAL_RCCEx_GetPeriphCLKConfig), (44 bytes).
    Removing stm32f1xx_hal_rcc_ex.o(i.HAL_RCCEx_GetPeriphCLKFreq), (168 bytes).
    Removing stm32f1xx_hal_rcc_ex.o(i.HAL_RCCEx_PeriphCLKConfig), (236 bytes).
    Removing stm32f1xx_hal_rcc_ex.o(.constdata), (18 bytes).
    Removing stm32f1xx_hal_gpio.o(.rev16_text), (4 bytes).
    Removing stm32f1xx_hal_gpio.o(.revsh_text), (4 bytes).
    Removing stm32f1xx_hal_gpio.o(.rrx_text), (6 bytes).
    Removing stm32f1xx_hal_gpio.o(i.HAL_GPIO_DeInit), (280 bytes).
    Removing stm32f1xx_hal_gpio.o(i.HAL_GPIO_EXTI_Callback), (2 bytes).
    Removing stm32f1xx_hal_gpio.o(i.HAL_GPIO_LockPin), (34 bytes).
    Removing stm32f1xx_hal_gpio.o(i.HAL_GPIO_TogglePin), (16 bytes).
    Removing stm32f1xx_hal_dma.o(.rev16_text), (4 bytes).
    Removing stm32f1xx_hal_dma.o(.revsh_text), (4 bytes).
    Removing stm32f1xx_hal_dma.o(.rrx_text), (6 bytes).
    Removing stm32f1xx_hal_dma.o(i.HAL_DMA_DeInit), (92 bytes).
    Removing stm32f1xx_hal_dma.o(i.HAL_DMA_GetError), (4 bytes).
    Removing stm32f1xx_hal_dma.o(i.HAL_DMA_GetState), (6 bytes).
    Removing stm32f1xx_hal_dma.o(i.HAL_DMA_PollForTransfer), (532 bytes).
    Removing stm32f1xx_hal_dma.o(i.HAL_DMA_RegisterCallback), (74 bytes).
    Removing stm32f1xx_hal_dma.o(i.HAL_DMA_Start), (80 bytes).
    Removing stm32f1xx_hal_dma.o(i.HAL_DMA_UnRegisterCallback), (82 bytes).
    Removing stm32f1xx_hal_cortex.o(.rev16_text), (4 bytes).
    Removing stm32f1xx_hal_cortex.o(.revsh_text), (4 bytes).
    Removing stm32f1xx_hal_cortex.o(.rrx_text), (6 bytes).
    Removing stm32f1xx_hal_cortex.o(i.HAL_NVIC_ClearPendingIRQ), (26 bytes).
    Removing stm32f1xx_hal_cortex.o(i.HAL_NVIC_DisableIRQ), (34 bytes).
    Removing stm32f1xx_hal_cortex.o(i.HAL_NVIC_GetActive), (36 bytes).
    Removing stm32f1xx_hal_cortex.o(i.HAL_NVIC_GetPendingIRQ), (36 bytes).
    Removing stm32f1xx_hal_cortex.o(i.HAL_NVIC_GetPriority), (82 bytes).
    Removing stm32f1xx_hal_cortex.o(i.HAL_NVIC_GetPriorityGrouping), (16 bytes).
    Removing stm32f1xx_hal_cortex.o(i.HAL_NVIC_SetPendingIRQ), (26 bytes).
    Removing stm32f1xx_hal_cortex.o(i.HAL_NVIC_SystemReset), (36 bytes).
    Removing stm32f1xx_hal_cortex.o(i.HAL_SYSTICK_CLKSourceConfig), (24 bytes).
    Removing stm32f1xx_hal_cortex.o(i.HAL_SYSTICK_Callback), (2 bytes).
    Removing stm32f1xx_hal_cortex.o(i.HAL_SYSTICK_IRQHandler), (8 bytes).
    Removing stm32f1xx_hal_pwr.o(.rev16_text), (4 bytes).
    Removing stm32f1xx_hal_pwr.o(.revsh_text), (4 bytes).
    Removing stm32f1xx_hal_pwr.o(.rrx_text), (6 bytes).
    Removing stm32f1xx_hal_pwr.o(i.HAL_PWR_ConfigPVD), (124 bytes).
    Removing stm32f1xx_hal_pwr.o(i.HAL_PWR_DeInit), (24 bytes).
    Removing stm32f1xx_hal_pwr.o(i.HAL_PWR_DisableBkUpAccess), (12 bytes).
    Removing stm32f1xx_hal_pwr.o(i.HAL_PWR_DisablePVD), (12 bytes).
    Removing stm32f1xx_hal_pwr.o(i.HAL_PWR_DisableSEVOnPend), (16 bytes).
    Removing stm32f1xx_hal_pwr.o(i.HAL_PWR_DisableSleepOnExit), (16 bytes).
    Removing stm32f1xx_hal_pwr.o(i.HAL_PWR_DisableWakeUpPin), (28 bytes).
    Removing stm32f1xx_hal_pwr.o(i.HAL_PWR_EnableBkUpAccess), (12 bytes).
    Removing stm32f1xx_hal_pwr.o(i.HAL_PWR_EnablePVD), (12 bytes).
    Removing stm32f1xx_hal_pwr.o(i.HAL_PWR_EnableSEVOnPend), (16 bytes).
    Removing stm32f1xx_hal_pwr.o(i.HAL_PWR_EnableSleepOnExit), (16 bytes).
    Removing stm32f1xx_hal_pwr.o(i.HAL_PWR_EnableWakeUpPin), (28 bytes).
    Removing stm32f1xx_hal_pwr.o(i.HAL_PWR_EnterSLEEPMode), (32 bytes).
    Removing stm32f1xx_hal_pwr.o(i.HAL_PWR_EnterSTANDBYMode), (32 bytes).
    Removing stm32f1xx_hal_pwr.o(i.HAL_PWR_EnterSTOPMode), (68 bytes).
    Removing stm32f1xx_hal_pwr.o(i.HAL_PWR_PVDCallback), (2 bytes).
    Removing stm32f1xx_hal_pwr.o(i.HAL_PWR_PVD_IRQHandler), (28 bytes).
    Removing stm32f1xx_hal_pwr.o(i.PWR_OverloadWfe), (6 bytes).
    Removing stm32f1xx_hal_flash.o(.rev16_text), (4 bytes).
    Removing stm32f1xx_hal_flash.o(.revsh_text), (4 bytes).
    Removing stm32f1xx_hal_flash.o(.rrx_text), (6 bytes).
    Removing stm32f1xx_hal_flash.o(i.FLASH_Program_HalfWord), (28 bytes).
    Removing stm32f1xx_hal_flash.o(i.FLASH_SetErrorCode), (92 bytes).
    Removing stm32f1xx_hal_flash.o(i.FLASH_WaitForLastOperation), (84 bytes).
    Removing stm32f1xx_hal_flash.o(i.HAL_FLASH_EndOfOperationCallback), (2 bytes).
    Removing stm32f1xx_hal_flash.o(i.HAL_FLASH_GetError), (12 bytes).
    Removing stm32f1xx_hal_flash.o(i.HAL_FLASH_IRQHandler), (264 bytes).
    Removing stm32f1xx_hal_flash.o(i.HAL_FLASH_Lock), (20 bytes).
    Removing stm32f1xx_hal_flash.o(i.HAL_FLASH_OB_Launch), (4 bytes).
    Removing stm32f1xx_hal_flash.o(i.HAL_FLASH_OB_Lock), (20 bytes).
    Removing stm32f1xx_hal_flash.o(i.HAL_FLASH_OB_Unlock), (36 bytes).
    Removing stm32f1xx_hal_flash.o(i.HAL_FLASH_OperationErrorCallback), (2 bytes).
    Removing stm32f1xx_hal_flash.o(i.HAL_FLASH_Program), (128 bytes).
    Removing stm32f1xx_hal_flash.o(i.HAL_FLASH_Program_IT), (80 bytes).
    Removing stm32f1xx_hal_flash.o(i.HAL_FLASH_Unlock), (40 bytes).
    Removing stm32f1xx_hal_flash.o(.bss), (32 bytes).
    Removing stm32f1xx_hal_flash_ex.o(.rev16_text), (4 bytes).
    Removing stm32f1xx_hal_flash_ex.o(.revsh_text), (4 bytes).
    Removing stm32f1xx_hal_flash_ex.o(.rrx_text), (6 bytes).
    Removing stm32f1xx_hal_flash_ex.o(i.FLASH_MassErase), (36 bytes).
    Removing stm32f1xx_hal_flash_ex.o(i.FLASH_OB_DisableWRP), (176 bytes).
    Removing stm32f1xx_hal_flash_ex.o(i.FLASH_OB_EnableWRP), (176 bytes).
    Removing stm32f1xx_hal_flash_ex.o(i.FLASH_OB_GetRDP), (24 bytes).
    Removing stm32f1xx_hal_flash_ex.o(i.FLASH_OB_RDP_LevelConfig), (100 bytes).
    Removing stm32f1xx_hal_flash_ex.o(i.FLASH_PageErase), (36 bytes).
    Removing stm32f1xx_hal_flash_ex.o(i.HAL_FLASHEx_Erase), (168 bytes).
    Removing stm32f1xx_hal_flash_ex.o(i.HAL_FLASHEx_Erase_IT), (72 bytes).
    Removing stm32f1xx_hal_flash_ex.o(i.HAL_FLASHEx_OBErase), (84 bytes).
    Removing stm32f1xx_hal_flash_ex.o(i.HAL_FLASHEx_OBGetConfig), (36 bytes).
    Removing stm32f1xx_hal_flash_ex.o(i.HAL_FLASHEx_OBGetUserData), (32 bytes).
    Removing stm32f1xx_hal_flash_ex.o(i.HAL_FLASHEx_OBProgram), (200 bytes).
    Removing stm32f1xx_hal_exti.o(.rev16_text), (4 bytes).
    Removing stm32f1xx_hal_exti.o(.revsh_text), (4 bytes).
    Removing stm32f1xx_hal_exti.o(.rrx_text), (6 bytes).
    Removing stm32f1xx_hal_exti.o(i.HAL_EXTI_ClearConfigLine), (104 bytes).
    Removing stm32f1xx_hal_exti.o(i.HAL_EXTI_ClearPending), (20 bytes).
    Removing stm32f1xx_hal_exti.o(i.HAL_EXTI_GenerateSWI), (20 bytes).
    Removing stm32f1xx_hal_exti.o(i.HAL_EXTI_GetConfigLine), (140 bytes).
    Removing stm32f1xx_hal_exti.o(i.HAL_EXTI_GetHandle), (12 bytes).
    Removing stm32f1xx_hal_exti.o(i.HAL_EXTI_GetPending), (24 bytes).
    Removing stm32f1xx_hal_exti.o(i.HAL_EXTI_IRQHandler), (36 bytes).
    Removing stm32f1xx_hal_exti.o(i.HAL_EXTI_RegisterCallback), (14 bytes).
    Removing stm32f1xx_hal_exti.o(i.HAL_EXTI_SetConfigLine), (164 bytes).
    Removing stm32f1xx_hal_tim.o(.rev16_text), (4 bytes).
    Removing stm32f1xx_hal_tim.o(.revsh_text), (4 bytes).
    Removing stm32f1xx_hal_tim.o(.rrx_text), (6 bytes).
    Removing stm32f1xx_hal_tim.o(i.HAL_TIM_Base_DeInit), (92 bytes).
    Removing stm32f1xx_hal_tim.o(i.HAL_TIM_Base_GetState), (6 bytes).
    Removing stm32f1xx_hal_tim.o(i.HAL_TIM_Base_MspDeInit), (2 bytes).
    Removing stm32f1xx_hal_tim.o(i.HAL_TIM_Base_MspInit), (2 bytes).
    Removing stm32f1xx_hal_tim.o(i.HAL_TIM_Base_Start), (80 bytes).
    Removing stm32f1xx_hal_tim.o(i.HAL_TIM_Base_Start_DMA), (152 bytes).
    Removing stm32f1xx_hal_tim.o(i.HAL_TIM_Base_Start_IT), (88 bytes).
    Removing stm32f1xx_hal_tim.o(i.HAL_TIM_Base_Stop), (38 bytes).
    Removing stm32f1xx_hal_tim.o(i.HAL_TIM_Base_Stop_DMA), (58 bytes).
    Removing stm32f1xx_hal_tim.o(i.HAL_TIM_Base_Stop_IT), (48 bytes).
    Removing stm32f1xx_hal_tim.o(i.HAL_TIM_ConfigOCrefClear), (216 bytes).
    Removing stm32f1xx_hal_tim.o(i.HAL_TIM_ConfigTI1Input), (16 bytes).
    Removing stm32f1xx_hal_tim.o(i.HAL_TIM_DMABurstState), (6 bytes).
    Removing stm32f1xx_hal_tim.o(i.HAL_TIM_DMABurst_MultiReadStart), (332 bytes).
    Removing stm32f1xx_hal_tim.o(i.HAL_TIM_DMABurst_MultiWriteStart), (332 bytes).
    Removing stm32f1xx_hal_tim.o(i.HAL_TIM_DMABurst_ReadStart), (18 bytes).
    Removing stm32f1xx_hal_tim.o(i.HAL_TIM_DMABurst_ReadStop), (106 bytes).
    Removing stm32f1xx_hal_tim.o(i.HAL_TIM_DMABurst_WriteStart), (18 bytes).
    Removing stm32f1xx_hal_tim.o(i.HAL_TIM_DMABurst_WriteStop), (106 bytes).
    Removing stm32f1xx_hal_tim.o(i.HAL_TIM_Encoder_DeInit), (76 bytes).
    Removing stm32f1xx_hal_tim.o(i.HAL_TIM_Encoder_GetState), (6 bytes).
    Removing stm32f1xx_hal_tim.o(i.HAL_TIM_Encoder_Init), (164 bytes).
    Removing stm32f1xx_hal_tim.o(i.HAL_TIM_Encoder_MspDeInit), (2 bytes).
    Removing stm32f1xx_hal_tim.o(i.HAL_TIM_Encoder_MspInit), (2 bytes).
    Removing stm32f1xx_hal_tim.o(i.HAL_TIM_Encoder_Start), (142 bytes).
    Removing stm32f1xx_hal_tim.o(i.HAL_TIM_Encoder_Start_DMA), (428 bytes).
    Removing stm32f1xx_hal_tim.o(i.HAL_TIM_Encoder_Start_IT), (182 bytes).
    Removing stm32f1xx_hal_tim.o(i.HAL_TIM_Encoder_Stop), (102 bytes).
    Removing stm32f1xx_hal_tim.o(i.HAL_TIM_Encoder_Stop_DMA), (172 bytes).
    Removing stm32f1xx_hal_tim.o(i.HAL_TIM_Encoder_Stop_IT), (144 bytes).
    Removing stm32f1xx_hal_tim.o(i.HAL_TIM_ErrorCallback), (2 bytes).
    Removing stm32f1xx_hal_tim.o(i.HAL_TIM_GenerateEvent), (38 bytes).
    Removing stm32f1xx_hal_tim.o(i.HAL_TIM_GetActiveChannel), (4 bytes).
    Removing stm32f1xx_hal_tim.o(i.HAL_TIM_GetChannelState), (34 bytes).
    Removing stm32f1xx_hal_tim.o(i.HAL_TIM_IC_CaptureCallback), (2 bytes).
    Removing stm32f1xx_hal_tim.o(i.HAL_TIM_IC_CaptureHalfCpltCallback), (2 bytes).
    Removing stm32f1xx_hal_tim.o(i.HAL_TIM_IC_ConfigChannel), (292 bytes).
    Removing stm32f1xx_hal_tim.o(i.HAL_TIM_IC_DeInit), (92 bytes).
    Removing stm32f1xx_hal_tim.o(i.HAL_TIM_IC_GetState), (6 bytes).
    Removing stm32f1xx_hal_tim.o(i.HAL_TIM_IC_Init), (90 bytes).
    Removing stm32f1xx_hal_tim.o(i.HAL_TIM_IC_MspDeInit), (2 bytes).
    Removing stm32f1xx_hal_tim.o(i.HAL_TIM_IC_MspInit), (2 bytes).
    Removing stm32f1xx_hal_tim.o(i.HAL_TIM_IC_Start), (184 bytes).
    Removing stm32f1xx_hal_tim.o(i.HAL_TIM_IC_Start_DMA), (416 bytes).
    Removing stm32f1xx_hal_tim.o(i.HAL_TIM_IC_Start_IT), (228 bytes).
    Removing stm32f1xx_hal_tim.o(i.HAL_TIM_IC_Stop), (82 bytes).
    Removing stm32f1xx_hal_tim.o(i.HAL_TIM_IC_Stop_DMA), (160 bytes).
    Removing stm32f1xx_hal_tim.o(i.HAL_TIM_IC_Stop_IT), (146 bytes).
    Removing stm32f1xx_hal_tim.o(i.HAL_TIM_IRQHandler), (304 bytes).
    Removing stm32f1xx_hal_tim.o(i.HAL_TIM_OC_ConfigChannel), (82 bytes).
    Removing stm32f1xx_hal_tim.o(i.HAL_TIM_OC_DeInit), (92 bytes).
    Removing stm32f1xx_hal_tim.o(i.HAL_TIM_OC_DelayElapsedCallback), (2 bytes).
    Removing stm32f1xx_hal_tim.o(i.HAL_TIM_OC_GetState), (6 bytes).
    Removing stm32f1xx_hal_tim.o(i.HAL_TIM_OC_Init), (90 bytes).
    Removing stm32f1xx_hal_tim.o(i.HAL_TIM_OC_MspDeInit), (2 bytes).
    Removing stm32f1xx_hal_tim.o(i.HAL_TIM_OC_MspInit), (2 bytes).
    Removing stm32f1xx_hal_tim.o(i.HAL_TIM_OC_Start), (156 bytes).
    Removing stm32f1xx_hal_tim.o(i.HAL_TIM_OC_Start_DMA), (404 bytes).
    Removing stm32f1xx_hal_tim.o(i.HAL_TIM_OC_Start_IT), (200 bytes).
    Removing stm32f1xx_hal_tim.o(i.HAL_TIM_OC_Stop), (112 bytes).
    Removing stm32f1xx_hal_tim.o(i.HAL_TIM_OC_Stop_DMA), (196 bytes).
    Removing stm32f1xx_hal_tim.o(i.HAL_TIM_OC_Stop_IT), (176 bytes).
    Removing stm32f1xx_hal_tim.o(i.HAL_TIM_OnePulse_ConfigChannel), (230 bytes).
    Removing stm32f1xx_hal_tim.o(i.HAL_TIM_OnePulse_DeInit), (76 bytes).
    Removing stm32f1xx_hal_tim.o(i.HAL_TIM_OnePulse_GetState), (6 bytes).
    Removing stm32f1xx_hal_tim.o(i.HAL_TIM_OnePulse_Init), (86 bytes).
    Removing stm32f1xx_hal_tim.o(i.HAL_TIM_OnePulse_MspDeInit), (2 bytes).
    Removing stm32f1xx_hal_tim.o(i.HAL_TIM_OnePulse_MspInit), (2 bytes).
    Removing stm32f1xx_hal_tim.o(i.HAL_TIM_OnePulse_Start), (104 bytes).
    Removing stm32f1xx_hal_tim.o(i.HAL_TIM_OnePulse_Start_IT), (124 bytes).
    Removing stm32f1xx_hal_tim.o(i.HAL_TIM_OnePulse_Stop), (100 bytes).
    Removing stm32f1xx_hal_tim.o(i.HAL_TIM_OnePulse_Stop_IT), (120 bytes).
    Removing stm32f1xx_hal_tim.o(i.HAL_TIM_PWM_DeInit), (92 bytes).
    Removing stm32f1xx_hal_tim.o(i.HAL_TIM_PWM_GetState), (6 bytes).
    Removing stm32f1xx_hal_tim.o(i.HAL_TIM_PWM_MspDeInit), (2 bytes).
    Removing stm32f1xx_hal_tim.o(i.HAL_TIM_PWM_PulseFinishedCallback), (2 bytes).
    Removing stm32f1xx_hal_tim.o(i.HAL_TIM_PWM_PulseFinishedHalfCpltCallback), (2 bytes).
    Removing stm32f1xx_hal_tim.o(i.HAL_TIM_PWM_Start), (156 bytes).
    Removing stm32f1xx_hal_tim.o(i.HAL_TIM_PWM_Start_DMA), (404 bytes).
    Removing stm32f1xx_hal_tim.o(i.HAL_TIM_PWM_Start_IT), (200 bytes).
    Removing stm32f1xx_hal_tim.o(i.HAL_TIM_PWM_Stop), (112 bytes).
    Removing stm32f1xx_hal_tim.o(i.HAL_TIM_PWM_Stop_DMA), (196 bytes).
    Removing stm32f1xx_hal_tim.o(i.HAL_TIM_PWM_Stop_IT), (176 bytes).
    Removing stm32f1xx_hal_tim.o(i.HAL_TIM_PeriodElapsedCallback), (2 bytes).
    Removing stm32f1xx_hal_tim.o(i.HAL_TIM_PeriodElapsedHalfCpltCallback), (2 bytes).
    Removing stm32f1xx_hal_tim.o(i.HAL_TIM_ReadCapturedValue), (42 bytes).
    Removing stm32f1xx_hal_tim.o(i.HAL_TIM_SlaveConfigSynchro), (86 bytes).
    Removing stm32f1xx_hal_tim.o(i.HAL_TIM_SlaveConfigSynchro_IT), (86 bytes).
    Removing stm32f1xx_hal_tim.o(i.HAL_TIM_TriggerCallback), (2 bytes).
    Removing stm32f1xx_hal_tim.o(i.HAL_TIM_TriggerHalfCpltCallback), (2 bytes).
    Removing stm32f1xx_hal_tim.o(i.TIM_CCxChannelCmd), (26 bytes).
    Removing stm32f1xx_hal_tim.o(i.TIM_DMACaptureCplt), (110 bytes).
    Removing stm32f1xx_hal_tim.o(i.TIM_DMACaptureHalfCplt), (56 bytes).
    Removing stm32f1xx_hal_tim.o(i.TIM_DMADelayPulseCplt), (94 bytes).
    Removing stm32f1xx_hal_tim.o(i.TIM_DMADelayPulseHalfCplt), (56 bytes).
    Removing stm32f1xx_hal_tim.o(i.TIM_DMAError), (84 bytes).
    Removing stm32f1xx_hal_tim.o(i.TIM_DMAPeriodElapsedCplt), (22 bytes).
    Removing stm32f1xx_hal_tim.o(i.TIM_DMAPeriodElapsedHalfCplt), (10 bytes).
    Removing stm32f1xx_hal_tim.o(i.TIM_DMATriggerCplt), (22 bytes).
    Removing stm32f1xx_hal_tim.o(i.TIM_DMATriggerHalfCplt), (10 bytes).
    Removing stm32f1xx_hal_tim.o(i.TIM_SlaveTimer_SetConfig), (140 bytes).
    Removing stm32f1xx_hal_tim.o(i.TIM_TI1_SetConfig), (88 bytes).
    Removing stm32f1xx_hal_tim.o(i.TIM_TI2_SetConfig), (54 bytes).
    Removing stm32f1xx_hal_tim_ex.o(.rev16_text), (4 bytes).
    Removing stm32f1xx_hal_tim_ex.o(.revsh_text), (4 bytes).
    Removing stm32f1xx_hal_tim_ex.o(.rrx_text), (6 bytes).
    Removing stm32f1xx_hal_tim_ex.o(i.HAL_TIMEx_BreakCallback), (2 bytes).
    Removing stm32f1xx_hal_tim_ex.o(i.HAL_TIMEx_CommutCallback), (2 bytes).
    Removing stm32f1xx_hal_tim_ex.o(i.HAL_TIMEx_CommutHalfCpltCallback), (2 bytes).
    Removing stm32f1xx_hal_tim_ex.o(i.HAL_TIMEx_ConfigCommutEvent), (112 bytes).
    Removing stm32f1xx_hal_tim_ex.o(i.HAL_TIMEx_ConfigCommutEvent_DMA), (144 bytes).
    Removing stm32f1xx_hal_tim_ex.o(i.HAL_TIMEx_ConfigCommutEvent_IT), (112 bytes).
    Removing stm32f1xx_hal_tim_ex.o(i.HAL_TIMEx_GetChannelNState), (34 bytes).
    Removing stm32f1xx_hal_tim_ex.o(i.HAL_TIMEx_HallSensor_DeInit), (76 bytes).
    Removing stm32f1xx_hal_tim_ex.o(i.HAL_TIMEx_HallSensor_GetState), (6 bytes).
    Removing stm32f1xx_hal_tim_ex.o(i.HAL_TIMEx_HallSensor_Init), (208 bytes).
    Removing stm32f1xx_hal_tim_ex.o(i.HAL_TIMEx_HallSensor_MspDeInit), (2 bytes).
    Removing stm32f1xx_hal_tim_ex.o(i.HAL_TIMEx_HallSensor_MspInit), (2 bytes).
    Removing stm32f1xx_hal_tim_ex.o(i.HAL_TIMEx_HallSensor_Start), (128 bytes).
    Removing stm32f1xx_hal_tim_ex.o(i.HAL_TIMEx_HallSensor_Start_DMA), (184 bytes).
    Removing stm32f1xx_hal_tim_ex.o(i.HAL_TIMEx_HallSensor_Start_IT), (140 bytes).
    Removing stm32f1xx_hal_tim_ex.o(i.HAL_TIMEx_HallSensor_Stop), (58 bytes).
    Removing stm32f1xx_hal_tim_ex.o(i.HAL_TIMEx_HallSensor_Stop_DMA), (70 bytes).
    Removing stm32f1xx_hal_tim_ex.o(i.HAL_TIMEx_HallSensor_Stop_IT), (68 bytes).
    Removing stm32f1xx_hal_tim_ex.o(i.HAL_TIMEx_OCN_Start), (152 bytes).
    Removing stm32f1xx_hal_tim_ex.o(i.HAL_TIMEx_OCN_Start_DMA), (352 bytes).
    Removing stm32f1xx_hal_tim_ex.o(i.HAL_TIMEx_OCN_Start_IT), (192 bytes).
    Removing stm32f1xx_hal_tim_ex.o(i.HAL_TIMEx_OCN_Stop), (104 bytes).
    Removing stm32f1xx_hal_tim_ex.o(i.HAL_TIMEx_OCN_Stop_DMA), (168 bytes).
    Removing stm32f1xx_hal_tim_ex.o(i.HAL_TIMEx_OCN_Stop_IT), (170 bytes).
    Removing stm32f1xx_hal_tim_ex.o(i.HAL_TIMEx_OnePulseN_Start), (100 bytes).
    Removing stm32f1xx_hal_tim_ex.o(i.HAL_TIMEx_OnePulseN_Start_IT), (120 bytes).
    Removing stm32f1xx_hal_tim_ex.o(i.HAL_TIMEx_OnePulseN_Stop), (98 bytes).
    Removing stm32f1xx_hal_tim_ex.o(i.HAL_TIMEx_OnePulseN_Stop_IT), (120 bytes).
    Removing stm32f1xx_hal_tim_ex.o(i.HAL_TIMEx_PWMN_Start), (152 bytes).
    Removing stm32f1xx_hal_tim_ex.o(i.HAL_TIMEx_PWMN_Start_DMA), (352 bytes).
    Removing stm32f1xx_hal_tim_ex.o(i.HAL_TIMEx_PWMN_Start_IT), (192 bytes).
    Removing stm32f1xx_hal_tim_ex.o(i.HAL_TIMEx_PWMN_Stop), (104 bytes).
    Removing stm32f1xx_hal_tim_ex.o(i.HAL_TIMEx_PWMN_Stop_DMA), (168 bytes).
    Removing stm32f1xx_hal_tim_ex.o(i.HAL_TIMEx_PWMN_Stop_IT), (170 bytes).
    Removing stm32f1xx_hal_tim_ex.o(i.HAL_TIMEx_RemapConfig), (4 bytes).
    Removing stm32f1xx_hal_tim_ex.o(i.TIMEx_DMACommutationCplt), (16 bytes).
    Removing stm32f1xx_hal_tim_ex.o(i.TIMEx_DMACommutationHalfCplt), (16 bytes).
    Removing stm32f1xx_hal_tim_ex.o(i.TIM_CCxNChannelCmd), (26 bytes).
    Removing stm32f1xx_hal_tim_ex.o(i.TIM_DMADelayPulseNCplt), (74 bytes).
    Removing stm32f1xx_hal_tim_ex.o(i.TIM_DMAErrorCCxN), (62 bytes).
    Removing stm32f1xx_hal_uart.o(.rev16_text), (4 bytes).
    Removing stm32f1xx_hal_uart.o(.revsh_text), (4 bytes).
    Removing stm32f1xx_hal_uart.o(.rrx_text), (6 bytes).
    Removing stm32f1xx_hal_uart.o(i.HAL_HalfDuplex_EnableReceiver), (50 bytes).
    Removing stm32f1xx_hal_uart.o(i.HAL_HalfDuplex_EnableTransmitter), (50 bytes).
    Removing stm32f1xx_hal_uart.o(i.HAL_LIN_Init), (130 bytes).
    Removing stm32f1xx_hal_uart.o(i.HAL_LIN_SendBreak), (60 bytes).
    Removing stm32f1xx_hal_uart.o(i.HAL_MultiProcessor_EnterMuteMode), (62 bytes).
    Removing stm32f1xx_hal_uart.o(i.HAL_MultiProcessor_ExitMuteMode), (62 bytes).
    Removing stm32f1xx_hal_uart.o(i.HAL_MultiProcessor_Init), (144 bytes).
    Removing stm32f1xx_hal_uart.o(i.HAL_UARTEx_GetRxEventType), (4 bytes).
    Removing stm32f1xx_hal_uart.o(i.HAL_UARTEx_ReceiveToIdle), (240 bytes).
    Removing stm32f1xx_hal_uart.o(i.HAL_UARTEx_ReceiveToIdle_DMA), (74 bytes).
    Removing stm32f1xx_hal_uart.o(i.HAL_UARTEx_ReceiveToIdle_IT), (78 bytes).
    Removing stm32f1xx_hal_uart.o(i.HAL_UART_Abort), (210 bytes).
    Removing stm32f1xx_hal_uart.o(i.HAL_UART_AbortCpltCallback), (2 bytes).
    Removing stm32f1xx_hal_uart.o(i.HAL_UART_AbortReceive), (148 bytes).
    Removing stm32f1xx_hal_uart.o(i.HAL_UART_AbortReceiveCpltCallback), (2 bytes).
    Removing stm32f1xx_hal_uart.o(i.HAL_UART_AbortReceive_IT), (152 bytes).
    Removing stm32f1xx_hal_uart.o(i.HAL_UART_AbortTransmit), (98 bytes).
    Removing stm32f1xx_hal_uart.o(i.HAL_UART_AbortTransmitCpltCallback), (2 bytes).
    Removing stm32f1xx_hal_uart.o(i.HAL_UART_AbortTransmit_IT), (104 bytes).
    Removing stm32f1xx_hal_uart.o(i.HAL_UART_Abort_IT), (244 bytes).
    Removing stm32f1xx_hal_uart.o(i.HAL_UART_DMAPause), (120 bytes).
    Removing stm32f1xx_hal_uart.o(i.HAL_UART_DMAResume), (114 bytes).
    Removing stm32f1xx_hal_uart.o(i.HAL_UART_DeInit), (54 bytes).
    Removing stm32f1xx_hal_uart.o(i.HAL_UART_ErrorCallback), (2 bytes).
    Removing stm32f1xx_hal_uart.o(i.HAL_UART_GetError), (4 bytes).
    Removing stm32f1xx_hal_uart.o(i.HAL_UART_GetState), (10 bytes).
    Removing stm32f1xx_hal_uart.o(i.HAL_UART_MspDeInit), (2 bytes).
    Removing stm32f1xx_hal_uart.o(i.HAL_UART_MspInit), (2 bytes).
    Removing stm32f1xx_hal_uart.o(i.HAL_UART_Receive), (176 bytes).
    Removing stm32f1xx_hal_uart.o(i.HAL_UART_Receive_IT), (28 bytes).
    Removing stm32f1xx_hal_uart.o(i.HAL_UART_RxCpltCallback), (2 bytes).
    Removing stm32f1xx_hal_uart.o(i.HAL_UART_RxHalfCpltCallback), (2 bytes).
    Removing stm32f1xx_hal_uart.o(i.HAL_UART_Transmit_DMA), (120 bytes).
    Removing stm32f1xx_hal_uart.o(i.HAL_UART_Transmit_IT), (50 bytes).
    Removing stm32f1xx_hal_uart.o(i.HAL_UART_TxCpltCallback), (2 bytes).
    Removing stm32f1xx_hal_uart.o(i.HAL_UART_TxHalfCpltCallback), (2 bytes).
    Removing stm32f1xx_hal_uart.o(i.UART_DMARxAbortCallback), (44 bytes).
    Removing stm32f1xx_hal_uart.o(i.UART_DMARxOnlyAbortCallback), (22 bytes).
    Removing stm32f1xx_hal_uart.o(i.UART_DMATransmitCplt), (66 bytes).
    Removing stm32f1xx_hal_uart.o(i.UART_DMATxAbortCallback), (44 bytes).
    Removing stm32f1xx_hal_uart.o(i.UART_DMATxHalfCplt), (10 bytes).
    Removing stm32f1xx_hal_uart.o(i.UART_DMATxOnlyAbortCallback), (20 bytes).
    Removing stm32f1xx_hal_uart.o(i.UART_Start_Receive_IT), (54 bytes).
    Removing system_stm32f1xx.o(.rev16_text), (4 bytes).
    Removing system_stm32f1xx.o(.revsh_text), (4 bytes).
    Removing system_stm32f1xx.o(.rrx_text), (6 bytes).
    Removing system_stm32f1xx.o(i.SystemCoreClockUpdate), (116 bytes).
    Removing sx1281.o(.rev16_text), (4 bytes).
    Removing sx1281.o(.revsh_text), (4 bytes).
    Removing sx1281.o(.rrx_text), (6 bytes).
    Removing sx1281.o(i.OnCadDone), (20 bytes).
    Removing sx1281.o(i.SX1281_SetBLEBaudrate), (76 bytes).
    Removing sx1281.o(i.SX1281_SetFLRCBaudrate), (76 bytes).
    Removing sx1281.o(i.SX1281_SetGFSKBaudrate), (76 bytes).
    Removing sx1281.o(i.SX1281_SetLORABaudrate), (76 bytes).
    Removing sx1281.o(i.SX1281_SetMode), (116 bytes).
    Removing sx1281.o(i.SX1281_SetPacketConfig), (28 bytes).
    Removing sx1281.o(i.SX1281_SetRFFrequency), (48 bytes).
    Removing sx1281.o(i.SX1281_SetRXSingle), (44 bytes).
    Removing sx1281.o(i.SX1281_SetRXSuccessive), (44 bytes).
    Removing sx1281.o(i.SX1281_SetSleep), (12 bytes).
    Removing sx1281.o(i.SetBLEAdvertisingPacket), (2 bytes).
    Removing sx1281.o(.data), (2 bytes).
    Removing sx1281_driver.o(.rev16_text), (4 bytes).
    Removing sx1281_driver.o(.revsh_text), (4 bytes).
    Removing sx1281_driver.o(.rrx_text), (6 bytes).
    Removing sx1281_driver.o(i.SX1281GetHexFileLineFields), (236 bytes).
    Removing sx1281_driver.o(i.SX1281ParseHexFileLine), (48 bytes).
    Removing sx1281_driver_gpio.o(.rev16_text), (4 bytes).
    Removing sx1281_driver_gpio.o(.revsh_text), (4 bytes).
    Removing sx1281_driver_gpio.o(.rrx_text), (6 bytes).
    Removing sx1281_driver_gpio.o(i.GpioDeInit), (2 bytes).
    Removing sx1281_driver_gpio.o(i.GpioLaunchIrqHandler), (28 bytes).
    Removing sx1281_driver_hal.o(.rev16_text), (4 bytes).
    Removing sx1281_driver_hal.o(.revsh_text), (4 bytes).
    Removing sx1281_driver_hal.o(.rrx_text), (6 bytes).
    Removing sx1281_driver_hal.o(i.SX120HalWakeup), (60 bytes).
    Removing sx1281_driver_hal.o(i.SX1281HalClearInstructionRam), (88 bytes).
    Removing sx1281_driver_spi.o(.rev16_text), (4 bytes).
    Removing sx1281_driver_spi.o(.revsh_text), (4 bytes).
    Removing sx1281_driver_spi.o(.rrx_text), (6 bytes).
    Removing sx1281_driver_spi.o(i.SpiDeInit), (2 bytes).
    Removing sx1281_driver_uart.o(.rev16_text), (4 bytes).
    Removing sx1281_driver_uart.o(.revsh_text), (4 bytes).
    Removing sx1281_driver_uart.o(.rrx_text), (6 bytes).
    Removing sx1281_header.o(.rev16_text), (4 bytes).
    Removing sx1281_header.o(.revsh_text), (4 bytes).
    Removing sx1281_header.o(.rrx_text), (6 bytes).
    Removing sx1281_header.o(i.HwSetLowPower), (2 bytes).
    Removing gpio_1.o(.rev16_text), (4 bytes).
    Removing gpio_1.o(.revsh_text), (4 bytes).
    Removing gpio_1.o(.rrx_text), (6 bytes).
    Removing gpio_1.o(i.BSP_GPIO_DisableIRQ), (36 bytes).
    Removing gpio_1.o(i.BSP_GPIO_EnableIRQ), (36 bytes).
    Removing gpio_1.o(i.BSP_GPIO_ReadPin), (36 bytes).
    Removing gpio_1.o(i.BSP_GPIO_RegisterCallback), (68 bytes).
    Removing gpio_1.o(i.BSP_GPIO_TogglePin), (36 bytes).
    Removing gpio_1.o(i.BSP_GPIO_WritePin), (40 bytes).
    Removing gpio_1.o(.constdata), (72 bytes).
    Removing spi_1.o(.rev16_text), (4 bytes).
    Removing spi_1.o(.revsh_text), (4 bytes).
    Removing spi_1.o(.rrx_text), (6 bytes).
    Removing spi_1.o(i.BSP_SPI_MemRead), (68 bytes).
    Removing spi_1.o(i.BSP_SPI_MemReadByte), (42 bytes).
    Removing spi_1.o(i.BSP_SPI_MemWrite), (68 bytes).
    Removing spi_1.o(i.BSP_SPI_MemWriteByte), (36 bytes).
    Removing spi_1.o(i.BSP_SPI_Receive), (42 bytes).
    Removing spi_1.o(i.HAL_SPI_AbortCpltCallback), (56 bytes).
    Removing uart.o(.rev16_text), (4 bytes).
    Removing uart.o(.revsh_text), (4 bytes).
    Removing uart.o(.rrx_text), (6 bytes).
    Removing uart.o(i.BSP_UART_IRQHandler), (72 bytes).
    Removing uart.o(i.BSP_UART_Receive), (44 bytes).
    Removing uart.o(i.BSP_UART_RegisterCallback), (36 bytes).
    Removing uart.o(i.BSP_UART_Transmit), (44 bytes).
    Removing uart.o(i.HAL_UART_AbortCpltCallback), (40 bytes).
    Removing uart.o(i.HAL_UART_AbortReceiveCpltCallback), (40 bytes).
    Removing uart.o(i.HAL_UART_AbortTransmitCpltCallback), (40 bytes).
    Removing uart.o(i.HAL_UART_TxHalfCpltCallback), (36 bytes).
    Removing lcd.o(.rev16_text), (4 bytes).
    Removing lcd.o(.revsh_text), (4 bytes).
    Removing lcd.o(.rrx_text), (6 bytes).
    Removing lcd.o(i.LCD_DrawFloat), (72 bytes).
    Removing lcd.o(i.LCD_DrawHollowCircle), (190 bytes).
    Removing lcd.o(i.LCD_DrawInteger), (56 bytes).
    Removing lcd.o(i.LCD_DrawLine), (160 bytes).
    Removing lcd.o(i.LCD_DrawRectangle), (70 bytes).
    Removing lcd.o(i.LCD_DrawSolidCircle), (142 bytes).
    Removing lcd.o(i.LCD_DrawSolidRectangle), (74 bytes).
    Removing crc8.o(i.CRC8_Calc), (28 bytes).
    Removing crc8.o(i.CRC8_Verify), (36 bytes).
    Removing crc8.o(.constdata), (256 bytes).
    Removing crc16.o(i.CRC16_Calc), (36 bytes).
    Removing crc16.o(i.CRC16_Verify), (48 bytes).
    Removing crc16.o(.constdata), (512 bytes).
    Removing user_math.o(i.fAbs), (12 bytes).
    Removing fadd.o(.text), (176 bytes).
    Removing fmul.o(.text), (100 bytes).
    Removing fdiv.o(.text), (124 bytes).
    Removing fscalb.o(.text), (24 bytes).
    Removing f2d.o(.text), (38 bytes).
    Removing cfcmple.o(.text), (20 bytes).
    Removing cfrcmple.o(.text), (20 bytes).
    Removing fepilogue.o(.text), (110 bytes).
    Removing user_math.o(i.InvSqrt), (88 bytes).
    Removing user_math.o(i.AbsClip), (42 bytes).
    Removing user_math.o(i.Clip), (34 bytes).
    Removing user_math.o(i.Sign), (16 bytes).
    Removing user_math.o(i.ResetMoveVector), (10 bytes).
    Removing user_math.o(i.CircleError), (74 bytes).
    Removing user_math.o(i.CircleAdd), (58 bytes).
    Removing user_math.o(i.CircleReverse), (20 bytes).
    Removing user_math.o(i.CalculateRpm), (136 bytes).

519 unused section(s) (total 31704 bytes) removed from the image.

==============================================================================

Image Symbol Table

    Local Symbols

    Symbol Name                              Value     Ov Type        Size  Object(Section)

    ../Core/Src/dma.c                        0x00000000   Number         0  dma.o ABSOLUTE
    ../Core/Src/gpio.c                       0x00000000   Number         0  gpio.o ABSOLUTE
    ../Core/Src/main.c                       0x00000000   Number         0  main.o ABSOLUTE
    ../Core/Src/spi.c                        0x00000000   Number         0  spi.o ABSOLUTE
    ../Core/Src/stm32f1xx_hal_msp.c          0x00000000   Number         0  stm32f1xx_hal_msp.o ABSOLUTE
    ../Core/Src/stm32f1xx_it.c               0x00000000   Number         0  stm32f1xx_it.o ABSOLUTE
    ../Core/Src/system_stm32f1xx.c           0x00000000   Number         0  system_stm32f1xx.o ABSOLUTE
    ../Core/Src/tim.c                        0x00000000   Number         0  tim.o ABSOLUTE
    ../Core/Src/usart.c                      0x00000000   Number         0  usart.o ABSOLUTE
    ../Drivers/STM32F1xx_HAL_Driver/Src/stm32f1xx_hal.c 0x00000000   Number         0  stm32f1xx_hal.o ABSOLUTE
    ../Drivers/STM32F1xx_HAL_Driver/Src/stm32f1xx_hal_cortex.c 0x00000000   Number         0  stm32f1xx_hal_cortex.o ABSOLUTE
    ../Drivers/STM32F1xx_HAL_Driver/Src/stm32f1xx_hal_dma.c 0x00000000   Number         0  stm32f1xx_hal_dma.o ABSOLUTE
    ../Drivers/STM32F1xx_HAL_Driver/Src/stm32f1xx_hal_exti.c 0x00000000   Number         0  stm32f1xx_hal_exti.o ABSOLUTE
    ../Drivers/STM32F1xx_HAL_Driver/Src/stm32f1xx_hal_flash.c 0x00000000   Number         0  stm32f1xx_hal_flash.o ABSOLUTE
    ../Drivers/STM32F1xx_HAL_Driver/Src/stm32f1xx_hal_flash_ex.c 0x00000000   Number         0  stm32f1xx_hal_flash_ex.o ABSOLUTE
    ../Drivers/STM32F1xx_HAL_Driver/Src/stm32f1xx_hal_gpio.c 0x00000000   Number         0  stm32f1xx_hal_gpio.o ABSOLUTE
    ../Drivers/STM32F1xx_HAL_Driver/Src/stm32f1xx_hal_gpio_ex.c 0x00000000   Number         0  stm32f1xx_hal_gpio_ex.o ABSOLUTE
    ../Drivers/STM32F1xx_HAL_Driver/Src/stm32f1xx_hal_pwr.c 0x00000000   Number         0  stm32f1xx_hal_pwr.o ABSOLUTE
    ../Drivers/STM32F1xx_HAL_Driver/Src/stm32f1xx_hal_rcc.c 0x00000000   Number         0  stm32f1xx_hal_rcc.o ABSOLUTE
    ../Drivers/STM32F1xx_HAL_Driver/Src/stm32f1xx_hal_rcc_ex.c 0x00000000   Number         0  stm32f1xx_hal_rcc_ex.o ABSOLUTE
    ../Drivers/STM32F1xx_HAL_Driver/Src/stm32f1xx_hal_spi.c 0x00000000   Number         0  stm32f1xx_hal_spi.o ABSOLUTE
    ../Drivers/STM32F1xx_HAL_Driver/Src/stm32f1xx_hal_tim.c 0x00000000   Number         0  stm32f1xx_hal_tim.o ABSOLUTE
    ../Drivers/STM32F1xx_HAL_Driver/Src/stm32f1xx_hal_tim_ex.c 0x00000000   Number         0  stm32f1xx_hal_tim_ex.o ABSOLUTE
    ../Drivers/STM32F1xx_HAL_Driver/Src/stm32f1xx_hal_uart.c 0x00000000   Number         0  stm32f1xx_hal_uart.o ABSOLUTE
    ../clib/microlib/ctype/ctype.c           0x00000000   Number         0  isspace_c.o ABSOLUTE
    ../clib/microlib/ctype/ctype.c           0x00000000   Number         0  ctype_c.o ABSOLUTE
    ../clib/microlib/division.c              0x00000000   Number         0  uldiv.o ABSOLUTE
    ../clib/microlib/division.c              0x00000000   Number         0  uidiv.o ABSOLUTE
    ../clib/microlib/init/entry.s            0x00000000   Number         0  entry12a.o ABSOLUTE
    ../clib/microlib/init/entry.s            0x00000000   Number         0  entry10b.o ABSOLUTE
    ../clib/microlib/init/entry.s            0x00000000   Number         0  entry10a.o ABSOLUTE
    ../clib/microlib/init/entry.s            0x00000000   Number         0  entry11a.o ABSOLUTE
    ../clib/microlib/init/entry.s            0x00000000   Number         0  entry9a.o ABSOLUTE
    ../clib/microlib/init/entry.s            0x00000000   Number         0  entry8b.o ABSOLUTE
    ../clib/microlib/init/entry.s            0x00000000   Number         0  entry8a.o ABSOLUTE
    ../clib/microlib/init/entry.s            0x00000000   Number         0  entry7b.o ABSOLUTE
    ../clib/microlib/init/entry.s            0x00000000   Number         0  entry7a.o ABSOLUTE
    ../clib/microlib/init/entry.s            0x00000000   Number         0  entry5.o ABSOLUTE
    ../clib/microlib/init/entry.s            0x00000000   Number         0  entry12b.o ABSOLUTE
    ../clib/microlib/init/entry.s            0x00000000   Number         0  entry2.o ABSOLUTE
    ../clib/microlib/init/entry.s            0x00000000   Number         0  entry11b.o ABSOLUTE
    ../clib/microlib/init/entry.s            0x00000000   Number         0  entry9b.o ABSOLUTE
    ../clib/microlib/init/entry.s            0x00000000   Number         0  entry.o ABSOLUTE
    ../clib/microlib/longlong.c              0x00000000   Number         0  llshl.o ABSOLUTE
    ../clib/microlib/longlong.c              0x00000000   Number         0  llsshr.o ABSOLUTE
    ../clib/microlib/longlong.c              0x00000000   Number         0  llushr.o ABSOLUTE
    ../clib/microlib/malloc/malloc.c         0x00000000   Number         0  malloca.o ABSOLUTE
    ../clib/microlib/malloc/malloc.c         0x00000000   Number         0  mallocra.o ABSOLUTE
    ../clib/microlib/malloc/malloc.c         0x00000000   Number         0  malloc.o ABSOLUTE
    ../clib/microlib/malloc/malloc.c         0x00000000   Number         0  mallocr.o ABSOLUTE
    ../clib/microlib/malloc/mvars.c          0x00000000   Number         0  mvars.o ABSOLUTE
    ../clib/microlib/printf/printf.c         0x00000000   Number         0  printf7.o ABSOLUTE
    ../clib/microlib/printf/printf.c         0x00000000   Number         0  printfa.o ABSOLUTE
    ../clib/microlib/printf/printf.c         0x00000000   Number         0  printf8.o ABSOLUTE
    ../clib/microlib/printf/printf.c         0x00000000   Number         0  printf6.o ABSOLUTE
    ../clib/microlib/printf/printf.c         0x00000000   Number         0  printf5.o ABSOLUTE
    ../clib/microlib/printf/printf.c         0x00000000   Number         0  printf4.o ABSOLUTE
    ../clib/microlib/printf/printf.c         0x00000000   Number         0  printf3.o ABSOLUTE
    ../clib/microlib/printf/printf.c         0x00000000   Number         0  printf2.o ABSOLUTE
    ../clib/microlib/printf/printf.c         0x00000000   Number         0  printf1.o ABSOLUTE
    ../clib/microlib/printf/printf.c         0x00000000   Number         0  printf0.o ABSOLUTE
    ../clib/microlib/printf/printf.c         0x00000000   Number         0  printfb.o ABSOLUTE
    ../clib/microlib/printf/stubs.s          0x00000000   Number         0  stubs.o ABSOLUTE
    ../clib/microlib/stdio/streams.c         0x00000000   Number         0  stdout.o ABSOLUTE
    ../clib/microlib/string/memcpy.c         0x00000000   Number         0  memcpya.o ABSOLUTE
    ../clib/microlib/string/memcpy.c         0x00000000   Number         0  memcpyb.o ABSOLUTE
    ../clib/microlib/string/memset.c         0x00000000   Number         0  memseta.o ABSOLUTE
    ../clib/microlib/string/strcpy.c         0x00000000   Number         0  strcpy.o ABSOLUTE
    ../clib/microlib/string/strlen.c         0x00000000   Number         0  strlen.o ABSOLUTE
    ../clib/microlib/stubs.s                 0x00000000   Number         0  iusefp.o ABSOLUTE
    ../clib/scanf.c                          0x00000000   Number         0  __0sscanf.o ABSOLUTE
    ../clib/scanf.c                          0x00000000   Number         0  _sgetc.o ABSOLUTE
    ../clib/scanf.c                          0x00000000   Number         0  _chval.o ABSOLUTE
    ../clib/scanf.c                          0x00000000   Number         0  scanf_char.o ABSOLUTE
    ../clib/scanf.c                          0x00000000   Number         0  _scanf.o ABSOLUTE
    ../clib/scanf.c                          0x00000000   Number         0  _scanf_int.o ABSOLUTE
    ../fplib/microlib/f2d.c                  0x00000000   Number         0  f2d.o ABSOLUTE
    ../fplib/microlib/fpadd.c                0x00000000   Number         0  fadd.o ABSOLUTE
    ../fplib/microlib/fpadd.c                0x00000000   Number         0  dadd.o ABSOLUTE
    ../fplib/microlib/fpdiv.c                0x00000000   Number         0  ddiv.o ABSOLUTE
    ../fplib/microlib/fpdiv.c                0x00000000   Number         0  fdiv.o ABSOLUTE
    ../fplib/microlib/fpepilogue.c           0x00000000   Number         0  fepilogue.o ABSOLUTE
    ../fplib/microlib/fpepilogue.c           0x00000000   Number         0  depilogue.o ABSOLUTE
    ../fplib/microlib/fpfix.c                0x00000000   Number         0  dfixui.o ABSOLUTE
    ../fplib/microlib/fpfix.c                0x00000000   Number         0  dfixul.o ABSOLUTE
    ../fplib/microlib/fpflt.c                0x00000000   Number         0  dflti.o ABSOLUTE
    ../fplib/microlib/fpflt.c                0x00000000   Number         0  dfltui.o ABSOLUTE
    ../fplib/microlib/fpmul.c                0x00000000   Number         0  dmul.o ABSOLUTE
    ../fplib/microlib/fpmul.c                0x00000000   Number         0  fmul.o ABSOLUTE
    ../fplib/microlib/fpscalb.c              0x00000000   Number         0  fscalb.o ABSOLUTE
    ..\Core\Src\dma.c                        0x00000000   Number         0  dma.o ABSOLUTE
    ..\Core\Src\gpio.c                       0x00000000   Number         0  gpio.o ABSOLUTE
    ..\Core\Src\main.c                       0x00000000   Number         0  main.o ABSOLUTE
    ..\Core\Src\spi.c                        0x00000000   Number         0  spi.o ABSOLUTE
    ..\Core\Src\stm32f1xx_hal_msp.c          0x00000000   Number         0  stm32f1xx_hal_msp.o ABSOLUTE
    ..\Core\Src\stm32f1xx_it.c               0x00000000   Number         0  stm32f1xx_it.o ABSOLUTE
    ..\Core\Src\system_stm32f1xx.c           0x00000000   Number         0  system_stm32f1xx.o ABSOLUTE
    ..\Core\Src\tim.c                        0x00000000   Number         0  tim.o ABSOLUTE
    ..\Core\Src\usart.c                      0x00000000   Number         0  usart.o ABSOLUTE
    ..\Drivers\STM32F1xx_HAL_Driver\Src\stm32f1xx_hal.c 0x00000000   Number         0  stm32f1xx_hal.o ABSOLUTE
    ..\Drivers\STM32F1xx_HAL_Driver\Src\stm32f1xx_hal_cortex.c 0x00000000   Number         0  stm32f1xx_hal_cortex.o ABSOLUTE
    ..\Drivers\STM32F1xx_HAL_Driver\Src\stm32f1xx_hal_dma.c 0x00000000   Number         0  stm32f1xx_hal_dma.o ABSOLUTE
    ..\Drivers\STM32F1xx_HAL_Driver\Src\stm32f1xx_hal_exti.c 0x00000000   Number         0  stm32f1xx_hal_exti.o ABSOLUTE
    ..\Drivers\STM32F1xx_HAL_Driver\Src\stm32f1xx_hal_flash.c 0x00000000   Number         0  stm32f1xx_hal_flash.o ABSOLUTE
    ..\Drivers\STM32F1xx_HAL_Driver\Src\stm32f1xx_hal_flash_ex.c 0x00000000   Number         0  stm32f1xx_hal_flash_ex.o ABSOLUTE
    ..\Drivers\STM32F1xx_HAL_Driver\Src\stm32f1xx_hal_gpio.c 0x00000000   Number         0  stm32f1xx_hal_gpio.o ABSOLUTE
    ..\Drivers\STM32F1xx_HAL_Driver\Src\stm32f1xx_hal_gpio_ex.c 0x00000000   Number         0  stm32f1xx_hal_gpio_ex.o ABSOLUTE
    ..\Drivers\STM32F1xx_HAL_Driver\Src\stm32f1xx_hal_pwr.c 0x00000000   Number         0  stm32f1xx_hal_pwr.o ABSOLUTE
    ..\Drivers\STM32F1xx_HAL_Driver\Src\stm32f1xx_hal_rcc.c 0x00000000   Number         0  stm32f1xx_hal_rcc.o ABSOLUTE
    ..\Drivers\STM32F1xx_HAL_Driver\Src\stm32f1xx_hal_rcc_ex.c 0x00000000   Number         0  stm32f1xx_hal_rcc_ex.o ABSOLUTE
    ..\Drivers\STM32F1xx_HAL_Driver\Src\stm32f1xx_hal_spi.c 0x00000000   Number         0  stm32f1xx_hal_spi.o ABSOLUTE
    ..\Drivers\STM32F1xx_HAL_Driver\Src\stm32f1xx_hal_tim.c 0x00000000   Number         0  stm32f1xx_hal_tim.o ABSOLUTE
    ..\Drivers\STM32F1xx_HAL_Driver\Src\stm32f1xx_hal_tim_ex.c 0x00000000   Number         0  stm32f1xx_hal_tim_ex.o ABSOLUTE
    ..\Drivers\STM32F1xx_HAL_Driver\Src\stm32f1xx_hal_uart.c 0x00000000   Number         0  stm32f1xx_hal_uart.o ABSOLUTE
    ..\User\bsp\gpio.c                       0x00000000   Number         0  gpio_1.o ABSOLUTE
    ..\User\bsp\spi.c                        0x00000000   Number         0  spi_1.o ABSOLUTE
    ..\User\bsp\uart.c                       0x00000000   Number         0  uart.o ABSOLUTE
    ..\User\component\crc16.c                0x00000000   Number         0  crc16.o ABSOLUTE
    ..\User\component\crc8.c                 0x00000000   Number         0  crc8.o ABSOLUTE
    ..\User\component\user_math.c            0x00000000   Number         0  user_math.o ABSOLUTE
    ..\User\device\lcd_driver\lcd.c          0x00000000   Number         0  lcd.o ABSOLUTE
    ..\\User\\bsp\\gpio.c                    0x00000000   Number         0  gpio_1.o ABSOLUTE
    ..\\User\\bsp\\spi.c                     0x00000000   Number         0  spi_1.o ABSOLUTE
    ..\\User\\bsp\\uart.c                    0x00000000   Number         0  uart.o ABSOLUTE
    ..\\User\\device\\lcd_driver\\lcd.c      0x00000000   Number         0  lcd.o ABSOLUTE
    ..\\sx1281-driver-c\\sx1281.c            0x00000000   Number         0  sx1281.o ABSOLUTE
    ..\\sx1281-driver-c\\sx1281_driver.c     0x00000000   Number         0  sx1281_driver.o ABSOLUTE
    ..\\sx1281-driver-c\\sx1281_driver_gpio.c 0x00000000   Number         0  sx1281_driver_gpio.o ABSOLUTE
    ..\\sx1281-driver-c\\sx1281_driver_hal.c 0x00000000   Number         0  sx1281_driver_hal.o ABSOLUTE
    ..\\sx1281-driver-c\\sx1281_driver_spi.c 0x00000000   Number         0  sx1281_driver_spi.o ABSOLUTE
    ..\\sx1281-driver-c\\sx1281_driver_uart.c 0x00000000   Number         0  sx1281_driver_uart.o ABSOLUTE
    ..\\sx1281-driver-c\\sx1281_header.c     0x00000000   Number         0  sx1281_header.o ABSOLUTE
    ..\sx1281-driver-c\sx1281.c              0x00000000   Number         0  sx1281.o ABSOLUTE
    ..\sx1281-driver-c\sx1281_driver.c       0x00000000   Number         0  sx1281_driver.o ABSOLUTE
    ..\sx1281-driver-c\sx1281_driver_gpio.c  0x00000000   Number         0  sx1281_driver_gpio.o ABSOLUTE
    ..\sx1281-driver-c\sx1281_driver_hal.c   0x00000000   Number         0  sx1281_driver_hal.o ABSOLUTE
    ..\sx1281-driver-c\sx1281_driver_spi.c   0x00000000   Number         0  sx1281_driver_spi.o ABSOLUTE
    ..\sx1281-driver-c\sx1281_driver_uart.c  0x00000000   Number         0  sx1281_driver_uart.o ABSOLUTE
    ..\sx1281-driver-c\sx1281_header.c       0x00000000   Number         0  sx1281_header.o ABSOLUTE
    cdrcmple.s                               0x00000000   Number         0  cdrcmple.o ABSOLUTE
    cfcmple.s                                0x00000000   Number         0  cfcmple.o ABSOLUTE
    cfrcmple.s                               0x00000000   Number         0  cfrcmple.o ABSOLUTE
    dc.s                                     0x00000000   Number         0  dc.o ABSOLUTE
    handlers.s                               0x00000000   Number         0  handlers.o ABSOLUTE
    init.s                                   0x00000000   Number         0  init.o ABSOLUTE
    startup_stm32f103xb.s                    0x00000000   Number         0  startup_stm32f103xb.o ABSOLUTE
    RESET                                    0x08000000   Section      236  startup_stm32f103xb.o(RESET)
    .ARM.Collect$$$$00000000                 0x080000ec   Section        0  entry.o(.ARM.Collect$$$$00000000)
    .ARM.Collect$$$$00000001                 0x080000ec   Section        4  entry2.o(.ARM.Collect$$$$00000001)
    .ARM.Collect$$$$00000004                 0x080000f0   Section        4  entry5.o(.ARM.Collect$$$$00000004)
    .ARM.Collect$$$$00000008                 0x080000f4   Section        0  entry7b.o(.ARM.Collect$$$$00000008)
    .ARM.Collect$$$$0000000A                 0x080000f4   Section        0  entry8b.o(.ARM.Collect$$$$0000000A)
    .ARM.Collect$$$$0000000B                 0x080000f4   Section        8  entry9a.o(.ARM.Collect$$$$0000000B)
    .ARM.Collect$$$$0000000E                 0x080000fc   Section        4  entry12b.o(.ARM.Collect$$$$0000000E)
    .ARM.Collect$$$$0000000F                 0x08000100   Section        0  entry10a.o(.ARM.Collect$$$$0000000F)
    .ARM.Collect$$$$00000011                 0x08000100   Section        0  entry11a.o(.ARM.Collect$$$$00000011)
    .ARM.Collect$$$$00002712                 0x08000100   Section        4  entry2.o(.ARM.Collect$$$$00002712)
    __lit__00000000                          0x08000100   Data           4  entry2.o(.ARM.Collect$$$$00002712)
    .text                                    0x08000104   Section       36  startup_stm32f103xb.o(.text)
    .text                                    0x08000128   Section        0  llushr.o(.text)
    .text                                    0x08000148   Section        0  memcpya.o(.text)
    .text                                    0x0800016c   Section        0  memseta.o(.text)
    .text                                    0x08000190   Section        0  strcpy.o(.text)
    .text                                    0x080001a2   Section        0  dmul.o(.text)
    .text                                    0x08000286   Section        0  ddiv.o(.text)
    .text                                    0x08000364   Section        0  dflti.o(.text)
    .text                                    0x08000386   Section        0  dfltui.o(.text)
    .text                                    0x080003a0   Section        0  dfixui.o(.text)
    .text                                    0x080003d2   Section        0  uidiv.o(.text)
    .text                                    0x080003fe   Section        0  uldiv.o(.text)
    .text                                    0x08000460   Section        0  iusefp.o(.text)
    .text                                    0x08000460   Section        0  depilogue.o(.text)
    .text                                    0x0800051a   Section        0  dadd.o(.text)
    .text                                    0x08000668   Section        0  dfixul.o(.text)
    .text                                    0x08000698   Section       48  cdrcmple.o(.text)
    .text                                    0x080006c8   Section       36  init.o(.text)
    .text                                    0x080006ec   Section        0  llshl.o(.text)
    .text                                    0x0800070a   Section        0  llsshr.o(.text)
    i.BSP_SPI_GetHandle                      0x08000730   Section        0  spi_1.o(i.BSP_SPI_GetHandle)
    i.BSP_SPI_GetState                       0x0800074c   Section        0  spi_1.o(i.BSP_SPI_GetState)
    i.BSP_SPI_RegisterCallback               0x08000764   Section        0  spi_1.o(i.BSP_SPI_RegisterCallback)
    i.BSP_SPI_Transmit                       0x08000780   Section        0  spi_1.o(i.BSP_SPI_Transmit)
    i.BSP_SPI_TransmitReceive                0x080007aa   Section        0  spi_1.o(i.BSP_SPI_TransmitReceive)
    i.BSP_UART_GetHandle                     0x080007d8   Section        0  uart.o(i.BSP_UART_GetHandle)
    i.BusFault_Handler                       0x080007e8   Section        0  stm32f1xx_it.o(i.BusFault_Handler)
    i.DMA1_Channel2_IRQHandler               0x080007ec   Section        0  stm32f1xx_it.o(i.DMA1_Channel2_IRQHandler)
    i.DMA1_Channel3_IRQHandler               0x080007f8   Section        0  stm32f1xx_it.o(i.DMA1_Channel3_IRQHandler)
    i.DMA1_Channel5_IRQHandler               0x08000804   Section        0  stm32f1xx_it.o(i.DMA1_Channel5_IRQHandler)
    i.DMA1_Channel6_IRQHandler               0x08000810   Section        0  stm32f1xx_it.o(i.DMA1_Channel6_IRQHandler)
    i.DMA1_Channel7_IRQHandler               0x0800081c   Section        0  stm32f1xx_it.o(i.DMA1_Channel7_IRQHandler)
    i.DMA_SetConfig                          0x08000828   Section        0  stm32f1xx_hal_dma.o(i.DMA_SetConfig)
    DMA_SetConfig                            0x08000829   Thumb Code    42  stm32f1xx_hal_dma.o(i.DMA_SetConfig)
    i.DebugMon_Handler                       0x08000852   Section        0  stm32f1xx_it.o(i.DebugMon_Handler)
    i.EXTI15_10_IRQHandler                   0x08000854   Section        0  stm32f1xx_it.o(i.EXTI15_10_IRQHandler)
    i.EXTI9_5_IRQHandler                     0x0800085c   Section        0  stm32f1xx_it.o(i.EXTI9_5_IRQHandler)
    i.Error_Handler                          0x08000874   Section        0  main.o(i.Error_Handler)
    i.GpioGetBitPos                          0x08000878   Section        0  sx1281_driver_gpio.o(i.GpioGetBitPos)
    i.GpioInit                               0x080008a8   Section        0  sx1281_driver_gpio.o(i.GpioInit)
    i.GpioRead                               0x080008aa   Section        0  sx1281_driver_gpio.o(i.GpioRead)
    i.GpioSetIrq                             0x080008b0   Section        0  sx1281_driver_gpio.o(i.GpioSetIrq)
    i.GpioWrite                              0x080008e8   Section        0  sx1281_driver_gpio.o(i.GpioWrite)
    i.HAL_DMA_Abort                          0x080008ee   Section        0  stm32f1xx_hal_dma.o(i.HAL_DMA_Abort)
    i.HAL_DMA_Abort_IT                       0x08000934   Section        0  stm32f1xx_hal_dma.o(i.HAL_DMA_Abort_IT)
    i.HAL_DMA_IRQHandler                     0x080009cc   Section        0  stm32f1xx_hal_dma.o(i.HAL_DMA_IRQHandler)
    i.HAL_DMA_Init                           0x08000b20   Section        0  stm32f1xx_hal_dma.o(i.HAL_DMA_Init)
    i.HAL_DMA_Start_IT                       0x08000b7c   Section        0  stm32f1xx_hal_dma.o(i.HAL_DMA_Start_IT)
    i.HAL_Delay                              0x08000bec   Section        0  stm32f1xx_hal.o(i.HAL_Delay)
    i.HAL_GPIO_EXTI_Callback                 0x08000c10   Section        0  gpio_1.o(i.HAL_GPIO_EXTI_Callback)
    i.HAL_GPIO_EXTI_IRQHandler               0x08000c3c   Section        0  stm32f1xx_hal_gpio.o(i.HAL_GPIO_EXTI_IRQHandler)
    i.HAL_GPIO_Init                          0x08000c54   Section        0  stm32f1xx_hal_gpio.o(i.HAL_GPIO_Init)
    i.HAL_GPIO_ReadPin                       0x08000e34   Section        0  stm32f1xx_hal_gpio.o(i.HAL_GPIO_ReadPin)
    i.HAL_GPIO_WritePin                      0x08000e3e   Section        0  stm32f1xx_hal_gpio.o(i.HAL_GPIO_WritePin)
    i.HAL_GetTick                            0x08000e48   Section        0  stm32f1xx_hal.o(i.HAL_GetTick)
    i.HAL_HalfDuplex_Init                    0x08000e54   Section        0  stm32f1xx_hal_uart.o(i.HAL_HalfDuplex_Init)
    i.HAL_IncTick                            0x08000ec4   Section        0  stm32f1xx_hal.o(i.HAL_IncTick)
    i.HAL_Init                               0x08000ed4   Section        0  stm32f1xx_hal.o(i.HAL_Init)
    i.HAL_InitTick                           0x08000ef8   Section        0  stm32f1xx_hal.o(i.HAL_InitTick)
    i.HAL_MspInit                            0x08000f38   Section        0  stm32f1xx_hal_msp.o(i.HAL_MspInit)
    i.HAL_NVIC_EnableIRQ                     0x08000f74   Section        0  stm32f1xx_hal_cortex.o(i.HAL_NVIC_EnableIRQ)
    i.HAL_NVIC_SetPriority                   0x08000f90   Section        0  stm32f1xx_hal_cortex.o(i.HAL_NVIC_SetPriority)
    i.HAL_NVIC_SetPriorityGrouping           0x08000fd0   Section        0  stm32f1xx_hal_cortex.o(i.HAL_NVIC_SetPriorityGrouping)
    i.HAL_RCC_ClockConfig                    0x08000ff4   Section        0  stm32f1xx_hal_rcc.o(i.HAL_RCC_ClockConfig)
    i.HAL_RCC_GetPCLK1Freq                   0x08001120   Section        0  stm32f1xx_hal_rcc.o(i.HAL_RCC_GetPCLK1Freq)
    i.HAL_RCC_GetPCLK2Freq                   0x08001140   Section        0  stm32f1xx_hal_rcc.o(i.HAL_RCC_GetPCLK2Freq)
    i.HAL_RCC_GetSysClockFreq                0x08001160   Section        0  stm32f1xx_hal_rcc.o(i.HAL_RCC_GetSysClockFreq)
    i.HAL_RCC_OscConfig                      0x080011b4   Section        0  stm32f1xx_hal_rcc.o(i.HAL_RCC_OscConfig)
    i.HAL_SPI_ErrorCallback                  0x080014d4   Section        0  spi_1.o(i.HAL_SPI_ErrorCallback)
    i.HAL_SPI_GetState                       0x0800150c   Section        0  stm32f1xx_hal_spi.o(i.HAL_SPI_GetState)
    i.HAL_SPI_Init                           0x08001512   Section        0  stm32f1xx_hal_spi.o(i.HAL_SPI_Init)
    i.HAL_SPI_MspInit                        0x080015c4   Section        0  spi.o(i.HAL_SPI_MspInit)
    i.HAL_SPI_RxCpltCallback                 0x080016fc   Section        0  spi_1.o(i.HAL_SPI_RxCpltCallback)
    i.HAL_SPI_RxHalfCpltCallback             0x08001734   Section        0  spi_1.o(i.HAL_SPI_RxHalfCpltCallback)
    i.HAL_SPI_Transmit                       0x0800176c   Section        0  stm32f1xx_hal_spi.o(i.HAL_SPI_Transmit)
    i.HAL_SPI_TransmitReceive                0x080018d2   Section        0  stm32f1xx_hal_spi.o(i.HAL_SPI_TransmitReceive)
    i.HAL_SPI_TransmitReceive_DMA            0x08001ac4   Section        0  stm32f1xx_hal_spi.o(i.HAL_SPI_TransmitReceive_DMA)
    i.HAL_SPI_Transmit_DMA                   0x08001bd4   Section        0  stm32f1xx_hal_spi.o(i.HAL_SPI_Transmit_DMA)
    i.HAL_SPI_TxCpltCallback                 0x08001ca0   Section        0  spi_1.o(i.HAL_SPI_TxCpltCallback)
    i.HAL_SPI_TxHalfCpltCallback             0x08001cc4   Section        0  spi_1.o(i.HAL_SPI_TxHalfCpltCallback)
    i.HAL_SPI_TxRxCpltCallback               0x08001cfc   Section        0  spi_1.o(i.HAL_SPI_TxRxCpltCallback)
    i.HAL_SPI_TxRxHalfCpltCallback           0x08001d34   Section        0  spi_1.o(i.HAL_SPI_TxRxHalfCpltCallback)
    i.HAL_SYSTICK_Config                     0x08001d6c   Section        0  stm32f1xx_hal_cortex.o(i.HAL_SYSTICK_Config)
    i.HAL_TIMEx_ConfigBreakDeadTime          0x08001d94   Section        0  stm32f1xx_hal_tim_ex.o(i.HAL_TIMEx_ConfigBreakDeadTime)
    i.HAL_TIMEx_MasterConfigSynchronization  0x08001de8   Section        0  stm32f1xx_hal_tim_ex.o(i.HAL_TIMEx_MasterConfigSynchronization)
    i.HAL_TIM_Base_Init                      0x08001e50   Section        0  stm32f1xx_hal_tim.o(i.HAL_TIM_Base_Init)
    i.HAL_TIM_Base_MspInit                   0x08001eac   Section        0  tim.o(i.HAL_TIM_Base_MspInit)
    i.HAL_TIM_ConfigClockSource              0x08001ed4   Section        0  stm32f1xx_hal_tim.o(i.HAL_TIM_ConfigClockSource)
    i.HAL_TIM_MspPostInit                    0x08001fb0   Section        0  tim.o(i.HAL_TIM_MspPostInit)
    i.HAL_TIM_PWM_ConfigChannel              0x08001ffc   Section        0  stm32f1xx_hal_tim.o(i.HAL_TIM_PWM_ConfigChannel)
    i.HAL_TIM_PWM_Init                       0x080020c8   Section        0  stm32f1xx_hal_tim.o(i.HAL_TIM_PWM_Init)
    i.HAL_TIM_PWM_MspInit                    0x08002122   Section        0  stm32f1xx_hal_tim.o(i.HAL_TIM_PWM_MspInit)
    i.HAL_UARTEx_RxEventCallback             0x08002124   Section        0  stm32f1xx_hal_uart.o(i.HAL_UARTEx_RxEventCallback)
    i.HAL_UART_DMAStop                       0x08002126   Section        0  stm32f1xx_hal_uart.o(i.HAL_UART_DMAStop)
    i.HAL_UART_ErrorCallback                 0x08002198   Section        0  uart.o(i.HAL_UART_ErrorCallback)
    i.HAL_UART_IRQHandler                    0x080021c0   Section        0  stm32f1xx_hal_uart.o(i.HAL_UART_IRQHandler)
    i.HAL_UART_Init                          0x0800242c   Section        0  stm32f1xx_hal_uart.o(i.HAL_UART_Init)
    i.HAL_UART_MspInit                       0x08002490   Section        0  usart.o(i.HAL_UART_MspInit)
    i.HAL_UART_Receive_DMA                   0x080025a8   Section        0  stm32f1xx_hal_uart.o(i.HAL_UART_Receive_DMA)
    i.HAL_UART_RxCpltCallback                0x080025c4   Section        0  uart.o(i.HAL_UART_RxCpltCallback)
    i.HAL_UART_RxHalfCpltCallback            0x080025ec   Section        0  uart.o(i.HAL_UART_RxHalfCpltCallback)
    i.HAL_UART_Transmit                      0x08002614   Section        0  stm32f1xx_hal_uart.o(i.HAL_UART_Transmit)
    i.HAL_UART_TxCpltCallback                0x080026b4   Section        0  uart.o(i.HAL_UART_TxCpltCallback)
    i.HardFault_Handler                      0x080026dc   Section        0  stm32f1xx_it.o(i.HardFault_Handler)
    i.LCD_Clear                              0x080026de   Section        0  lcd.o(i.LCD_Clear)
    i.LCD_DrawBitmap                         0x08002730   Section        0  lcd.o(i.LCD_DrawBitmap)
    i.LCD_DrawChar                           0x080027b0   Section        0  lcd.o(i.LCD_DrawChar)
    i.LCD_DrawPoint                          0x08002914   Section        0  lcd.o(i.LCD_DrawPoint)
    i.LCD_DrawString                         0x08002970   Section        0  lcd.o(i.LCD_DrawString)
    i.LCD_Init                               0x080029e0   Section        0  lcd.o(i.LCD_Init)
    i.LCD_SetAddressWindow                   0x08002b40   Section        0  lcd.o(i.LCD_SetAddressWindow)
    LCD_SetAddressWindow                     0x08002b41   Thumb Code   100  lcd.o(i.LCD_SetAddressWindow)
    i.LCD_WriteCommand                       0x08002ba4   Section        0  lcd.o(i.LCD_WriteCommand)
    LCD_WriteCommand                         0x08002ba5   Thumb Code    56  lcd.o(i.LCD_WriteCommand)
    i.LCD_WriteData                          0x08002be4   Section        0  lcd.o(i.LCD_WriteData)
    LCD_WriteData                            0x08002be5   Thumb Code    54  lcd.o(i.LCD_WriteData)
    i.LCD_WriteDataBuffer                    0x08002c24   Section        0  lcd.o(i.LCD_WriteDataBuffer)
    LCD_WriteDataBuffer                      0x08002c25   Thumb Code    72  lcd.o(i.LCD_WriteDataBuffer)
    i.LCD_WriteDataBuffer_DMA                0x08002c74   Section        0  lcd.o(i.LCD_WriteDataBuffer_DMA)
    LCD_WriteDataBuffer_DMA                  0x08002c75   Thumb Code    72  lcd.o(i.LCD_WriteDataBuffer_DMA)
    i.MSP_GetIRQn                            0x08002cc4   Section        0  sx1281_driver_gpio.o(i.MSP_GetIRQn)
    i.MX_DMA_Init                            0x08002d00   Section        0  dma.o(i.MX_DMA_Init)
    i.MX_GPIO_Init                           0x08002d6c   Section        0  gpio.o(i.MX_GPIO_Init)
    i.MX_SPI1_Init                           0x08002e84   Section        0  spi.o(i.MX_SPI1_Init)
    i.MX_SPI2_Init                           0x08002ecc   Section        0  spi.o(i.MX_SPI2_Init)
    i.MX_TIM1_Init                           0x08002f14   Section        0  tim.o(i.MX_TIM1_Init)
    i.MX_USART1_UART_Init                    0x08002fd8   Section        0  usart.o(i.MX_USART1_UART_Init)
    i.MX_USART2_UART_Init                    0x08003010   Section        0  usart.o(i.MX_USART2_UART_Init)
    i.MemManage_Handler                      0x08003048   Section        0  stm32f1xx_it.o(i.MemManage_Handler)
    i.NMI_Handler                            0x0800304a   Section        0  stm32f1xx_it.o(i.NMI_Handler)
    i.OnRxDone                               0x0800304c   Section        0  sx1281.o(i.OnRxDone)
    i.OnRxError                              0x08003060   Section        0  sx1281.o(i.OnRxError)
    i.OnRxTimeout                            0x08003074   Section        0  sx1281.o(i.OnRxTimeout)
    i.OnTxDone                               0x08003088   Section        0  sx1281.o(i.OnTxDone)
    i.OnTxTimeout                            0x0800309c   Section        0  sx1281.o(i.OnTxTimeout)
    i.PendSV_Handler                         0x080030b0   Section        0  stm32f1xx_it.o(i.PendSV_Handler)
    i.SPI_DMAError                           0x080030b2   Section        0  stm32f1xx_hal_spi.o(i.SPI_DMAError)
    SPI_DMAError                             0x080030b3   Thumb Code    34  stm32f1xx_hal_spi.o(i.SPI_DMAError)
    i.SPI_DMAHalfReceiveCplt                 0x080030d4   Section        0  stm32f1xx_hal_spi.o(i.SPI_DMAHalfReceiveCplt)
    SPI_DMAHalfReceiveCplt                   0x080030d5   Thumb Code    10  stm32f1xx_hal_spi.o(i.SPI_DMAHalfReceiveCplt)
    i.SPI_DMAHalfTransmitCplt                0x080030de   Section        0  stm32f1xx_hal_spi.o(i.SPI_DMAHalfTransmitCplt)
    SPI_DMAHalfTransmitCplt                  0x080030df   Thumb Code    10  stm32f1xx_hal_spi.o(i.SPI_DMAHalfTransmitCplt)
    i.SPI_DMAHalfTransmitReceiveCplt         0x080030e8   Section        0  stm32f1xx_hal_spi.o(i.SPI_DMAHalfTransmitReceiveCplt)
    SPI_DMAHalfTransmitReceiveCplt           0x080030e9   Thumb Code    10  stm32f1xx_hal_spi.o(i.SPI_DMAHalfTransmitReceiveCplt)
    i.SPI_DMAReceiveCplt                     0x080030f2   Section        0  stm32f1xx_hal_spi.o(i.SPI_DMAReceiveCplt)
    SPI_DMAReceiveCplt                       0x080030f3   Thumb Code   106  stm32f1xx_hal_spi.o(i.SPI_DMAReceiveCplt)
    i.SPI_DMATransmitCplt                    0x0800315c   Section        0  stm32f1xx_hal_spi.o(i.SPI_DMATransmitCplt)
    SPI_DMATransmitCplt                      0x0800315d   Thumb Code   100  stm32f1xx_hal_spi.o(i.SPI_DMATransmitCplt)
    i.SPI_DMATransmitReceiveCplt             0x080031c0   Section        0  stm32f1xx_hal_spi.o(i.SPI_DMATransmitReceiveCplt)
    SPI_DMATransmitReceiveCplt               0x080031c1   Thumb Code    90  stm32f1xx_hal_spi.o(i.SPI_DMATransmitReceiveCplt)
    i.SPI_EndRxTransaction                   0x0800321a   Section        0  stm32f1xx_hal_spi.o(i.SPI_EndRxTransaction)
    SPI_EndRxTransaction                     0x0800321b   Thumb Code    92  stm32f1xx_hal_spi.o(i.SPI_EndRxTransaction)
    i.SPI_EndRxTxTransaction                 0x08003276   Section        0  stm32f1xx_hal_spi.o(i.SPI_EndRxTxTransaction)
    SPI_EndRxTxTransaction                   0x08003277   Thumb Code    52  stm32f1xx_hal_spi.o(i.SPI_EndRxTxTransaction)
    i.SPI_Get                                0x080032ac   Section        0  spi_1.o(i.SPI_Get)
    SPI_Get                                  0x080032ad   Thumb Code    26  spi_1.o(i.SPI_Get)
    i.SPI_WaitFlagStateUntilTimeout          0x080032d0   Section        0  stm32f1xx_hal_spi.o(i.SPI_WaitFlagStateUntilTimeout)
    SPI_WaitFlagStateUntilTimeout            0x080032d1   Thumb Code   180  stm32f1xx_hal_spi.o(i.SPI_WaitFlagStateUntilTimeout)
    i.SVC_Handler                            0x08003388   Section        0  stm32f1xx_it.o(i.SVC_Handler)
    i.SX1281Calibrate                        0x0800338a   Section        0  sx1281_driver.o(i.SX1281Calibrate)
    i.SX1281ClearIrqStatus                   0x080033c8   Section        0  sx1281_driver.o(i.SX1281ClearIrqStatus)
    i.SX1281GetFirmwareVersion               0x080033e0   Section        0  sx1281_driver.o(i.SX1281GetFirmwareVersion)
    i.SX1281GetFrequencyError                0x080033fc   Section        0  sx1281_driver.o(i.SX1281GetFrequencyError)
    i.SX1281GetIrqStatus                     0x08003494   Section        0  sx1281_driver.o(i.SX1281GetIrqStatus)
    i.SX1281GetLoRaBandwidth                 0x080034a8   Section        0  sx1281_driver.o(i.SX1281GetLoRaBandwidth)
    i.SX1281GetOpMode                        0x080034e4   Section        0  sx1281_driver.o(i.SX1281GetOpMode)
    i.SX1281GetPacketStatus                  0x080034f0   Section        0  sx1281_driver.o(i.SX1281GetPacketStatus)
    i.SX1281GetPacketType                    0x08003704   Section        0  sx1281_driver.o(i.SX1281GetPacketType)
    i.SX1281GetPayload                       0x08003710   Section        0  sx1281_driver.o(i.SX1281GetPayload)
    i.SX1281GetRssiInst                      0x08003738   Section        0  sx1281_driver.o(i.SX1281GetRssiInst)
    i.SX1281GetRxBufferStatus                0x0800375c   Section        0  sx1281_driver.o(i.SX1281GetRxBufferStatus)
    i.SX1281GetStatus                        0x080037a4   Section        0  sx1281_driver.o(i.SX1281GetStatus)
    i.SX1281HalGetDioStatus                  0x080037bc   Section        0  sx1281_driver_hal.o(i.SX1281HalGetDioStatus)
    i.SX1281HalInit                          0x080037e0   Section        0  sx1281_driver_hal.o(i.SX1281HalInit)
    i.SX1281HalIoIrqInit                     0x080037f4   Section        0  sx1281_driver_hal.o(i.SX1281HalIoIrqInit)
    i.SX1281HalReadBuffer                    0x08003804   Section        0  sx1281_driver_hal.o(i.SX1281HalReadBuffer)
    i.SX1281HalReadCommand                   0x08003870   Section        0  sx1281_driver_hal.o(i.SX1281HalReadCommand)
    i.SX1281HalReadRegister                  0x080038dc   Section        0  sx1281_driver_hal.o(i.SX1281HalReadRegister)
    i.SX1281HalReadRegisters                 0x080038ec   Section        0  sx1281_driver_hal.o(i.SX1281HalReadRegisters)
    i.SX1281HalReset                         0x0800395c   Section        0  sx1281_driver_hal.o(i.SX1281HalReset)
    i.SX1281HalWaitOnBusy                    0x08003990   Section        0  sx1281_driver_hal.o(i.SX1281HalWaitOnBusy)
    i.SX1281HalWriteBuffer                   0x080039ac   Section        0  sx1281_driver_hal.o(i.SX1281HalWriteBuffer)
    i.SX1281HalWriteCommand                  0x080039f4   Section        0  sx1281_driver_hal.o(i.SX1281HalWriteCommand)
    i.SX1281HalWriteRegister                 0x08003a4c   Section        0  sx1281_driver_hal.o(i.SX1281HalWriteRegister)
    i.SX1281HalWriteRegisters                0x08003a58   Section        0  sx1281_driver_hal.o(i.SX1281HalWriteRegisters)
    i.SX1281Init                             0x08003aa8   Section        0  sx1281_driver.o(i.SX1281Init)
    i.SX1281OnDioIrq                         0x08003ab8   Section        0  sx1281_driver.o(i.SX1281OnDioIrq)
    i.SX1281ProcessIrqs                      0x08003acc   Section        0  sx1281_driver.o(i.SX1281ProcessIrqs)
    i.SX1281SendPayload                      0x08003c18   Section        0  sx1281_driver.o(i.SX1281SendPayload)
    i.SX1281SetAutoFS                        0x08003c2a   Section        0  sx1281_driver.o(i.SX1281SetAutoFS)
    i.SX1281SetAutoTx                        0x08003c38   Section        0  sx1281_driver.o(i.SX1281SetAutoTx)
    i.SX1281SetBleAccessAddress              0x08003c52   Section        0  sx1281_driver.o(i.SX1281SetBleAccessAddress)
    i.SX1281SetBleAdvertizerAccessAddress    0x08003c88   Section        0  sx1281_driver.o(i.SX1281SetBleAdvertizerAccessAddress)
    i.SX1281SetBufferBaseAddresses           0x08003c94   Section        0  sx1281_driver.o(i.SX1281SetBufferBaseAddresses)
    i.SX1281SetCad                           0x08003cac   Section        0  sx1281_driver.o(i.SX1281SetCad)
    i.SX1281SetCadParams                     0x08003cc4   Section        0  sx1281_driver.o(i.SX1281SetCadParams)
    i.SX1281SetCrcPolynomial                 0x08003cdc   Section        0  sx1281_driver.o(i.SX1281SetCrcPolynomial)
    i.SX1281SetCrcSeed                       0x08003d04   Section        0  sx1281_driver.o(i.SX1281SetCrcSeed)
    i.SX1281SetDioIrqParams                  0x08003d2c   Section        0  sx1281_driver.o(i.SX1281SetDioIrqParams)
    i.SX1281SetFs                            0x08003d64   Section        0  sx1281_driver.o(i.SX1281SetFs)
    i.SX1281SetInterruptMode                 0x08003d7c   Section        0  sx1281_driver.o(i.SX1281SetInterruptMode)
    i.SX1281SetLongPreamble                  0x08003d88   Section        0  sx1281_driver.o(i.SX1281SetLongPreamble)
    i.SX1281SetModulationParams              0x08003d98   Section        0  sx1281_driver.o(i.SX1281SetModulationParams)
    i.SX1281SetPacketParams                  0x08003e2c   Section        0  sx1281_driver.o(i.SX1281SetPacketParams)
    i.SX1281SetPacketType                    0x08003f04   Section        0  sx1281_driver.o(i.SX1281SetPacketType)
    i.SX1281SetPayload                       0x08003f20   Section        0  sx1281_driver.o(i.SX1281SetPayload)
    i.SX1281SetPollingMode                   0x08003f2c   Section        0  sx1281_driver.o(i.SX1281SetPollingMode)
    i.SX1281SetRegistersDefault              0x08003f38   Section        0  sx1281_driver.o(i.SX1281SetRegistersDefault)
    i.SX1281SetRegulatorMode                 0x08003f5c   Section        0  sx1281_driver.o(i.SX1281SetRegulatorMode)
    i.SX1281SetRfFrequency                   0x08003f6c   Section        0  sx1281_driver.o(i.SX1281SetRfFrequency)
    i.SX1281SetRx                            0x08003fa0   Section        0  sx1281_driver.o(i.SX1281SetRx)
    i.SX1281SetRxDutyCycle                   0x08003fd0   Section        0  sx1281_driver.o(i.SX1281SetRxDutyCycle)
    i.SX1281SetSaveContext                   0x08004000   Section        0  sx1281_driver.o(i.SX1281SetSaveContext)
    i.SX1281SetSleep                         0x0800400c   Section        0  sx1281_driver.o(i.SX1281SetSleep)
    i.SX1281SetStandby                       0x08004044   Section        0  sx1281_driver.o(i.SX1281SetStandby)
    i.SX1281SetSyncWord                      0x08004068   Section        0  sx1281_driver.o(i.SX1281SetSyncWord)
    i.SX1281SetSyncWordErrorTolerance        0x080040d4   Section        0  sx1281_driver.o(i.SX1281SetSyncWordErrorTolerance)
    i.SX1281SetTx                            0x080040f8   Section        0  sx1281_driver.o(i.SX1281SetTx)
    i.SX1281SetTxContinuousPreamble          0x08004128   Section        0  sx1281_driver.o(i.SX1281SetTxContinuousPreamble)
    i.SX1281SetTxContinuousWave              0x08004132   Section        0  sx1281_driver.o(i.SX1281SetTxContinuousWave)
    i.SX1281SetTxParams                      0x0800413c   Section        0  sx1281_driver.o(i.SX1281SetTxParams)
    i.SX1281SetWhiteningSeed                 0x08004154   Section        0  sx1281_driver.o(i.SX1281SetWhiteningSeed)
    i.SX1281_BSPInit                         0x08004174   Section        0  sx1281_header.o(i.SX1281_BSPInit)
    i.SX1281_Callback                        0x08004184   Section        0  sx1281.o(i.SX1281_Callback)
    i.SX1281_GetState                        0x0800429c   Section        0  sx1281.o(i.SX1281_GetState)
    i.SX1281_Init                            0x080042b4   Section        0  sx1281.o(i.SX1281_Init)
    i.SX1281_Running                         0x08004580   Section        0  sx1281.o(i.SX1281_Running)
    i.SX1281_SetTX                           0x08004598   Section        0  sx1281.o(i.SX1281_SetTX)
    i.SpiIn                                  0x080045c8   Section        0  sx1281_driver_spi.o(i.SpiIn)
    i.SpiInOut                               0x080045e0   Section        0  sx1281_driver_spi.o(i.SpiInOut)
    i.SpiInit                                0x08004600   Section        0  sx1281_driver_spi.o(i.SpiInit)
    i.SysTick_Handler                        0x08004624   Section        0  stm32f1xx_it.o(i.SysTick_Handler)
    i.SystemClock_Config                     0x08004628   Section        0  main.o(i.SystemClock_Config)
    i.SystemInit                             0x08004688   Section        0  system_stm32f1xx.o(i.SystemInit)
    i.TIM_Base_SetConfig                     0x0800468c   Section        0  stm32f1xx_hal_tim.o(i.TIM_Base_SetConfig)
    i.TIM_ETR_SetConfig                      0x08004704   Section        0  stm32f1xx_hal_tim.o(i.TIM_ETR_SetConfig)
    i.TIM_ITRx_SetConfig                     0x08004718   Section        0  stm32f1xx_hal_tim.o(i.TIM_ITRx_SetConfig)
    TIM_ITRx_SetConfig                       0x08004719   Thumb Code    16  stm32f1xx_hal_tim.o(i.TIM_ITRx_SetConfig)
    i.TIM_OC1_SetConfig                      0x08004728   Section        0  stm32f1xx_hal_tim.o(i.TIM_OC1_SetConfig)
    TIM_OC1_SetConfig                        0x08004729   Thumb Code    74  stm32f1xx_hal_tim.o(i.TIM_OC1_SetConfig)
    i.TIM_OC2_SetConfig                      0x08004778   Section        0  stm32f1xx_hal_tim.o(i.TIM_OC2_SetConfig)
    i.TIM_OC3_SetConfig                      0x080047d0   Section        0  stm32f1xx_hal_tim.o(i.TIM_OC3_SetConfig)
    TIM_OC3_SetConfig                        0x080047d1   Thumb Code    82  stm32f1xx_hal_tim.o(i.TIM_OC3_SetConfig)
    i.TIM_OC4_SetConfig                      0x08004828   Section        0  stm32f1xx_hal_tim.o(i.TIM_OC4_SetConfig)
    TIM_OC4_SetConfig                        0x08004829   Thumb Code    64  stm32f1xx_hal_tim.o(i.TIM_OC4_SetConfig)
    i.TIM_TI1_ConfigInputStage               0x0800486c   Section        0  stm32f1xx_hal_tim.o(i.TIM_TI1_ConfigInputStage)
    TIM_TI1_ConfigInputStage                 0x0800486d   Thumb Code    34  stm32f1xx_hal_tim.o(i.TIM_TI1_ConfigInputStage)
    i.TIM_TI2_ConfigInputStage               0x0800488e   Section        0  stm32f1xx_hal_tim.o(i.TIM_TI2_ConfigInputStage)
    TIM_TI2_ConfigInputStage                 0x0800488f   Thumb Code    36  stm32f1xx_hal_tim.o(i.TIM_TI2_ConfigInputStage)
    i.UART_DMAAbortOnError                   0x080048b2   Section        0  stm32f1xx_hal_uart.o(i.UART_DMAAbortOnError)
    UART_DMAAbortOnError                     0x080048b3   Thumb Code    16  stm32f1xx_hal_uart.o(i.UART_DMAAbortOnError)
    i.UART_DMAError                          0x080048c2   Section        0  stm32f1xx_hal_uart.o(i.UART_DMAError)
    UART_DMAError                            0x080048c3   Thumb Code    74  stm32f1xx_hal_uart.o(i.UART_DMAError)
    i.UART_DMAReceiveCplt                    0x0800490c   Section        0  stm32f1xx_hal_uart.o(i.UART_DMAReceiveCplt)
    UART_DMAReceiveCplt                      0x0800490d   Thumb Code   134  stm32f1xx_hal_uart.o(i.UART_DMAReceiveCplt)
    i.UART_DMARxHalfCplt                     0x08004992   Section        0  stm32f1xx_hal_uart.o(i.UART_DMARxHalfCplt)
    UART_DMARxHalfCplt                       0x08004993   Thumb Code    30  stm32f1xx_hal_uart.o(i.UART_DMARxHalfCplt)
    i.UART_EndRxTransfer                     0x080049b0   Section        0  stm32f1xx_hal_uart.o(i.UART_EndRxTransfer)
    UART_EndRxTransfer                       0x080049b1   Thumb Code    78  stm32f1xx_hal_uart.o(i.UART_EndRxTransfer)
    i.UART_EndTxTransfer                     0x080049fe   Section        0  stm32f1xx_hal_uart.o(i.UART_EndTxTransfer)
    UART_EndTxTransfer                       0x080049ff   Thumb Code    28  stm32f1xx_hal_uart.o(i.UART_EndTxTransfer)
    i.UART_Get                               0x08004a1c   Section        0  uart.o(i.UART_Get)
    UART_Get                                 0x08004a1d   Thumb Code    16  uart.o(i.UART_Get)
    i.UART_Receive_IT                        0x08004a30   Section        0  stm32f1xx_hal_uart.o(i.UART_Receive_IT)
    UART_Receive_IT                          0x08004a31   Thumb Code   194  stm32f1xx_hal_uart.o(i.UART_Receive_IT)
    i.UART_SetConfig                         0x08004af4   Section        0  stm32f1xx_hal_uart.o(i.UART_SetConfig)
    UART_SetConfig                           0x08004af5   Thumb Code   178  stm32f1xx_hal_uart.o(i.UART_SetConfig)
    i.UART_Start_Receive_DMA                 0x08004bac   Section        0  stm32f1xx_hal_uart.o(i.UART_Start_Receive_DMA)
    i.UART_WaitOnFlagUntilTimeout            0x08004c3c   Section        0  stm32f1xx_hal_uart.o(i.UART_WaitOnFlagUntilTimeout)
    UART_WaitOnFlagUntilTimeout              0x08004c3d   Thumb Code   114  stm32f1xx_hal_uart.o(i.UART_WaitOnFlagUntilTimeout)
    i.USART2_IRQHandler                      0x08004cb0   Section        0  stm32f1xx_it.o(i.USART2_IRQHandler)
    i.USAR_UART_IDLECallback                 0x08004cc8   Section        0  usart.o(i.USAR_UART_IDLECallback)
    i.USER_UART_IRQHandler                   0x08004d58   Section        0  usart.o(i.USER_UART_IRQHandler)
    i.UsageFault_Handler                     0x08004da8   Section        0  stm32f1xx_it.o(i.UsageFault_Handler)
    i.__0printf                              0x08004dac   Section        0  printfa.o(i.__0printf)
    i.__NVIC_SetPriority                     0x08004dcc   Section        0  stm32f1xx_hal_cortex.o(i.__NVIC_SetPriority)
    __NVIC_SetPriority                       0x08004dcd   Thumb Code    32  stm32f1xx_hal_cortex.o(i.__NVIC_SetPriority)
    i.__scatterload_copy                     0x08004dec   Section       14  handlers.o(i.__scatterload_copy)
    i.__scatterload_null                     0x08004dfa   Section        2  handlers.o(i.__scatterload_null)
    i.__scatterload_zeroinit                 0x08004dfc   Section       14  handlers.o(i.__scatterload_zeroinit)
    i._fp_digits                             0x08004e0c   Section        0  printfa.o(i._fp_digits)
    _fp_digits                               0x08004e0d   Thumb Code   366  printfa.o(i._fp_digits)
    i._printf_core                           0x08004f90   Section        0  printfa.o(i._printf_core)
    _printf_core                             0x08004f91   Thumb Code  1704  printfa.o(i._printf_core)
    i._printf_post_padding                   0x08005644   Section        0  printfa.o(i._printf_post_padding)
    _printf_post_padding                     0x08005645   Thumb Code    36  printfa.o(i._printf_post_padding)
    i._printf_pre_padding                    0x08005668   Section        0  printfa.o(i._printf_pre_padding)
    _printf_pre_padding                      0x08005669   Thumb Code    46  printfa.o(i._printf_pre_padding)
    i.fputc                                  0x08005696   Section        0  sx1281_header.o(i.fputc)
    i.free                                   0x080056b0   Section        0  malloc.o(i.free)
    i.main                                   0x08005700   Section        0  main.o(i.main)
    i.malloc                                 0x080057a0   Section        0  malloc.o(i.malloc)
    i.tx_cplt_cb                             0x0800580c   Section        0  sx1281_driver_spi.o(i.tx_cplt_cb)
    tx_cplt_cb                               0x0800580d   Thumb Code     8  sx1281_driver_spi.o(i.tx_cplt_cb)
    i.txrx_cplt_cb                           0x08005818   Section        0  sx1281_driver_spi.o(i.txrx_cplt_cb)
    txrx_cplt_cb                             0x08005819   Thumb Code     8  sx1281_driver_spi.o(i.txrx_cplt_cb)
    .constdata                               0x08005824   Section       18  stm32f1xx_hal_rcc.o(.constdata)
    aPredivFactorTable                       0x08005824   Data           2  stm32f1xx_hal_rcc.o(.constdata)
    aPLLMULFactorTable                       0x08005826   Data          16  stm32f1xx_hal_rcc.o(.constdata)
    .constdata                               0x08005836   Section       16  system_stm32f1xx.o(.constdata)
    .constdata                               0x08005846   Section        8  system_stm32f1xx.o(.constdata)
    .constdata                               0x08005850   Section       81  sx1281.o(.constdata)
    .constdata                               0x080058a2   Section        4  sx1281_driver.o(.constdata)
    .constdata                               0x080058a8   Section      228  sx1281_driver_hal.o(.constdata)
    .constdata                               0x0800598c   Section    12160  lcd.o(.constdata)
    .constdata                               0x0800890c   Section      512  lcd.o(.constdata)
    .data                                    0x20000000   Section       12  stm32f1xx_hal.o(.data)
    .data                                    0x2000000c   Section        4  system_stm32f1xx.o(.data)
    .data                                    0x20000010   Section       40  sx1281.o(.data)
    .data                                    0x20000038   Section       16  sx1281_driver.o(.data)
    OperatingMode                            0x20000038   Data           1  sx1281_driver.o(.data)
    PacketType                               0x20000039   Data           1  sx1281_driver.o(.data)
    LoRaBandwidth                            0x2000003a   Data           1  sx1281_driver.o(.data)
    PollingMode                              0x2000003b   Data           1  sx1281_driver.o(.data)
    IrqState                                 0x2000003c   Data           1  sx1281_driver.o(.data)
    RadioCallbacks                           0x20000044   Data           4  sx1281_driver.o(.data)
    .data                                    0x20000048   Section        1  sx1281_driver_spi.o(.data)
    spi_done                                 0x20000048   Data           1  sx1281_driver_spi.o(.data)
    .data                                    0x20000049   Section        1  lcd.o(.data)
    lcd_orientation                          0x20000049   Data           1  lcd.o(.data)
    .data                                    0x2000004c   Section        4  stdout.o(.data)
    .data                                    0x20000050   Section        4  mvars.o(.data)
    .data                                    0x20000054   Section        4  mvars.o(.data)
    .bss                                     0x20000058   Section      320  main.o(.bss)
    .bss                                     0x20000198   Section      380  spi.o(.bss)
    .bss                                     0x20000314   Section       72  tim.o(.bss)
    .bss                                     0x2000035c   Section      790  usart.o(.bss)
    .bss                                     0x20000672   Section      255  sx1281.o(.bss)
    .bss                                     0x20000774   Section       64  sx1281_driver_gpio.o(.bss)
    GpioIrq                                  0x20000774   Data          64  sx1281_driver_gpio.o(.bss)
    .bss                                     0x200007b4   Section     8190  sx1281_driver_hal.o(.bss)
    halTxBuffer                              0x200007b4   Data        4095  sx1281_driver_hal.o(.bss)
    halRxBuffer                              0x200017b3   Data        4095  sx1281_driver_hal.o(.bss)
    .bss                                     0x200027b4   Section       64  gpio_1.o(.bss)
    GPIO_Callback                            0x200027b4   Data          64  gpio_1.o(.bss)
    .bss                                     0x200027f4   Section       64  spi_1.o(.bss)
    SPI_Callback                             0x200027f4   Data          64  spi_1.o(.bss)
    .bss                                     0x20002834   Section       36  uart.o(.bss)
    UART_Callback                            0x20002834   Data          36  uart.o(.bss)
    HEAP                                     0x20002858   Section      512  startup_stm32f103xb.o(HEAP)
    STACK                                    0x20002a58   Section     1024  startup_stm32f103xb.o(STACK)

    Global Symbols

    Symbol Name                              Value     Ov Type        Size  Object(Section)

    BuildAttributes$$THM_ISAv4$P$D$K$B$S$PE$A:L22UL41UL21$X:L11$S22US41US21$IEEE1$IW$USESV6$~STKCKD$USESV7$~SHL$OTIME$ROPI$EBA8$MICROLIB$REQ8$PRES8$EABIv2 0x00000000   Number         0  anon$$obj.o ABSOLUTE
    __ARM_use_no_argv                        0x00000000   Number         0  main.o ABSOLUTE
    _printf_a                                0x00000000   Number         0  stubs.o ABSOLUTE
    _printf_c                                0x00000000   Number         0  stubs.o ABSOLUTE
    _printf_charcount                        0x00000000   Number         0  stubs.o ABSOLUTE
    _printf_d                                0x00000000   Number         0  stubs.o ABSOLUTE
    _printf_e                                0x00000000   Number         0  stubs.o ABSOLUTE
    _printf_f                                0x00000000   Number         0  stubs.o ABSOLUTE
    _printf_flags                            0x00000000   Number         0  stubs.o ABSOLUTE
    _printf_fp_dec                           0x00000000   Number         0  stubs.o ABSOLUTE
    _printf_fp_hex                           0x00000000   Number         0  stubs.o ABSOLUTE
    _printf_g                                0x00000000   Number         0  stubs.o ABSOLUTE
    _printf_i                                0x00000000   Number         0  stubs.o ABSOLUTE
    _printf_int_dec                          0x00000000   Number         0  stubs.o ABSOLUTE
    _printf_l                                0x00000000   Number         0  stubs.o ABSOLUTE
    _printf_lc                               0x00000000   Number         0  stubs.o ABSOLUTE
    _printf_ll                               0x00000000   Number         0  stubs.o ABSOLUTE
    _printf_lld                              0x00000000   Number         0  stubs.o ABSOLUTE
    _printf_lli                              0x00000000   Number         0  stubs.o ABSOLUTE
    _printf_llo                              0x00000000   Number         0  stubs.o ABSOLUTE
    _printf_llu                              0x00000000   Number         0  stubs.o ABSOLUTE
    _printf_llx                              0x00000000   Number         0  stubs.o ABSOLUTE
    _printf_longlong_dec                     0x00000000   Number         0  stubs.o ABSOLUTE
    _printf_longlong_hex                     0x00000000   Number         0  stubs.o ABSOLUTE
    _printf_longlong_oct                     0x00000000   Number         0  stubs.o ABSOLUTE
    _printf_ls                               0x00000000   Number         0  stubs.o ABSOLUTE
    _printf_mbtowc                           0x00000000   Number         0  stubs.o ABSOLUTE
    _printf_n                                0x00000000   Number         0  stubs.o ABSOLUTE
    _printf_o                                0x00000000   Number         0  stubs.o ABSOLUTE
    _printf_p                                0x00000000   Number         0  stubs.o ABSOLUTE
    _printf_percent                          0x00000000   Number         0  stubs.o ABSOLUTE
    _printf_pre_padding                      0x00000000   Number         0  stubs.o ABSOLUTE
    _printf_return_value                     0x00000000   Number         0  stubs.o ABSOLUTE
    _printf_s                                0x00000000   Number         0  stubs.o ABSOLUTE
    _printf_sizespec                         0x00000000   Number         0  stubs.o ABSOLUTE
    _printf_str                              0x00000000   Number         0  stubs.o ABSOLUTE
    _printf_truncate_signed                  0x00000000   Number         0  stubs.o ABSOLUTE
    _printf_truncate_unsigned                0x00000000   Number         0  stubs.o ABSOLUTE
    _printf_u                                0x00000000   Number         0  stubs.o ABSOLUTE
    _printf_wc                               0x00000000   Number         0  stubs.o ABSOLUTE
    _printf_wctomb                           0x00000000   Number         0  stubs.o ABSOLUTE
    _printf_widthprec                        0x00000000   Number         0  stubs.o ABSOLUTE
    _printf_x                                0x00000000   Number         0  stubs.o ABSOLUTE
    __arm_fini_                               - Undefined Weak Reference
    __cpp_initialize__aeabi_                  - Undefined Weak Reference
    __cxa_finalize                            - Undefined Weak Reference
    __decompress                              - Undefined Weak Reference
    _clock_init                               - Undefined Weak Reference
    _microlib_exit                            - Undefined Weak Reference
    _scanf_longlong                           - Undefined Weak Reference
    _scanf_real                               - Undefined Weak Reference
    _scanf_string                             - Undefined Weak Reference
    __Vectors_Size                           0x000000ec   Number         0  startup_stm32f103xb.o ABSOLUTE
    __Vectors                                0x08000000   Data           4  startup_stm32f103xb.o(RESET)
    __Vectors_End                            0x080000ec   Data           0  startup_stm32f103xb.o(RESET)
    __main                                   0x080000ed   Thumb Code     0  entry.o(.ARM.Collect$$$$00000000)
    _main_stk                                0x080000ed   Thumb Code     0  entry2.o(.ARM.Collect$$$$00000001)
    _main_scatterload                        0x080000f1   Thumb Code     0  entry5.o(.ARM.Collect$$$$00000004)
    __main_after_scatterload                 0x080000f5   Thumb Code     0  entry5.o(.ARM.Collect$$$$00000004)
    _main_clock                              0x080000f5   Thumb Code     0  entry7b.o(.ARM.Collect$$$$00000008)
    _main_cpp_init                           0x080000f5   Thumb Code     0  entry8b.o(.ARM.Collect$$$$0000000A)
    _main_init                               0x080000f5   Thumb Code     0  entry9a.o(.ARM.Collect$$$$0000000B)
    __rt_lib_shutdown_fini                   0x080000fd   Thumb Code     0  entry12b.o(.ARM.Collect$$$$0000000E)
    __rt_final_cpp                           0x08000101   Thumb Code     0  entry10a.o(.ARM.Collect$$$$0000000F)
    __rt_final_exit                          0x08000101   Thumb Code     0  entry11a.o(.ARM.Collect$$$$00000011)
    Reset_Handler                            0x08000105   Thumb Code     8  startup_stm32f103xb.o(.text)
    ADC1_2_IRQHandler                        0x0800011f   Thumb Code     0  startup_stm32f103xb.o(.text)
    CAN1_RX1_IRQHandler                      0x0800011f   Thumb Code     0  startup_stm32f103xb.o(.text)
    CAN1_SCE_IRQHandler                      0x0800011f   Thumb Code     0  startup_stm32f103xb.o(.text)
    DMA1_Channel1_IRQHandler                 0x0800011f   Thumb Code     0  startup_stm32f103xb.o(.text)
    DMA1_Channel4_IRQHandler                 0x0800011f   Thumb Code     0  startup_stm32f103xb.o(.text)
    EXTI0_IRQHandler                         0x0800011f   Thumb Code     0  startup_stm32f103xb.o(.text)
    EXTI1_IRQHandler                         0x0800011f   Thumb Code     0  startup_stm32f103xb.o(.text)
    EXTI2_IRQHandler                         0x0800011f   Thumb Code     0  startup_stm32f103xb.o(.text)
    EXTI3_IRQHandler                         0x0800011f   Thumb Code     0  startup_stm32f103xb.o(.text)
    EXTI4_IRQHandler                         0x0800011f   Thumb Code     0  startup_stm32f103xb.o(.text)
    FLASH_IRQHandler                         0x0800011f   Thumb Code     0  startup_stm32f103xb.o(.text)
    I2C1_ER_IRQHandler                       0x0800011f   Thumb Code     0  startup_stm32f103xb.o(.text)
    I2C1_EV_IRQHandler                       0x0800011f   Thumb Code     0  startup_stm32f103xb.o(.text)
    I2C2_ER_IRQHandler                       0x0800011f   Thumb Code     0  startup_stm32f103xb.o(.text)
    I2C2_EV_IRQHandler                       0x0800011f   Thumb Code     0  startup_stm32f103xb.o(.text)
    PVD_IRQHandler                           0x0800011f   Thumb Code     0  startup_stm32f103xb.o(.text)
    RCC_IRQHandler                           0x0800011f   Thumb Code     0  startup_stm32f103xb.o(.text)
    RTC_Alarm_IRQHandler                     0x0800011f   Thumb Code     0  startup_stm32f103xb.o(.text)
    RTC_IRQHandler                           0x0800011f   Thumb Code     0  startup_stm32f103xb.o(.text)
    SPI1_IRQHandler                          0x0800011f   Thumb Code     0  startup_stm32f103xb.o(.text)
    SPI2_IRQHandler                          0x0800011f   Thumb Code     0  startup_stm32f103xb.o(.text)
    TAMPER_IRQHandler                        0x0800011f   Thumb Code     0  startup_stm32f103xb.o(.text)
    TIM1_BRK_IRQHandler                      0x0800011f   Thumb Code     0  startup_stm32f103xb.o(.text)
    TIM1_CC_IRQHandler                       0x0800011f   Thumb Code     0  startup_stm32f103xb.o(.text)
    TIM1_TRG_COM_IRQHandler                  0x0800011f   Thumb Code     0  startup_stm32f103xb.o(.text)
    TIM1_UP_IRQHandler                       0x0800011f   Thumb Code     0  startup_stm32f103xb.o(.text)
    TIM2_IRQHandler                          0x0800011f   Thumb Code     0  startup_stm32f103xb.o(.text)
    TIM3_IRQHandler                          0x0800011f   Thumb Code     0  startup_stm32f103xb.o(.text)
    TIM4_IRQHandler                          0x0800011f   Thumb Code     0  startup_stm32f103xb.o(.text)
    USART1_IRQHandler                        0x0800011f   Thumb Code     0  startup_stm32f103xb.o(.text)
    USART3_IRQHandler                        0x0800011f   Thumb Code     0  startup_stm32f103xb.o(.text)
    USBWakeUp_IRQHandler                     0x0800011f   Thumb Code     0  startup_stm32f103xb.o(.text)
    USB_HP_CAN1_TX_IRQHandler                0x0800011f   Thumb Code     0  startup_stm32f103xb.o(.text)
    USB_LP_CAN1_RX0_IRQHandler               0x0800011f   Thumb Code     0  startup_stm32f103xb.o(.text)
    WWDG_IRQHandler                          0x0800011f   Thumb Code     0  startup_stm32f103xb.o(.text)
    __aeabi_llsr                             0x08000129   Thumb Code    32  llushr.o(.text)
    _ll_ushift_r                             0x08000129   Thumb Code     0  llushr.o(.text)
    __aeabi_memcpy                           0x08000149   Thumb Code    36  memcpya.o(.text)
    __aeabi_memcpy4                          0x08000149   Thumb Code     0  memcpya.o(.text)
    __aeabi_memcpy8                          0x08000149   Thumb Code     0  memcpya.o(.text)
    __aeabi_memset                           0x0800016d   Thumb Code    14  memseta.o(.text)
    __aeabi_memset4                          0x0800016d   Thumb Code     0  memseta.o(.text)
    __aeabi_memset8                          0x0800016d   Thumb Code     0  memseta.o(.text)
    __aeabi_memclr                           0x0800017b   Thumb Code     4  memseta.o(.text)
    __aeabi_memclr4                          0x0800017b   Thumb Code     0  memseta.o(.text)
    __aeabi_memclr8                          0x0800017b   Thumb Code     0  memseta.o(.text)
    _memset$wrapper                          0x0800017f   Thumb Code    18  memseta.o(.text)
    strcpy                                   0x08000191   Thumb Code    18  strcpy.o(.text)
    __aeabi_dmul                             0x080001a3   Thumb Code   228  dmul.o(.text)
    __aeabi_ddiv                             0x08000287   Thumb Code   222  ddiv.o(.text)
    __aeabi_i2d                              0x08000365   Thumb Code    34  dflti.o(.text)
    __aeabi_ui2d                             0x08000387   Thumb Code    26  dfltui.o(.text)
    __aeabi_d2uiz                            0x080003a1   Thumb Code    50  dfixui.o(.text)
    __aeabi_uidiv                            0x080003d3   Thumb Code     0  uidiv.o(.text)
    __aeabi_uidivmod                         0x080003d3   Thumb Code    44  uidiv.o(.text)
    __aeabi_uldivmod                         0x080003ff   Thumb Code    98  uldiv.o(.text)
    __I$use$fp                               0x08000461   Thumb Code     0  iusefp.o(.text)
    _double_round                            0x08000461   Thumb Code    30  depilogue.o(.text)
    _double_epilogue                         0x0800047f   Thumb Code   156  depilogue.o(.text)
    __aeabi_dadd                             0x0800051b   Thumb Code   322  dadd.o(.text)
    __aeabi_dsub                             0x0800065d   Thumb Code     6  dadd.o(.text)
    __aeabi_drsub                            0x08000663   Thumb Code     6  dadd.o(.text)
    __aeabi_d2ulz                            0x08000669   Thumb Code    48  dfixul.o(.text)
    __aeabi_cdrcmple                         0x08000699   Thumb Code    48  cdrcmple.o(.text)
    __scatterload                            0x080006c9   Thumb Code    28  init.o(.text)
    __scatterload_rt2                        0x080006c9   Thumb Code     0  init.o(.text)
    __aeabi_llsl                             0x080006ed   Thumb Code    30  llshl.o(.text)
    _ll_shift_l                              0x080006ed   Thumb Code     0  llshl.o(.text)
    __aeabi_lasr                             0x0800070b   Thumb Code    36  llsshr.o(.text)
    _ll_sshift_r                             0x0800070b   Thumb Code     0  llsshr.o(.text)
    BSP_SPI_GetHandle                        0x08000731   Thumb Code    18  spi_1.o(i.BSP_SPI_GetHandle)
    BSP_SPI_GetState                         0x0800074d   Thumb Code    24  spi_1.o(i.BSP_SPI_GetState)
    BSP_SPI_RegisterCallback                 0x08000765   Thumb Code    22  spi_1.o(i.BSP_SPI_RegisterCallback)
    BSP_SPI_Transmit                         0x08000781   Thumb Code    42  spi_1.o(i.BSP_SPI_Transmit)
    BSP_SPI_TransmitReceive                  0x080007ab   Thumb Code    46  spi_1.o(i.BSP_SPI_TransmitReceive)
    BSP_UART_GetHandle                       0x080007d9   Thumb Code    10  uart.o(i.BSP_UART_GetHandle)
    BusFault_Handler                         0x080007e9   Thumb Code     2  stm32f1xx_it.o(i.BusFault_Handler)
    DMA1_Channel2_IRQHandler                 0x080007ed   Thumb Code     6  stm32f1xx_it.o(i.DMA1_Channel2_IRQHandler)
    DMA1_Channel3_IRQHandler                 0x080007f9   Thumb Code     6  stm32f1xx_it.o(i.DMA1_Channel3_IRQHandler)
    DMA1_Channel5_IRQHandler                 0x08000805   Thumb Code     6  stm32f1xx_it.o(i.DMA1_Channel5_IRQHandler)
    DMA1_Channel6_IRQHandler                 0x08000811   Thumb Code     6  stm32f1xx_it.o(i.DMA1_Channel6_IRQHandler)
    DMA1_Channel7_IRQHandler                 0x0800081d   Thumb Code     6  stm32f1xx_it.o(i.DMA1_Channel7_IRQHandler)
    DebugMon_Handler                         0x08000853   Thumb Code     2  stm32f1xx_it.o(i.DebugMon_Handler)
    EXTI15_10_IRQHandler                     0x08000855   Thumb Code     8  stm32f1xx_it.o(i.EXTI15_10_IRQHandler)
    EXTI9_5_IRQHandler                       0x0800085d   Thumb Code    24  stm32f1xx_it.o(i.EXTI9_5_IRQHandler)
    Error_Handler                            0x08000875   Thumb Code     4  main.o(i.Error_Handler)
    GpioGetBitPos                            0x08000879   Thumb Code    48  sx1281_driver_gpio.o(i.GpioGetBitPos)
    GpioInit                                 0x080008a9   Thumb Code     2  sx1281_driver_gpio.o(i.GpioInit)
    GpioRead                                 0x080008ab   Thumb Code     4  sx1281_driver_gpio.o(i.GpioRead)
    GpioSetIrq                               0x080008b1   Thumb Code    50  sx1281_driver_gpio.o(i.GpioSetIrq)
    GpioWrite                                0x080008e9   Thumb Code     6  sx1281_driver_gpio.o(i.GpioWrite)
    HAL_DMA_Abort                            0x080008ef   Thumb Code    70  stm32f1xx_hal_dma.o(i.HAL_DMA_Abort)
    HAL_DMA_Abort_IT                         0x08000935   Thumb Code   148  stm32f1xx_hal_dma.o(i.HAL_DMA_Abort_IT)
    HAL_DMA_IRQHandler                       0x080009cd   Thumb Code   316  stm32f1xx_hal_dma.o(i.HAL_DMA_IRQHandler)
    HAL_DMA_Init                             0x08000b21   Thumb Code    84  stm32f1xx_hal_dma.o(i.HAL_DMA_Init)
    HAL_DMA_Start_IT                         0x08000b7d   Thumb Code   112  stm32f1xx_hal_dma.o(i.HAL_DMA_Start_IT)
    HAL_Delay                                0x08000bed   Thumb Code    32  stm32f1xx_hal.o(i.HAL_Delay)
    HAL_GPIO_EXTI_Callback                   0x08000c11   Thumb Code    40  gpio_1.o(i.HAL_GPIO_EXTI_Callback)
    HAL_GPIO_EXTI_IRQHandler                 0x08000c3d   Thumb Code    18  stm32f1xx_hal_gpio.o(i.HAL_GPIO_EXTI_IRQHandler)
    HAL_GPIO_Init                            0x08000c55   Thumb Code   446  stm32f1xx_hal_gpio.o(i.HAL_GPIO_Init)
    HAL_GPIO_ReadPin                         0x08000e35   Thumb Code    10  stm32f1xx_hal_gpio.o(i.HAL_GPIO_ReadPin)
    HAL_GPIO_WritePin                        0x08000e3f   Thumb Code    10  stm32f1xx_hal_gpio.o(i.HAL_GPIO_WritePin)
    HAL_GetTick                              0x08000e49   Thumb Code     6  stm32f1xx_hal.o(i.HAL_GetTick)
    HAL_HalfDuplex_Init                      0x08000e55   Thumb Code   110  stm32f1xx_hal_uart.o(i.HAL_HalfDuplex_Init)
    HAL_IncTick                              0x08000ec5   Thumb Code    12  stm32f1xx_hal.o(i.HAL_IncTick)
    HAL_Init                                 0x08000ed5   Thumb Code    32  stm32f1xx_hal.o(i.HAL_Init)
    HAL_InitTick                             0x08000ef9   Thumb Code    54  stm32f1xx_hal.o(i.HAL_InitTick)
    HAL_MspInit                              0x08000f39   Thumb Code    52  stm32f1xx_hal_msp.o(i.HAL_MspInit)
    HAL_NVIC_EnableIRQ                       0x08000f75   Thumb Code    26  stm32f1xx_hal_cortex.o(i.HAL_NVIC_EnableIRQ)
    HAL_NVIC_SetPriority                     0x08000f91   Thumb Code    60  stm32f1xx_hal_cortex.o(i.HAL_NVIC_SetPriority)
    HAL_NVIC_SetPriorityGrouping             0x08000fd1   Thumb Code    26  stm32f1xx_hal_cortex.o(i.HAL_NVIC_SetPriorityGrouping)
    HAL_RCC_ClockConfig                      0x08000ff5   Thumb Code   280  stm32f1xx_hal_rcc.o(i.HAL_RCC_ClockConfig)
    HAL_RCC_GetPCLK1Freq                     0x08001121   Thumb Code    20  stm32f1xx_hal_rcc.o(i.HAL_RCC_GetPCLK1Freq)
    HAL_RCC_GetPCLK2Freq                     0x08001141   Thumb Code    20  stm32f1xx_hal_rcc.o(i.HAL_RCC_GetPCLK2Freq)
    HAL_RCC_GetSysClockFreq                  0x08001161   Thumb Code    64  stm32f1xx_hal_rcc.o(i.HAL_RCC_GetSysClockFreq)
    HAL_RCC_OscConfig                        0x080011b5   Thumb Code   778  stm32f1xx_hal_rcc.o(i.HAL_RCC_OscConfig)
    HAL_SPI_ErrorCallback                    0x080014d5   Thumb Code    50  spi_1.o(i.HAL_SPI_ErrorCallback)
    HAL_SPI_GetState                         0x0800150d   Thumb Code     6  stm32f1xx_hal_spi.o(i.HAL_SPI_GetState)
    HAL_SPI_Init                             0x08001513   Thumb Code   178  stm32f1xx_hal_spi.o(i.HAL_SPI_Init)
    HAL_SPI_MspInit                          0x080015c5   Thumb Code   284  spi.o(i.HAL_SPI_MspInit)
    HAL_SPI_RxCpltCallback                   0x080016fd   Thumb Code    50  spi_1.o(i.HAL_SPI_RxCpltCallback)
    HAL_SPI_RxHalfCpltCallback               0x08001735   Thumb Code    50  spi_1.o(i.HAL_SPI_RxHalfCpltCallback)
    HAL_SPI_Transmit                         0x0800176d   Thumb Code   358  stm32f1xx_hal_spi.o(i.HAL_SPI_Transmit)
    HAL_SPI_TransmitReceive                  0x080018d3   Thumb Code   496  stm32f1xx_hal_spi.o(i.HAL_SPI_TransmitReceive)
    HAL_SPI_TransmitReceive_DMA              0x08001ac5   Thumb Code   252  stm32f1xx_hal_spi.o(i.HAL_SPI_TransmitReceive_DMA)
    HAL_SPI_Transmit_DMA                     0x08001bd5   Thumb Code   190  stm32f1xx_hal_spi.o(i.HAL_SPI_Transmit_DMA)
    HAL_SPI_TxCpltCallback                   0x08001ca1   Thumb Code    30  spi_1.o(i.HAL_SPI_TxCpltCallback)
    HAL_SPI_TxHalfCpltCallback               0x08001cc5   Thumb Code    50  spi_1.o(i.HAL_SPI_TxHalfCpltCallback)
    HAL_SPI_TxRxCpltCallback                 0x08001cfd   Thumb Code    50  spi_1.o(i.HAL_SPI_TxRxCpltCallback)
    HAL_SPI_TxRxHalfCpltCallback             0x08001d35   Thumb Code    50  spi_1.o(i.HAL_SPI_TxRxHalfCpltCallback)
    HAL_SYSTICK_Config                       0x08001d6d   Thumb Code    40  stm32f1xx_hal_cortex.o(i.HAL_SYSTICK_Config)
    HAL_TIMEx_ConfigBreakDeadTime            0x08001d95   Thumb Code    84  stm32f1xx_hal_tim_ex.o(i.HAL_TIMEx_ConfigBreakDeadTime)
    HAL_TIMEx_MasterConfigSynchronization    0x08001de9   Thumb Code    92  stm32f1xx_hal_tim_ex.o(i.HAL_TIMEx_MasterConfigSynchronization)
    HAL_TIM_Base_Init                        0x08001e51   Thumb Code    90  stm32f1xx_hal_tim.o(i.HAL_TIM_Base_Init)
    HAL_TIM_Base_MspInit                     0x08001ead   Thumb Code    30  tim.o(i.HAL_TIM_Base_MspInit)
    HAL_TIM_ConfigClockSource                0x08001ed5   Thumb Code   220  stm32f1xx_hal_tim.o(i.HAL_TIM_ConfigClockSource)
    HAL_TIM_MspPostInit                      0x08001fb1   Thumb Code    64  tim.o(i.HAL_TIM_MspPostInit)
    HAL_TIM_PWM_ConfigChannel                0x08001ffd   Thumb Code   204  stm32f1xx_hal_tim.o(i.HAL_TIM_PWM_ConfigChannel)
    HAL_TIM_PWM_Init                         0x080020c9   Thumb Code    90  stm32f1xx_hal_tim.o(i.HAL_TIM_PWM_Init)
    HAL_TIM_PWM_MspInit                      0x08002123   Thumb Code     2  stm32f1xx_hal_tim.o(i.HAL_TIM_PWM_MspInit)
    HAL_UARTEx_RxEventCallback               0x08002125   Thumb Code     2  stm32f1xx_hal_uart.o(i.HAL_UARTEx_RxEventCallback)
    HAL_UART_DMAStop                         0x08002127   Thumb Code   112  stm32f1xx_hal_uart.o(i.HAL_UART_DMAStop)
    HAL_UART_ErrorCallback                   0x08002199   Thumb Code    34  uart.o(i.HAL_UART_ErrorCallback)
    HAL_UART_IRQHandler                      0x080021c1   Thumb Code   616  stm32f1xx_hal_uart.o(i.HAL_UART_IRQHandler)
    HAL_UART_Init                            0x0800242d   Thumb Code   100  stm32f1xx_hal_uart.o(i.HAL_UART_Init)
    HAL_UART_MspInit                         0x08002491   Thumb Code   254  usart.o(i.HAL_UART_MspInit)
    HAL_UART_Receive_DMA                     0x080025a9   Thumb Code    28  stm32f1xx_hal_uart.o(i.HAL_UART_Receive_DMA)
    HAL_UART_RxCpltCallback                  0x080025c5   Thumb Code    34  uart.o(i.HAL_UART_RxCpltCallback)
    HAL_UART_RxHalfCpltCallback              0x080025ed   Thumb Code    34  uart.o(i.HAL_UART_RxHalfCpltCallback)
    HAL_UART_Transmit                        0x08002615   Thumb Code   160  stm32f1xx_hal_uart.o(i.HAL_UART_Transmit)
    HAL_UART_TxCpltCallback                  0x080026b5   Thumb Code    34  uart.o(i.HAL_UART_TxCpltCallback)
    HardFault_Handler                        0x080026dd   Thumb Code     2  stm32f1xx_it.o(i.HardFault_Handler)
    LCD_Clear                                0x080026df   Thumb Code    82  lcd.o(i.LCD_Clear)
    LCD_DrawBitmap                           0x08002731   Thumb Code   128  lcd.o(i.LCD_DrawBitmap)
    LCD_DrawChar                             0x080027b1   Thumb Code   342  lcd.o(i.LCD_DrawChar)
    LCD_DrawPoint                            0x08002915   Thumb Code    88  lcd.o(i.LCD_DrawPoint)
    LCD_DrawString                           0x08002971   Thumb Code   110  lcd.o(i.LCD_DrawString)
    LCD_Init                                 0x080029e1   Thumb Code   304  lcd.o(i.LCD_Init)
    MSP_GetIRQn                              0x08002cc5   Thumb Code    58  sx1281_driver_gpio.o(i.MSP_GetIRQn)
    MX_DMA_Init                              0x08002d01   Thumb Code   104  dma.o(i.MX_DMA_Init)
    MX_GPIO_Init                             0x08002d6d   Thumb Code   258  gpio.o(i.MX_GPIO_Init)
    MX_SPI1_Init                             0x08002e85   Thumb Code    62  spi.o(i.MX_SPI1_Init)
    MX_SPI2_Init                             0x08002ecd   Thumb Code    62  spi.o(i.MX_SPI2_Init)
    MX_TIM1_Init                             0x08002f15   Thumb Code   188  tim.o(i.MX_TIM1_Init)
    MX_USART1_UART_Init                      0x08002fd9   Thumb Code    48  usart.o(i.MX_USART1_UART_Init)
    MX_USART2_UART_Init                      0x08003011   Thumb Code    48  usart.o(i.MX_USART2_UART_Init)
    MemManage_Handler                        0x08003049   Thumb Code     2  stm32f1xx_it.o(i.MemManage_Handler)
    NMI_Handler                              0x0800304b   Thumb Code     2  stm32f1xx_it.o(i.NMI_Handler)
    OnRxDone                                 0x0800304d   Thumb Code    14  sx1281.o(i.OnRxDone)
    OnRxError                                0x08003061   Thumb Code    14  sx1281.o(i.OnRxError)
    OnRxTimeout                              0x08003075   Thumb Code    14  sx1281.o(i.OnRxTimeout)
    OnTxDone                                 0x08003089   Thumb Code    14  sx1281.o(i.OnTxDone)
    OnTxTimeout                              0x0800309d   Thumb Code    14  sx1281.o(i.OnTxTimeout)
    PendSV_Handler                           0x080030b1   Thumb Code     2  stm32f1xx_it.o(i.PendSV_Handler)
    SVC_Handler                              0x08003389   Thumb Code     2  stm32f1xx_it.o(i.SVC_Handler)
    SX1281Calibrate                          0x0800338b   Thumb Code    62  sx1281_driver.o(i.SX1281Calibrate)
    SX1281ClearIrqStatus                     0x080033c9   Thumb Code    24  sx1281_driver.o(i.SX1281ClearIrqStatus)
    SX1281GetFirmwareVersion                 0x080033e1   Thumb Code    26  sx1281_driver.o(i.SX1281GetFirmwareVersion)
    SX1281GetFrequencyError                  0x080033fd   Thumb Code   132  sx1281_driver.o(i.SX1281GetFrequencyError)
    SX1281GetIrqStatus                       0x08003495   Thumb Code    20  sx1281_driver.o(i.SX1281GetIrqStatus)
    SX1281GetLoRaBandwidth                   0x080034a9   Thumb Code    38  sx1281_driver.o(i.SX1281GetLoRaBandwidth)
    SX1281GetOpMode                          0x080034e5   Thumb Code     6  sx1281_driver.o(i.SX1281GetOpMode)
    SX1281GetPacketStatus                    0x080034f1   Thumb Code   526  sx1281_driver.o(i.SX1281GetPacketStatus)
    SX1281GetPacketType                      0x08003705   Thumb Code     6  sx1281_driver.o(i.SX1281GetPacketType)
    SX1281GetPayload                         0x08003711   Thumb Code    40  sx1281_driver.o(i.SX1281GetPayload)
    SX1281GetRssiInst                        0x08003739   Thumb Code    34  sx1281_driver.o(i.SX1281GetRssiInst)
    SX1281GetRxBufferStatus                  0x0800375d   Thumb Code    68  sx1281_driver.o(i.SX1281GetRxBufferStatus)
    SX1281GetStatus                          0x080037a5   Thumb Code    24  sx1281_driver.o(i.SX1281GetStatus)
    SX1281HalGetDioStatus                    0x080037bd   Thumb Code    32  sx1281_driver_hal.o(i.SX1281HalGetDioStatus)
    SX1281HalInit                            0x080037e1   Thumb Code    18  sx1281_driver_hal.o(i.SX1281HalInit)
    SX1281HalIoIrqInit                       0x080037f5   Thumb Code    12  sx1281_driver_hal.o(i.SX1281HalIoIrqInit)
    SX1281HalReadBuffer                      0x08003805   Thumb Code    96  sx1281_driver_hal.o(i.SX1281HalReadBuffer)
    SX1281HalReadCommand                     0x08003871   Thumb Code    94  sx1281_driver_hal.o(i.SX1281HalReadCommand)
    SX1281HalReadRegister                    0x080038dd   Thumb Code    16  sx1281_driver_hal.o(i.SX1281HalReadRegister)
    SX1281HalReadRegisters                   0x080038ed   Thumb Code   100  sx1281_driver_hal.o(i.SX1281HalReadRegisters)
    SX1281HalReset                           0x0800395d   Thumb Code    46  sx1281_driver_hal.o(i.SX1281HalReset)
    SX1281HalWaitOnBusy                      0x08003991   Thumb Code    22  sx1281_driver_hal.o(i.SX1281HalWaitOnBusy)
    SX1281HalWriteBuffer                     0x080039ad   Thumb Code    64  sx1281_driver_hal.o(i.SX1281HalWriteBuffer)
    SX1281HalWriteCommand                    0x080039f5   Thumb Code    78  sx1281_driver_hal.o(i.SX1281HalWriteCommand)
    SX1281HalWriteRegister                   0x08003a4d   Thumb Code    12  sx1281_driver_hal.o(i.SX1281HalWriteRegister)
    SX1281HalWriteRegisters                  0x08003a59   Thumb Code    72  sx1281_driver_hal.o(i.SX1281HalWriteRegisters)
    SX1281Init                               0x08003aa9   Thumb Code    12  sx1281_driver.o(i.SX1281Init)
    SX1281OnDioIrq                           0x08003ab9   Thumb Code    16  sx1281_driver.o(i.SX1281OnDioIrq)
    SX1281ProcessIrqs                        0x08003acd   Thumb Code   328  sx1281_driver.o(i.SX1281ProcessIrqs)
    SX1281SendPayload                        0x08003c19   Thumb Code    18  sx1281_driver.o(i.SX1281SendPayload)
    SX1281SetAutoFS                          0x08003c2b   Thumb Code    14  sx1281_driver.o(i.SX1281SetAutoFS)
    SX1281SetAutoTx                          0x08003c39   Thumb Code    26  sx1281_driver.o(i.SX1281SetAutoTx)
    SX1281SetBleAccessAddress                0x08003c53   Thumb Code    52  sx1281_driver.o(i.SX1281SetBleAccessAddress)
    SX1281SetBleAdvertizerAccessAddress      0x08003c89   Thumb Code     6  sx1281_driver.o(i.SX1281SetBleAdvertizerAccessAddress)
    SX1281SetBufferBaseAddresses             0x08003c95   Thumb Code    22  sx1281_driver.o(i.SX1281SetBufferBaseAddresses)
    SX1281SetCad                             0x08003cad   Thumb Code    20  sx1281_driver.o(i.SX1281SetCad)
    SX1281SetCadParams                       0x08003cc5   Thumb Code    20  sx1281_driver.o(i.SX1281SetCadParams)
    SX1281SetCrcPolynomial                   0x08003cdd   Thumb Code    36  sx1281_driver.o(i.SX1281SetCrcPolynomial)
    SX1281SetCrcSeed                         0x08003d05   Thumb Code    36  sx1281_driver.o(i.SX1281SetCrcSeed)
    SX1281SetDioIrqParams                    0x08003d2d   Thumb Code    54  sx1281_driver.o(i.SX1281SetDioIrqParams)
    SX1281SetFs                              0x08003d65   Thumb Code    20  sx1281_driver.o(i.SX1281SetFs)
    SX1281SetInterruptMode                   0x08003d7d   Thumb Code     8  sx1281_driver.o(i.SX1281SetInterruptMode)
    SX1281SetLongPreamble                    0x08003d89   Thumb Code    14  sx1281_driver.o(i.SX1281SetLongPreamble)
    SX1281SetModulationParams                0x08003d99   Thumb Code   142  sx1281_driver.o(i.SX1281SetModulationParams)
    SX1281SetPacketParams                    0x08003e2d   Thumb Code   212  sx1281_driver.o(i.SX1281SetPacketParams)
    SX1281SetPacketType                      0x08003f05   Thumb Code    22  sx1281_driver.o(i.SX1281SetPacketType)
    SX1281SetPayload                         0x08003f21   Thumb Code    10  sx1281_driver.o(i.SX1281SetPayload)
    SX1281SetPollingMode                     0x08003f2d   Thumb Code     8  sx1281_driver.o(i.SX1281SetPollingMode)
    SX1281SetRegistersDefault                0x08003f39   Thumb Code    32  sx1281_driver.o(i.SX1281SetRegistersDefault)
    SX1281SetRegulatorMode                   0x08003f5d   Thumb Code    14  sx1281_driver.o(i.SX1281SetRegulatorMode)
    SX1281SetRfFrequency                     0x08003f6d   Thumb Code    46  sx1281_driver.o(i.SX1281SetRfFrequency)
    SX1281SetRx                              0x08003fa1   Thumb Code    44  sx1281_driver.o(i.SX1281SetRx)
    SX1281SetRxDutyCycle                     0x08003fd1   Thumb Code    44  sx1281_driver.o(i.SX1281SetRxDutyCycle)
    SX1281SetSaveContext                     0x08004001   Thumb Code    10  sx1281_driver.o(i.SX1281SetSaveContext)
    SX1281SetSleep                           0x0800400d   Thumb Code    50  sx1281_driver.o(i.SX1281SetSleep)
    SX1281SetStandby                         0x08004045   Thumb Code    30  sx1281_driver.o(i.SX1281SetStandby)
    SX1281SetSyncWord                        0x08004069   Thumb Code   104  sx1281_driver.o(i.SX1281SetSyncWord)
    SX1281SetSyncWordErrorTolerance          0x080040d5   Thumb Code    34  sx1281_driver.o(i.SX1281SetSyncWordErrorTolerance)
    SX1281SetTx                              0x080040f9   Thumb Code    44  sx1281_driver.o(i.SX1281SetTx)
    SX1281SetTxContinuousPreamble            0x08004129   Thumb Code    10  sx1281_driver.o(i.SX1281SetTxContinuousPreamble)
    SX1281SetTxContinuousWave                0x08004133   Thumb Code    10  sx1281_driver.o(i.SX1281SetTxContinuousWave)
    SX1281SetTxParams                        0x0800413d   Thumb Code    24  sx1281_driver.o(i.SX1281SetTxParams)
    SX1281SetWhiteningSeed                   0x08004155   Thumb Code    26  sx1281_driver.o(i.SX1281SetWhiteningSeed)
    SX1281_BSPInit                           0x08004175   Thumb Code    14  sx1281_header.o(i.SX1281_BSPInit)
    SX1281_Callback                          0x08004185   Thumb Code   126  sx1281.o(i.SX1281_Callback)
    SX1281_GetState                          0x0800429d   Thumb Code    20  sx1281.o(i.SX1281_GetState)
    SX1281_Init                              0x080042b5   Thumb Code   492  sx1281.o(i.SX1281_Init)
    SX1281_Running                           0x08004581   Thumb Code    24  sx1281.o(i.SX1281_Running)
    SX1281_SetTX                             0x08004599   Thumb Code    36  sx1281.o(i.SX1281_SetTX)
    SpiIn                                    0x080045c9   Thumb Code    18  sx1281_driver_spi.o(i.SpiIn)
    SpiInOut                                 0x080045e1   Thumb Code    26  sx1281_driver_spi.o(i.SpiInOut)
    SpiInit                                  0x08004601   Thumb Code    26  sx1281_driver_spi.o(i.SpiInit)
    SysTick_Handler                          0x08004625   Thumb Code     4  stm32f1xx_it.o(i.SysTick_Handler)
    SystemClock_Config                       0x08004629   Thumb Code    96  main.o(i.SystemClock_Config)
    SystemInit                               0x08004689   Thumb Code     2  system_stm32f1xx.o(i.SystemInit)
    TIM_Base_SetConfig                       0x0800468d   Thumb Code   108  stm32f1xx_hal_tim.o(i.TIM_Base_SetConfig)
    TIM_ETR_SetConfig                        0x08004705   Thumb Code    20  stm32f1xx_hal_tim.o(i.TIM_ETR_SetConfig)
    TIM_OC2_SetConfig                        0x08004779   Thumb Code    84  stm32f1xx_hal_tim.o(i.TIM_OC2_SetConfig)
    UART_Start_Receive_DMA                   0x08004bad   Thumb Code   130  stm32f1xx_hal_uart.o(i.UART_Start_Receive_DMA)
    USART2_IRQHandler                        0x08004cb1   Thumb Code    18  stm32f1xx_it.o(i.USART2_IRQHandler)
    USAR_UART_IDLECallback                   0x08004cc9   Thumb Code   102  usart.o(i.USAR_UART_IDLECallback)
    USER_UART_IRQHandler                     0x08004d59   Thumb Code    46  usart.o(i.USER_UART_IRQHandler)
    UsageFault_Handler                       0x08004da9   Thumb Code     2  stm32f1xx_it.o(i.UsageFault_Handler)
    __0printf                                0x08004dad   Thumb Code    22  printfa.o(i.__0printf)
    __1printf                                0x08004dad   Thumb Code     0  printfa.o(i.__0printf)
    __2printf                                0x08004dad   Thumb Code     0  printfa.o(i.__0printf)
    __c89printf                              0x08004dad   Thumb Code     0  printfa.o(i.__0printf)
    printf                                   0x08004dad   Thumb Code     0  printfa.o(i.__0printf)
    __scatterload_copy                       0x08004ded   Thumb Code    14  handlers.o(i.__scatterload_copy)
    __scatterload_null                       0x08004dfb   Thumb Code     2  handlers.o(i.__scatterload_null)
    __scatterload_zeroinit                   0x08004dfd   Thumb Code    14  handlers.o(i.__scatterload_zeroinit)
    fputc                                    0x08005697   Thumb Code    24  sx1281_header.o(i.fputc)
    free                                     0x080056b1   Thumb Code    76  malloc.o(i.free)
    main                                     0x08005701   Thumb Code   134  main.o(i.main)
    malloc                                   0x080057a1   Thumb Code    92  malloc.o(i.malloc)
    AHBPrescTable                            0x08005836   Data          16  system_stm32f1xx.o(.constdata)
    APBPrescTable                            0x08005846   Data           8  system_stm32f1xx.o(.constdata)
    bleConfigList                            0x08005868   Data           9  sx1281.o(.constdata)
    loraConfigList                           0x08005871   Data          24  sx1281.o(.constdata)
    gfskConfigList                           0x08005889   Data          12  sx1281.o(.constdata)
    flrcConfigList                           0x08005895   Data          12  sx1281.o(.constdata)
    RadioRegsInit                            0x080058a2   Data           4  sx1281_driver.o(.constdata)
    Radio                                    0x080058a8   Data         228  sx1281_driver_hal.o(.constdata)
    ascii_1608                               0x0800598c   Data        1520  lcd.o(.constdata)
    ascii_2412                               0x08005f7c   Data        4560  lcd.o(.constdata)
    ascii_3216                               0x0800714c   Data        6080  lcd.o(.constdata)
    logo_M                                   0x0800890c   Data         512  lcd.o(.constdata)
    Region$$Table$$Base                      0x08008b0c   Number         0  anon$$obj.o(Region$$Table)
    Region$$Table$$Limit                     0x08008b2c   Number         0  anon$$obj.o(Region$$Table)
    uwTickFreq                               0x20000000   Data           1  stm32f1xx_hal.o(.data)
    uwTickPrio                               0x20000004   Data           4  stm32f1xx_hal.o(.data)
    uwTick                                   0x20000008   Data           4  stm32f1xx_hal.o(.data)
    SystemCoreClock                          0x2000000c   Data           4  system_stm32f1xx.o(.data)
    radioRXSize                              0x20000010   Data           1  sx1281.o(.data)
    sx1281_state                             0x20000011   Data           1  sx1281.o(.data)
    RxIrqMask                                0x20000012   Data           2  sx1281.o(.data)
    TxIrqMask                                0x20000014   Data           2  sx1281.o(.data)
    Callbacks                                0x20000018   Data          32  sx1281.o(.data)
    DioIrq                                   0x20000040   Data           4  sx1281_driver.o(.data)
    __stdout                                 0x2000004c   Data           4  stdout.o(.data)
    __microlib_freelist                      0x20000050   Data           4  mvars.o(.data)
    __microlib_freelist_initialised          0x20000054   Data           4  mvars.o(.data)
    radio                                    0x20000058   Data         320  main.o(.bss)
    hspi1                                    0x20000198   Data          88  spi.o(.bss)
    hspi2                                    0x200001f0   Data          88  spi.o(.bss)
    hdma_spi1_tx                             0x20000248   Data          68  spi.o(.bss)
    hdma_spi1_rx                             0x2000028c   Data          68  spi.o(.bss)
    hdma_spi2_tx                             0x200002d0   Data          68  spi.o(.bss)
    htim1                                    0x20000314   Data          72  tim.o(.bss)
    huart1                                   0x2000035c   Data          72  usart.o(.bss)
    huart2                                   0x200003a4   Data          72  usart.o(.bss)
    hdma_usart2_rx                           0x200003ec   Data          68  usart.o(.bss)
    hdma_usart2_tx                           0x20000430   Data          68  usart.o(.bss)
    uart_buffer                              0x20000474   Data         255  usart.o(.bss)
    uart_data                                0x20000573   Data         255  usart.o(.bss)
    radioRXBuffer                            0x20000672   Data         255  sx1281.o(.bss)
    __heap_base                              0x20002858   Data           0  startup_stm32f103xb.o(HEAP)
    __heap_limit                             0x20002a58   Data           0  startup_stm32f103xb.o(HEAP)
    __initial_sp                             0x20002e58   Data           0  startup_stm32f103xb.o(STACK)



==============================================================================

Memory Map of the image

  Image Entry point : 0x080000ed

  Load Region LR_IROM1 (Base: 0x08000000, Size: 0x00008b84, Max: 0x00010000, ABSOLUTE)

    Execution Region ER_IROM1 (Exec base: 0x08000000, Load base: 0x08000000, Size: 0x00008b2c, Max: 0x00010000, ABSOLUTE)

    Exec Addr    Load Addr    Size         Type   Attr      Idx    E Section Name        Object

    0x08000000   0x08000000   0x000000ec   Data   RO            3    RESET               startup_stm32f103xb.o
    0x080000ec   0x080000ec   0x00000000   Code   RO         4629  * .ARM.Collect$$$$00000000  mc_w.l(entry.o)
    0x080000ec   0x080000ec   0x00000004   Code   RO         4961    .ARM.Collect$$$$00000001  mc_w.l(entry2.o)
    0x080000f0   0x080000f0   0x00000004   Code   RO         4964    .ARM.Collect$$$$00000004  mc_w.l(entry5.o)
    0x080000f4   0x080000f4   0x00000000   Code   RO         4966    .ARM.Collect$$$$00000008  mc_w.l(entry7b.o)
    0x080000f4   0x080000f4   0x00000000   Code   RO         4968    .ARM.Collect$$$$0000000A  mc_w.l(entry8b.o)
    0x080000f4   0x080000f4   0x00000008   Code   RO         4969    .ARM.Collect$$$$0000000B  mc_w.l(entry9a.o)
    0x080000fc   0x080000fc   0x00000004   Code   RO         4976    .ARM.Collect$$$$0000000E  mc_w.l(entry12b.o)
    0x08000100   0x08000100   0x00000000   Code   RO         4971    .ARM.Collect$$$$0000000F  mc_w.l(entry10a.o)
    0x08000100   0x08000100   0x00000000   Code   RO         4973    .ARM.Collect$$$$00000011  mc_w.l(entry11a.o)
    0x08000100   0x08000100   0x00000004   Code   RO         4962    .ARM.Collect$$$$00002712  mc_w.l(entry2.o)
    0x08000104   0x08000104   0x00000024   Code   RO            4    .text               startup_stm32f103xb.o
    0x08000128   0x08000128   0x00000020   Code   RO         4632    .text               mc_w.l(llushr.o)
    0x08000148   0x08000148   0x00000024   Code   RO         4634    .text               mc_w.l(memcpya.o)
    0x0800016c   0x0800016c   0x00000024   Code   RO         4636    .text               mc_w.l(memseta.o)
    0x08000190   0x08000190   0x00000012   Code   RO         4640    .text               mc_w.l(strcpy.o)
    0x080001a2   0x080001a2   0x000000e4   Code   RO         4945    .text               mf_w.l(dmul.o)
    0x08000286   0x08000286   0x000000de   Code   RO         4947    .text               mf_w.l(ddiv.o)
    0x08000364   0x08000364   0x00000022   Code   RO         4949    .text               mf_w.l(dflti.o)
    0x08000386   0x08000386   0x0000001a   Code   RO         4951    .text               mf_w.l(dfltui.o)
    0x080003a0   0x080003a0   0x00000032   Code   RO         4953    .text               mf_w.l(dfixui.o)
    0x080003d2   0x080003d2   0x0000002c   Code   RO         4978    .text               mc_w.l(uidiv.o)
    0x080003fe   0x080003fe   0x00000062   Code   RO         4980    .text               mc_w.l(uldiv.o)
    0x08000460   0x08000460   0x00000000   Code   RO         4990    .text               mc_w.l(iusefp.o)
    0x08000460   0x08000460   0x000000ba   Code   RO         4993    .text               mf_w.l(depilogue.o)
    0x0800051a   0x0800051a   0x0000014e   Code   RO         4995    .text               mf_w.l(dadd.o)
    0x08000668   0x08000668   0x00000030   Code   RO         4997    .text               mf_w.l(dfixul.o)
    0x08000698   0x08000698   0x00000030   Code   RO         4999    .text               mf_w.l(cdrcmple.o)
    0x080006c8   0x080006c8   0x00000024   Code   RO         5001    .text               mc_w.l(init.o)
    0x080006ec   0x080006ec   0x0000001e   Code   RO         5003    .text               mc_w.l(llshl.o)
    0x0800070a   0x0800070a   0x00000024   Code   RO         5005    .text               mc_w.l(llsshr.o)
    0x0800072e   0x0800072e   0x00000002   PAD
    0x08000730   0x08000730   0x0000001c   Code   RO         4146    i.BSP_SPI_GetHandle  spi_1.o
    0x0800074c   0x0800074c   0x00000018   Code   RO         4147    i.BSP_SPI_GetState  spi_1.o
    0x08000764   0x08000764   0x0000001c   Code   RO         4153    i.BSP_SPI_RegisterCallback  spi_1.o
    0x08000780   0x08000780   0x0000002a   Code   RO         4154    i.BSP_SPI_Transmit  spi_1.o
    0x080007aa   0x080007aa   0x0000002e   Code   RO         4155    i.BSP_SPI_TransmitReceive  spi_1.o
    0x080007d8   0x080007d8   0x00000010   Code   RO         4279    i.BSP_UART_GetHandle  uart.o
    0x080007e8   0x080007e8   0x00000002   Code   RO          400    i.BusFault_Handler  stm32f1xx_it.o
    0x080007ea   0x080007ea   0x00000002   PAD
    0x080007ec   0x080007ec   0x0000000c   Code   RO          401    i.DMA1_Channel2_IRQHandler  stm32f1xx_it.o
    0x080007f8   0x080007f8   0x0000000c   Code   RO          402    i.DMA1_Channel3_IRQHandler  stm32f1xx_it.o
    0x08000804   0x08000804   0x0000000c   Code   RO          403    i.DMA1_Channel5_IRQHandler  stm32f1xx_it.o
    0x08000810   0x08000810   0x0000000c   Code   RO          404    i.DMA1_Channel6_IRQHandler  stm32f1xx_it.o
    0x0800081c   0x0800081c   0x0000000c   Code   RO          405    i.DMA1_Channel7_IRQHandler  stm32f1xx_it.o
    0x08000828   0x08000828   0x0000002a   Code   RO         1286    i.DMA_SetConfig     stm32f1xx_hal_dma.o
    0x08000852   0x08000852   0x00000002   Code   RO          406    i.DebugMon_Handler  stm32f1xx_it.o
    0x08000854   0x08000854   0x00000008   Code   RO          407    i.EXTI15_10_IRQHandler  stm32f1xx_it.o
    0x0800085c   0x0800085c   0x00000018   Code   RO          408    i.EXTI9_5_IRQHandler  stm32f1xx_it.o
    0x08000874   0x08000874   0x00000004   Code   RO           13    i.Error_Handler     main.o
    0x08000878   0x08000878   0x00000030   Code   RO         3784    i.GpioGetBitPos     sx1281_driver_gpio.o
    0x080008a8   0x080008a8   0x00000002   Code   RO         3785    i.GpioInit          sx1281_driver_gpio.o
    0x080008aa   0x080008aa   0x00000004   Code   RO         3787    i.GpioRead          sx1281_driver_gpio.o
    0x080008ae   0x080008ae   0x00000002   PAD
    0x080008b0   0x080008b0   0x00000038   Code   RO         3788    i.GpioSetIrq        sx1281_driver_gpio.o
    0x080008e8   0x080008e8   0x00000006   Code   RO         3789    i.GpioWrite         sx1281_driver_gpio.o
    0x080008ee   0x080008ee   0x00000046   Code   RO         1287    i.HAL_DMA_Abort     stm32f1xx_hal_dma.o
    0x08000934   0x08000934   0x00000098   Code   RO         1288    i.HAL_DMA_Abort_IT  stm32f1xx_hal_dma.o
    0x080009cc   0x080009cc   0x00000154   Code   RO         1292    i.HAL_DMA_IRQHandler  stm32f1xx_hal_dma.o
    0x08000b20   0x08000b20   0x0000005c   Code   RO         1293    i.HAL_DMA_Init      stm32f1xx_hal_dma.o
    0x08000b7c   0x08000b7c   0x00000070   Code   RO         1297    i.HAL_DMA_Start_IT  stm32f1xx_hal_dma.o
    0x08000bec   0x08000bec   0x00000024   Code   RO          913    i.HAL_Delay         stm32f1xx_hal.o
    0x08000c10   0x08000c10   0x0000002c   Code   RO         4089    i.HAL_GPIO_EXTI_Callback  gpio_1.o
    0x08000c3c   0x08000c3c   0x00000018   Code   RO         1222    i.HAL_GPIO_EXTI_IRQHandler  stm32f1xx_hal_gpio.o
    0x08000c54   0x08000c54   0x000001e0   Code   RO         1223    i.HAL_GPIO_Init     stm32f1xx_hal_gpio.o
    0x08000e34   0x08000e34   0x0000000a   Code   RO         1225    i.HAL_GPIO_ReadPin  stm32f1xx_hal_gpio.o
    0x08000e3e   0x08000e3e   0x0000000a   Code   RO         1227    i.HAL_GPIO_WritePin  stm32f1xx_hal_gpio.o
    0x08000e48   0x08000e48   0x0000000c   Code   RO          917    i.HAL_GetTick       stm32f1xx_hal.o
    0x08000e54   0x08000e54   0x0000006e   Code   RO         2858    i.HAL_HalfDuplex_Init  stm32f1xx_hal_uart.o
    0x08000ec2   0x08000ec2   0x00000002   PAD
    0x08000ec4   0x08000ec4   0x00000010   Code   RO          923    i.HAL_IncTick       stm32f1xx_hal.o
    0x08000ed4   0x08000ed4   0x00000024   Code   RO          924    i.HAL_Init          stm32f1xx_hal.o
    0x08000ef8   0x08000ef8   0x00000040   Code   RO          925    i.HAL_InitTick      stm32f1xx_hal.o
    0x08000f38   0x08000f38   0x0000003c   Code   RO          524    i.HAL_MspInit       stm32f1xx_hal_msp.o
    0x08000f74   0x08000f74   0x0000001a   Code   RO         1383    i.HAL_NVIC_EnableIRQ  stm32f1xx_hal_cortex.o
    0x08000f8e   0x08000f8e   0x00000002   PAD
    0x08000f90   0x08000f90   0x00000040   Code   RO         1389    i.HAL_NVIC_SetPriority  stm32f1xx_hal_cortex.o
    0x08000fd0   0x08000fd0   0x00000024   Code   RO         1390    i.HAL_NVIC_SetPriorityGrouping  stm32f1xx_hal_cortex.o
    0x08000ff4   0x08000ff4   0x0000012c   Code   RO         1081    i.HAL_RCC_ClockConfig  stm32f1xx_hal_rcc.o
    0x08001120   0x08001120   0x00000020   Code   RO         1088    i.HAL_RCC_GetPCLK1Freq  stm32f1xx_hal_rcc.o
    0x08001140   0x08001140   0x00000020   Code   RO         1089    i.HAL_RCC_GetPCLK2Freq  stm32f1xx_hal_rcc.o
    0x08001160   0x08001160   0x00000054   Code   RO         1090    i.HAL_RCC_GetSysClockFreq  stm32f1xx_hal_rcc.o
    0x080011b4   0x080011b4   0x00000320   Code   RO         1093    i.HAL_RCC_OscConfig  stm32f1xx_hal_rcc.o
    0x080014d4   0x080014d4   0x00000038   Code   RO         4157    i.HAL_SPI_ErrorCallback  spi_1.o
    0x0800150c   0x0800150c   0x00000006   Code   RO          593    i.HAL_SPI_GetState  stm32f1xx_hal_spi.o
    0x08001512   0x08001512   0x000000b2   Code   RO          595    i.HAL_SPI_Init      stm32f1xx_hal_spi.o
    0x080015c4   0x080015c4   0x00000138   Code   RO          245    i.HAL_SPI_MspInit   spi.o
    0x080016fc   0x080016fc   0x00000038   Code   RO         4158    i.HAL_SPI_RxCpltCallback  spi_1.o
    0x08001734   0x08001734   0x00000038   Code   RO         4159    i.HAL_SPI_RxHalfCpltCallback  spi_1.o
    0x0800176c   0x0800176c   0x00000166   Code   RO          603    i.HAL_SPI_Transmit  stm32f1xx_hal_spi.o
    0x080018d2   0x080018d2   0x000001f0   Code   RO          604    i.HAL_SPI_TransmitReceive  stm32f1xx_hal_spi.o
    0x08001ac2   0x08001ac2   0x00000002   PAD
    0x08001ac4   0x08001ac4   0x00000110   Code   RO          605    i.HAL_SPI_TransmitReceive_DMA  stm32f1xx_hal_spi.o
    0x08001bd4   0x08001bd4   0x000000cc   Code   RO          607    i.HAL_SPI_Transmit_DMA  stm32f1xx_hal_spi.o
    0x08001ca0   0x08001ca0   0x00000024   Code   RO         4160    i.HAL_SPI_TxCpltCallback  spi_1.o
    0x08001cc4   0x08001cc4   0x00000038   Code   RO         4161    i.HAL_SPI_TxHalfCpltCallback  spi_1.o
    0x08001cfc   0x08001cfc   0x00000038   Code   RO         4162    i.HAL_SPI_TxRxCpltCallback  spi_1.o
    0x08001d34   0x08001d34   0x00000038   Code   RO         4163    i.HAL_SPI_TxRxHalfCpltCallback  spi_1.o
    0x08001d6c   0x08001d6c   0x00000028   Code   RO         1394    i.HAL_SYSTICK_Config  stm32f1xx_hal_cortex.o
    0x08001d94   0x08001d94   0x00000054   Code   RO         2592    i.HAL_TIMEx_ConfigBreakDeadTime  stm32f1xx_hal_tim_ex.o
    0x08001de8   0x08001de8   0x00000068   Code   RO         2608    i.HAL_TIMEx_MasterConfigSynchronization  stm32f1xx_hal_tim_ex.o
    0x08001e50   0x08001e50   0x0000005a   Code   RO         1885    i.HAL_TIM_Base_Init  stm32f1xx_hal_tim.o
    0x08001eaa   0x08001eaa   0x00000002   PAD
    0x08001eac   0x08001eac   0x00000028   Code   RO          293    i.HAL_TIM_Base_MspInit  tim.o
    0x08001ed4   0x08001ed4   0x000000dc   Code   RO         1894    i.HAL_TIM_ConfigClockSource  stm32f1xx_hal_tim.o
    0x08001fb0   0x08001fb0   0x0000004c   Code   RO          294    i.HAL_TIM_MspPostInit  tim.o
    0x08001ffc   0x08001ffc   0x000000cc   Code   RO         1957    i.HAL_TIM_PWM_ConfigChannel  stm32f1xx_hal_tim.o
    0x080020c8   0x080020c8   0x0000005a   Code   RO         1960    i.HAL_TIM_PWM_Init  stm32f1xx_hal_tim.o
    0x08002122   0x08002122   0x00000002   Code   RO         1962    i.HAL_TIM_PWM_MspInit  stm32f1xx_hal_tim.o
    0x08002124   0x08002124   0x00000002   Code   RO         2868    i.HAL_UARTEx_RxEventCallback  stm32f1xx_hal_uart.o
    0x08002126   0x08002126   0x00000070   Code   RO         2880    i.HAL_UART_DMAStop  stm32f1xx_hal_uart.o
    0x08002196   0x08002196   0x00000002   PAD
    0x08002198   0x08002198   0x00000028   Code   RO         4287    i.HAL_UART_ErrorCallback  uart.o
    0x080021c0   0x080021c0   0x0000026c   Code   RO         2885    i.HAL_UART_IRQHandler  stm32f1xx_hal_uart.o
    0x0800242c   0x0800242c   0x00000064   Code   RO         2886    i.HAL_UART_Init     stm32f1xx_hal_uart.o
    0x08002490   0x08002490   0x00000118   Code   RO          341    i.HAL_UART_MspInit  usart.o
    0x080025a8   0x080025a8   0x0000001c   Code   RO         2890    i.HAL_UART_Receive_DMA  stm32f1xx_hal_uart.o
    0x080025c4   0x080025c4   0x00000028   Code   RO         4288    i.HAL_UART_RxCpltCallback  uart.o
    0x080025ec   0x080025ec   0x00000028   Code   RO         4289    i.HAL_UART_RxHalfCpltCallback  uart.o
    0x08002614   0x08002614   0x000000a0   Code   RO         2894    i.HAL_UART_Transmit  stm32f1xx_hal_uart.o
    0x080026b4   0x080026b4   0x00000028   Code   RO         4290    i.HAL_UART_TxCpltCallback  uart.o
    0x080026dc   0x080026dc   0x00000002   Code   RO          409    i.HardFault_Handler  stm32f1xx_it.o
    0x080026de   0x080026de   0x00000052   Code   RO         4382    i.LCD_Clear         lcd.o
    0x08002730   0x08002730   0x00000080   Code   RO         4383    i.LCD_DrawBitmap    lcd.o
    0x080027b0   0x080027b0   0x00000164   Code   RO         4384    i.LCD_DrawChar      lcd.o
    0x08002914   0x08002914   0x0000005c   Code   RO         4389    i.LCD_DrawPoint     lcd.o
    0x08002970   0x08002970   0x0000006e   Code   RO         4393    i.LCD_DrawString    lcd.o
    0x080029de   0x080029de   0x00000002   PAD
    0x080029e0   0x080029e0   0x00000160   Code   RO         4394    i.LCD_Init          lcd.o
    0x08002b40   0x08002b40   0x00000064   Code   RO         4395    i.LCD_SetAddressWindow  lcd.o
    0x08002ba4   0x08002ba4   0x00000040   Code   RO         4396    i.LCD_WriteCommand  lcd.o
    0x08002be4   0x08002be4   0x00000040   Code   RO         4397    i.LCD_WriteData     lcd.o
    0x08002c24   0x08002c24   0x00000050   Code   RO         4398    i.LCD_WriteDataBuffer  lcd.o
    0x08002c74   0x08002c74   0x00000050   Code   RO         4399    i.LCD_WriteDataBuffer_DMA  lcd.o
    0x08002cc4   0x08002cc4   0x0000003a   Code   RO         3790    i.MSP_GetIRQn       sx1281_driver_gpio.o
    0x08002cfe   0x08002cfe   0x00000002   PAD
    0x08002d00   0x08002d00   0x0000006c   Code   RO          220    i.MX_DMA_Init       dma.o
    0x08002d6c   0x08002d6c   0x00000118   Code   RO          196    i.MX_GPIO_Init      gpio.o
    0x08002e84   0x08002e84   0x00000048   Code   RO          246    i.MX_SPI1_Init      spi.o
    0x08002ecc   0x08002ecc   0x00000048   Code   RO          247    i.MX_SPI2_Init      spi.o
    0x08002f14   0x08002f14   0x000000c4   Code   RO          295    i.MX_TIM1_Init      tim.o
    0x08002fd8   0x08002fd8   0x00000038   Code   RO          342    i.MX_USART1_UART_Init  usart.o
    0x08003010   0x08003010   0x00000038   Code   RO          343    i.MX_USART2_UART_Init  usart.o
    0x08003048   0x08003048   0x00000002   Code   RO          410    i.MemManage_Handler  stm32f1xx_it.o
    0x0800304a   0x0800304a   0x00000002   Code   RO          411    i.NMI_Handler       stm32f1xx_it.o
    0x0800304c   0x0800304c   0x00000014   Code   RO         3258    i.OnRxDone          sx1281.o
    0x08003060   0x08003060   0x00000014   Code   RO         3259    i.OnRxError         sx1281.o
    0x08003074   0x08003074   0x00000014   Code   RO         3260    i.OnRxTimeout       sx1281.o
    0x08003088   0x08003088   0x00000014   Code   RO         3261    i.OnTxDone          sx1281.o
    0x0800309c   0x0800309c   0x00000014   Code   RO         3262    i.OnTxTimeout       sx1281.o
    0x080030b0   0x080030b0   0x00000002   Code   RO          412    i.PendSV_Handler    stm32f1xx_it.o
    0x080030b2   0x080030b2   0x00000022   Code   RO          623    i.SPI_DMAError      stm32f1xx_hal_spi.o
    0x080030d4   0x080030d4   0x0000000a   Code   RO          624    i.SPI_DMAHalfReceiveCplt  stm32f1xx_hal_spi.o
    0x080030de   0x080030de   0x0000000a   Code   RO          625    i.SPI_DMAHalfTransmitCplt  stm32f1xx_hal_spi.o
    0x080030e8   0x080030e8   0x0000000a   Code   RO          626    i.SPI_DMAHalfTransmitReceiveCplt  stm32f1xx_hal_spi.o
    0x080030f2   0x080030f2   0x0000006a   Code   RO          627    i.SPI_DMAReceiveCplt  stm32f1xx_hal_spi.o
    0x0800315c   0x0800315c   0x00000064   Code   RO          629    i.SPI_DMATransmitCplt  stm32f1xx_hal_spi.o
    0x080031c0   0x080031c0   0x0000005a   Code   RO          630    i.SPI_DMATransmitReceiveCplt  stm32f1xx_hal_spi.o
    0x0800321a   0x0800321a   0x0000005c   Code   RO          632    i.SPI_EndRxTransaction  stm32f1xx_hal_spi.o
    0x08003276   0x08003276   0x00000034   Code   RO          633    i.SPI_EndRxTxTransaction  stm32f1xx_hal_spi.o
    0x080032aa   0x080032aa   0x00000002   PAD
    0x080032ac   0x080032ac   0x00000024   Code   RO         4164    i.SPI_Get           spi_1.o
    0x080032d0   0x080032d0   0x000000b8   Code   RO          638    i.SPI_WaitFlagStateUntilTimeout  stm32f1xx_hal_spi.o
    0x08003388   0x08003388   0x00000002   Code   RO          413    i.SVC_Handler       stm32f1xx_it.o
    0x0800338a   0x0800338a   0x0000003e   Code   RO         3451    i.SX1281Calibrate   sx1281_driver.o
    0x080033c8   0x080033c8   0x00000018   Code   RO         3452    i.SX1281ClearIrqStatus  sx1281_driver.o
    0x080033e0   0x080033e0   0x0000001a   Code   RO         3453    i.SX1281GetFirmwareVersion  sx1281_driver.o
    0x080033fa   0x080033fa   0x00000002   PAD
    0x080033fc   0x080033fc   0x00000098   Code   RO         3454    i.SX1281GetFrequencyError  sx1281_driver.o
    0x08003494   0x08003494   0x00000014   Code   RO         3456    i.SX1281GetIrqStatus  sx1281_driver.o
    0x080034a8   0x080034a8   0x0000003c   Code   RO         3457    i.SX1281GetLoRaBandwidth  sx1281_driver.o
    0x080034e4   0x080034e4   0x0000000c   Code   RO         3458    i.SX1281GetOpMode   sx1281_driver.o
    0x080034f0   0x080034f0   0x00000214   Code   RO         3459    i.SX1281GetPacketStatus  sx1281_driver.o
    0x08003704   0x08003704   0x0000000c   Code   RO         3460    i.SX1281GetPacketType  sx1281_driver.o
    0x08003710   0x08003710   0x00000028   Code   RO         3461    i.SX1281GetPayload  sx1281_driver.o
    0x08003738   0x08003738   0x00000022   Code   RO         3462    i.SX1281GetRssiInst  sx1281_driver.o
    0x0800375a   0x0800375a   0x00000002   PAD
    0x0800375c   0x0800375c   0x00000048   Code   RO         3463    i.SX1281GetRxBufferStatus  sx1281_driver.o
    0x080037a4   0x080037a4   0x00000018   Code   RO         3464    i.SX1281GetStatus   sx1281_driver.o
    0x080037bc   0x080037bc   0x00000024   Code   RO         3860    i.SX1281HalGetDioStatus  sx1281_driver_hal.o
    0x080037e0   0x080037e0   0x00000012   Code   RO         3861    i.SX1281HalInit     sx1281_driver_hal.o
    0x080037f2   0x080037f2   0x00000002   PAD
    0x080037f4   0x080037f4   0x00000010   Code   RO         3862    i.SX1281HalIoIrqInit  sx1281_driver_hal.o
    0x08003804   0x08003804   0x0000006c   Code   RO         3863    i.SX1281HalReadBuffer  sx1281_driver_hal.o
    0x08003870   0x08003870   0x0000006c   Code   RO         3864    i.SX1281HalReadCommand  sx1281_driver_hal.o
    0x080038dc   0x080038dc   0x00000010   Code   RO         3865    i.SX1281HalReadRegister  sx1281_driver_hal.o
    0x080038ec   0x080038ec   0x00000070   Code   RO         3866    i.SX1281HalReadRegisters  sx1281_driver_hal.o
    0x0800395c   0x0800395c   0x00000034   Code   RO         3867    i.SX1281HalReset    sx1281_driver_hal.o
    0x08003990   0x08003990   0x0000001c   Code   RO         3868    i.SX1281HalWaitOnBusy  sx1281_driver_hal.o
    0x080039ac   0x080039ac   0x00000048   Code   RO         3869    i.SX1281HalWriteBuffer  sx1281_driver_hal.o
    0x080039f4   0x080039f4   0x00000058   Code   RO         3870    i.SX1281HalWriteCommand  sx1281_driver_hal.o
    0x08003a4c   0x08003a4c   0x0000000c   Code   RO         3871    i.SX1281HalWriteRegister  sx1281_driver_hal.o
    0x08003a58   0x08003a58   0x00000050   Code   RO         3872    i.SX1281HalWriteRegisters  sx1281_driver_hal.o
    0x08003aa8   0x08003aa8   0x00000010   Code   RO         3465    i.SX1281Init        sx1281_driver.o
    0x08003ab8   0x08003ab8   0x00000014   Code   RO         3466    i.SX1281OnDioIrq    sx1281_driver.o
    0x08003acc   0x08003acc   0x0000014c   Code   RO         3468    i.SX1281ProcessIrqs  sx1281_driver.o
    0x08003c18   0x08003c18   0x00000012   Code   RO         3469    i.SX1281SendPayload  sx1281_driver.o
    0x08003c2a   0x08003c2a   0x0000000e   Code   RO         3470    i.SX1281SetAutoFS   sx1281_driver.o
    0x08003c38   0x08003c38   0x0000001a   Code   RO         3471    i.SX1281SetAutoTx   sx1281_driver.o
    0x08003c52   0x08003c52   0x00000034   Code   RO         3472    i.SX1281SetBleAccessAddress  sx1281_driver.o
    0x08003c86   0x08003c86   0x00000002   PAD
    0x08003c88   0x08003c88   0x0000000c   Code   RO         3473    i.SX1281SetBleAdvertizerAccessAddress  sx1281_driver.o
    0x08003c94   0x08003c94   0x00000016   Code   RO         3474    i.SX1281SetBufferBaseAddresses  sx1281_driver.o
    0x08003caa   0x08003caa   0x00000002   PAD
    0x08003cac   0x08003cac   0x00000018   Code   RO         3475    i.SX1281SetCad      sx1281_driver.o
    0x08003cc4   0x08003cc4   0x00000018   Code   RO         3476    i.SX1281SetCadParams  sx1281_driver.o
    0x08003cdc   0x08003cdc   0x00000028   Code   RO         3477    i.SX1281SetCrcPolynomial  sx1281_driver.o
    0x08003d04   0x08003d04   0x00000028   Code   RO         3478    i.SX1281SetCrcSeed  sx1281_driver.o
    0x08003d2c   0x08003d2c   0x00000036   Code   RO         3479    i.SX1281SetDioIrqParams  sx1281_driver.o
    0x08003d62   0x08003d62   0x00000002   PAD
    0x08003d64   0x08003d64   0x00000018   Code   RO         3480    i.SX1281SetFs       sx1281_driver.o
    0x08003d7c   0x08003d7c   0x0000000c   Code   RO         3481    i.SX1281SetInterruptMode  sx1281_driver.o
    0x08003d88   0x08003d88   0x0000000e   Code   RO         3482    i.SX1281SetLongPreamble  sx1281_driver.o
    0x08003d96   0x08003d96   0x00000002   PAD
    0x08003d98   0x08003d98   0x00000094   Code   RO         3483    i.SX1281SetModulationParams  sx1281_driver.o
    0x08003e2c   0x08003e2c   0x000000d8   Code   RO         3484    i.SX1281SetPacketParams  sx1281_driver.o
    0x08003f04   0x08003f04   0x0000001c   Code   RO         3485    i.SX1281SetPacketType  sx1281_driver.o
    0x08003f20   0x08003f20   0x0000000a   Code   RO         3486    i.SX1281SetPayload  sx1281_driver.o
    0x08003f2a   0x08003f2a   0x00000002   PAD
    0x08003f2c   0x08003f2c   0x0000000c   Code   RO         3487    i.SX1281SetPollingMode  sx1281_driver.o
    0x08003f38   0x08003f38   0x00000024   Code   RO         3488    i.SX1281SetRegistersDefault  sx1281_driver.o
    0x08003f5c   0x08003f5c   0x0000000e   Code   RO         3489    i.SX1281SetRegulatorMode  sx1281_driver.o
    0x08003f6a   0x08003f6a   0x00000002   PAD
    0x08003f6c   0x08003f6c   0x00000034   Code   RO         3490    i.SX1281SetRfFrequency  sx1281_driver.o
    0x08003fa0   0x08003fa0   0x00000030   Code   RO         3491    i.SX1281SetRx       sx1281_driver.o
    0x08003fd0   0x08003fd0   0x00000030   Code   RO         3492    i.SX1281SetRxDutyCycle  sx1281_driver.o
    0x08004000   0x08004000   0x0000000a   Code   RO         3493    i.SX1281SetSaveContext  sx1281_driver.o
    0x0800400a   0x0800400a   0x00000002   PAD
    0x0800400c   0x0800400c   0x00000038   Code   RO         3494    i.SX1281SetSleep    sx1281_driver.o
    0x08004044   0x08004044   0x00000024   Code   RO         3495    i.SX1281SetStandby  sx1281_driver.o
    0x08004068   0x08004068   0x0000006c   Code   RO         3496    i.SX1281SetSyncWord  sx1281_driver.o
    0x080040d4   0x080040d4   0x00000022   Code   RO         3497    i.SX1281SetSyncWordErrorTolerance  sx1281_driver.o
    0x080040f6   0x080040f6   0x00000002   PAD
    0x080040f8   0x080040f8   0x00000030   Code   RO         3498    i.SX1281SetTx       sx1281_driver.o
    0x08004128   0x08004128   0x0000000a   Code   RO         3499    i.SX1281SetTxContinuousPreamble  sx1281_driver.o
    0x08004132   0x08004132   0x0000000a   Code   RO         3500    i.SX1281SetTxContinuousWave  sx1281_driver.o
    0x0800413c   0x0800413c   0x00000018   Code   RO         3501    i.SX1281SetTxParams  sx1281_driver.o
    0x08004154   0x08004154   0x00000020   Code   RO         3502    i.SX1281SetWhiteningSeed  sx1281_driver.o
    0x08004174   0x08004174   0x0000000e   Code   RO         4048    i.SX1281_BSPInit    sx1281_header.o
    0x08004182   0x08004182   0x00000002   PAD
    0x08004184   0x08004184   0x00000118   Code   RO         3263    i.SX1281_Callback   sx1281.o
    0x0800429c   0x0800429c   0x00000018   Code   RO         3264    i.SX1281_GetState   sx1281.o
    0x080042b4   0x080042b4   0x000002cc   Code   RO         3265    i.SX1281_Init       sx1281.o
    0x08004580   0x08004580   0x00000018   Code   RO         3266    i.SX1281_Running    sx1281.o
    0x08004598   0x08004598   0x00000030   Code   RO         3277    i.SX1281_SetTX      sx1281.o
    0x080045c8   0x080045c8   0x00000018   Code   RO         3976    i.SpiIn             sx1281_driver_spi.o
    0x080045e0   0x080045e0   0x00000020   Code   RO         3977    i.SpiInOut          sx1281_driver_spi.o
    0x08004600   0x08004600   0x00000024   Code   RO         3978    i.SpiInit           sx1281_driver_spi.o
    0x08004624   0x08004624   0x00000004   Code   RO          414    i.SysTick_Handler   stm32f1xx_it.o
    0x08004628   0x08004628   0x00000060   Code   RO           14    i.SystemClock_Config  main.o
    0x08004688   0x08004688   0x00000002   Code   RO         3220    i.SystemInit        system_stm32f1xx.o
    0x0800468a   0x0800468a   0x00000002   PAD
    0x0800468c   0x0800468c   0x00000078   Code   RO         1978    i.TIM_Base_SetConfig  stm32f1xx_hal_tim.o
    0x08004704   0x08004704   0x00000014   Code   RO         1989    i.TIM_ETR_SetConfig  stm32f1xx_hal_tim.o
    0x08004718   0x08004718   0x00000010   Code   RO         1990    i.TIM_ITRx_SetConfig  stm32f1xx_hal_tim.o
    0x08004728   0x08004728   0x00000050   Code   RO         1991    i.TIM_OC1_SetConfig  stm32f1xx_hal_tim.o
    0x08004778   0x08004778   0x00000058   Code   RO         1992    i.TIM_OC2_SetConfig  stm32f1xx_hal_tim.o
    0x080047d0   0x080047d0   0x00000058   Code   RO         1993    i.TIM_OC3_SetConfig  stm32f1xx_hal_tim.o
    0x08004828   0x08004828   0x00000044   Code   RO         1994    i.TIM_OC4_SetConfig  stm32f1xx_hal_tim.o
    0x0800486c   0x0800486c   0x00000022   Code   RO         1996    i.TIM_TI1_ConfigInputStage  stm32f1xx_hal_tim.o
    0x0800488e   0x0800488e   0x00000024   Code   RO         1998    i.TIM_TI2_ConfigInputStage  stm32f1xx_hal_tim.o
    0x080048b2   0x080048b2   0x00000010   Code   RO         2899    i.UART_DMAAbortOnError  stm32f1xx_hal_uart.o
    0x080048c2   0x080048c2   0x0000004a   Code   RO         2900    i.UART_DMAError     stm32f1xx_hal_uart.o
    0x0800490c   0x0800490c   0x00000086   Code   RO         2901    i.UART_DMAReceiveCplt  stm32f1xx_hal_uart.o
    0x08004992   0x08004992   0x0000001e   Code   RO         2903    i.UART_DMARxHalfCplt  stm32f1xx_hal_uart.o
    0x080049b0   0x080049b0   0x0000004e   Code   RO         2909    i.UART_EndRxTransfer  stm32f1xx_hal_uart.o
    0x080049fe   0x080049fe   0x0000001c   Code   RO         2910    i.UART_EndTxTransfer  stm32f1xx_hal_uart.o
    0x08004a1a   0x08004a1a   0x00000002   PAD
    0x08004a1c   0x08004a1c   0x00000014   Code   RO         4292    i.UART_Get          uart.o
    0x08004a30   0x08004a30   0x000000c2   Code   RO         2911    i.UART_Receive_IT   stm32f1xx_hal_uart.o
    0x08004af2   0x08004af2   0x00000002   PAD
    0x08004af4   0x08004af4   0x000000b8   Code   RO         2912    i.UART_SetConfig    stm32f1xx_hal_uart.o
    0x08004bac   0x08004bac   0x00000090   Code   RO         2913    i.UART_Start_Receive_DMA  stm32f1xx_hal_uart.o
    0x08004c3c   0x08004c3c   0x00000072   Code   RO         2915    i.UART_WaitOnFlagUntilTimeout  stm32f1xx_hal_uart.o
    0x08004cae   0x08004cae   0x00000002   PAD
    0x08004cb0   0x08004cb0   0x00000018   Code   RO          415    i.USART2_IRQHandler  stm32f1xx_it.o
    0x08004cc8   0x08004cc8   0x00000090   Code   RO          344    i.USAR_UART_IDLECallback  usart.o
    0x08004d58   0x08004d58   0x00000050   Code   RO          345    i.USER_UART_IRQHandler  usart.o
    0x08004da8   0x08004da8   0x00000002   Code   RO          416    i.UsageFault_Handler  stm32f1xx_it.o
    0x08004daa   0x08004daa   0x00000002   PAD
    0x08004dac   0x08004dac   0x00000020   Code   RO         4877    i.__0printf         mc_w.l(printfa.o)
    0x08004dcc   0x08004dcc   0x00000020   Code   RO         1396    i.__NVIC_SetPriority  stm32f1xx_hal_cortex.o
    0x08004dec   0x08004dec   0x0000000e   Code   RO         5016    i.__scatterload_copy  mc_w.l(handlers.o)
    0x08004dfa   0x08004dfa   0x00000002   Code   RO         5017    i.__scatterload_null  mc_w.l(handlers.o)
    0x08004dfc   0x08004dfc   0x0000000e   Code   RO         5018    i.__scatterload_zeroinit  mc_w.l(handlers.o)
    0x08004e0a   0x08004e0a   0x00000002   PAD
    0x08004e0c   0x08004e0c   0x00000184   Code   RO         4884    i._fp_digits        mc_w.l(printfa.o)
    0x08004f90   0x08004f90   0x000006b4   Code   RO         4885    i._printf_core      mc_w.l(printfa.o)
    0x08005644   0x08005644   0x00000024   Code   RO         4886    i._printf_post_padding  mc_w.l(printfa.o)
    0x08005668   0x08005668   0x0000002e   Code   RO         4887    i._printf_pre_padding  mc_w.l(printfa.o)
    0x08005696   0x08005696   0x00000018   Code   RO         4049    i.fputc             sx1281_header.o
    0x080056ae   0x080056ae   0x00000002   PAD
    0x080056b0   0x080056b0   0x00000050   Code   RO         4905    i.free              mc_w.l(malloc.o)
    0x08005700   0x08005700   0x000000a0   Code   RO           15    i.main              main.o
    0x080057a0   0x080057a0   0x0000006c   Code   RO         4906    i.malloc            mc_w.l(malloc.o)
    0x0800580c   0x0800580c   0x0000000c   Code   RO         3979    i.tx_cplt_cb        sx1281_driver_spi.o
    0x08005818   0x08005818   0x0000000c   Code   RO         3980    i.txrx_cplt_cb      sx1281_driver_spi.o
    0x08005824   0x08005824   0x00000012   Data   RO         1094    .constdata          stm32f1xx_hal_rcc.o
    0x08005836   0x08005836   0x00000010   Data   RO         3221    .constdata          system_stm32f1xx.o
    0x08005846   0x08005846   0x00000008   Data   RO         3222    .constdata          system_stm32f1xx.o
    0x0800584e   0x0800584e   0x00000002   PAD
    0x08005850   0x08005850   0x00000051   Data   RO         3280    .constdata          sx1281.o
    0x080058a1   0x080058a1   0x00000001   PAD
    0x080058a2   0x080058a2   0x00000004   Data   RO         3503    .constdata          sx1281_driver.o
    0x080058a6   0x080058a6   0x00000002   PAD
    0x080058a8   0x080058a8   0x000000e4   Data   RO         3874    .constdata          sx1281_driver_hal.o
    0x0800598c   0x0800598c   0x00002f80   Data   RO         4400    .constdata          lcd.o
    0x0800890c   0x0800890c   0x00000200   Data   RO         4401    .constdata          lcd.o
    0x08008b0c   0x08008b0c   0x00000020   Data   RO         5014    Region$$Table       anon$$obj.o


    Execution Region RW_IRAM1 (Exec base: 0x20000000, Load base: 0x08008b2c, Size: 0x00002e58, Max: 0x00005000, ABSOLUTE)

    Exec Addr    Load Addr    Size         Type   Attr      Idx    E Section Name        Object

    0x20000000   0x08008b2c   0x0000000c   Data   RW          931    .data               stm32f1xx_hal.o
    0x2000000c   0x08008b38   0x00000004   Data   RW         3223    .data               system_stm32f1xx.o
    0x20000010   0x08008b3c   0x00000028   Data   RW         3281    .data               sx1281.o
    0x20000038   0x08008b64   0x00000010   Data   RW         3504    .data               sx1281_driver.o
    0x20000048   0x08008b74   0x00000001   Data   RW         3981    .data               sx1281_driver_spi.o
    0x20000049   0x08008b75   0x00000001   Data   RW         4402    .data               lcd.o
    0x2000004a   0x08008b76   0x00000002   PAD
    0x2000004c   0x08008b78   0x00000004   Data   RW         4977    .data               mc_w.l(stdout.o)
    0x20000050   0x08008b7c   0x00000004   Data   RW         4982    .data               mc_w.l(mvars.o)
    0x20000054   0x08008b80   0x00000004   Data   RW         4983    .data               mc_w.l(mvars.o)
    0x20000058        -       0x00000140   Zero   RW           16    .bss                main.o
    0x20000198        -       0x0000017c   Zero   RW          248    .bss                spi.o
    0x20000314        -       0x00000048   Zero   RW          296    .bss                tim.o
    0x2000035c        -       0x00000316   Zero   RW          346    .bss                usart.o
    0x20000672        -       0x000000ff   Zero   RW         3279    .bss                sx1281.o
    0x20000771   0x08008b84   0x00000003   PAD
    0x20000774        -       0x00000040   Zero   RW         3791    .bss                sx1281_driver_gpio.o
    0x200007b4        -       0x00001ffe   Zero   RW         3873    .bss                sx1281_driver_hal.o
    0x200027b2   0x08008b84   0x00000002   PAD
    0x200027b4        -       0x00000040   Zero   RW         4090    .bss                gpio_1.o
    0x200027f4        -       0x00000040   Zero   RW         4165    .bss                spi_1.o
    0x20002834        -       0x00000024   Zero   RW         4293    .bss                uart.o
    0x20002858        -       0x00000200   Zero   RW            2    HEAP                startup_stm32f103xb.o
    0x20002a58        -       0x00000400   Zero   RW            1    STACK               startup_stm32f103xb.o


==============================================================================

Image component sizes


      Code (inc. data)   RO Data    RW Data    ZI Data      Debug   Object Name

       108          4          0          0          0        714   dma.o
       280         22          0          0          0        915   gpio.o
        44          4          0          0         64       1109   gpio_1.o
      1508        100      12672          1          0      11090   lcd.o
       260         26          0          0        320     448893   main.o
       456         48          0          0        380       2365   spi.o
       576         68          0          0         64       7837   spi_1.o
        36          8        236          0       1536        764   startup_stm32f103xb.o
       164         28          0         12          0       5601   stm32f1xx_hal.o
       198         14          0          0          0      28723   stm32f1xx_hal_cortex.o
       808         36          0          0          0       4726   stm32f1xx_hal_dma.o
       524         40          0          0          0       3922   stm32f1xx_hal_gpio.o
        60          8          0          0          0        798   stm32f1xx_hal_msp.o
      1248         86         18          0          0       4924   stm32f1xx_hal_rcc.o
      2202         38          0          0          0      12928   stm32f1xx_hal_spi.o
      1156         32          0          0          0      10388   stm32f1xx_hal_tim.o
       188         12          0          0          0       2036   stm32f1xx_hal_tim_ex.o
      2128         24          0          0          0      13304   stm32f1xx_hal_uart.o
       136         36          0          0          0       6889   stm32f1xx_it.o
      1192        430         81         40        255      20229   sx1281.o
      2794        170          4         16          0      27979   sx1281_driver.o
       174          6          0          0         64       5169   sx1281_driver_gpio.o
       746         84        228          0       8190      10942   sx1281_driver_hal.o
       116         30          0          1          0       2741   sx1281_driver_spi.o
        38          0          0          0          0        905   sx1281_header.o
         2          0         24          4          0       1007   system_stm32f1xx.o
       312         30          0          0         72       2172   tim.o
       196         34          0          0         36       3612   uart.o
       616        118          0          0        790       3691   usart.o

    ----------------------------------------------------------------------
     18322       1536      13300         76      11776     646373   Object Totals
         0          0         32          0          0          0   (incl. Generated)
        56          0          5          2          5          0   (incl. Padding)

    ----------------------------------------------------------------------

      Code (inc. data)   RO Data    RW Data    ZI Data      Debug   Library Member Name

         0          0          0          0          0          0   entry.o
         0          0          0          0          0          0   entry10a.o
         0          0          0          0          0          0   entry11a.o
         4          0          0          0          0          0   entry12b.o
         8          4          0          0          0          0   entry2.o
         4          0          0          0          0          0   entry5.o
         0          0          0          0          0          0   entry7b.o
         0          0          0          0          0          0   entry8b.o
         8          4          0          0          0          0   entry9a.o
        30          0          0          0          0          0   handlers.o
        36          8          0          0          0         68   init.o
         0          0          0          0          0          0   iusefp.o
        30          0          0          0          0         68   llshl.o
        36          0          0          0          0         68   llsshr.o
        32          0          0          0          0         68   llushr.o
       188         20          0          0          0        160   malloc.o
        36          0          0          0          0         68   memcpya.o
        36          0          0          0          0        108   memseta.o
         0          0          0          8          0          0   mvars.o
      2218         90          0          0          0        464   printfa.o
         0          0          0          4          0          0   stdout.o
        18          0          0          0          0         68   strcpy.o
        44          0          0          0          0         80   uidiv.o
        98          0          0          0          0         92   uldiv.o
        48          0          0          0          0         68   cdrcmple.o
       334          0          0          0          0        148   dadd.o
       222          0          0          0          0        100   ddiv.o
       186          0          0          0          0        176   depilogue.o
        50          0          0          0          0         76   dfixui.o
        48          0          0          0          0         68   dfixul.o
        34          0          0          0          0         76   dflti.o
        26          0          0          0          0         76   dfltui.o
       228          0          0          0          0         96   dmul.o

    ----------------------------------------------------------------------
      4006        126          0         12          0       2196   Library Totals
         4          0          0          0          0          0   (incl. Padding)

    ----------------------------------------------------------------------

      Code (inc. data)   RO Data    RW Data    ZI Data      Debug   Library Name

      2826        126          0         12          0       1312   mc_w.l
      1176          0          0          0          0        884   mf_w.l

    ----------------------------------------------------------------------
      4006        126          0         12          0       2196   Library Totals

    ----------------------------------------------------------------------

==============================================================================


      Code (inc. data)   RO Data    RW Data    ZI Data      Debug   

     22328       1662      13300         88      11776     636085   Grand Totals
     22328       1662      13300         88      11776     636085   ELF Image Totals
     22328       1662      13300         88          0          0   ROM Totals

==============================================================================

    Total RO  Size (Code + RO Data)                35628 (  34.79kB)
    Total RW  Size (RW Data + ZI Data)             11864 (  11.59kB)
    Total ROM Size (Code + RO Data + RW Data)      35716 (  34.88kB)

==============================================================================

